:100000005446495312280125000008000000000052
:10001000000000800100000058919D0700001000C2
:100020000000000000000000400000000000000090
:1000300000000000010000000000000000000000BF
:10004000544643530000100000D50100E65B6E5C8F
:10005000000001200101100007011000090110003B
:100060000B0110000D0110000F0110001F01100006
:100070001F0110001F0110001F01100011011000CE
:10008000130110001F01100015011000D3361000DD
:10009000CF3710001901100019011000E57111008F
:1000A00019011000E7121000ED12100019011000E4
:1000B000190110004333100019011000F312100051
:1000C000E7381000F90210004D1F10001901100050
:1000D0000000000000000000000000000000000020
:1000E0000000000000000000000000000000000010
:1000F0000000000000000000000000000000000000
:1001000000000000000000000000000000000000EF
:1001100000000000000000000000000000000000DF
:1001200000000000000000000000000000000000CF
:1001300000000000000000000000000000000000BF
:1001400000000000000000000000000000000000AF
:1001500000F010F8FEE7FEE7FEE7FEE7FEE7FEE749
:10016000FEE7FEE7FEE7FEE701480047FEE7FEE7A1
:100170001F01100000F002F800F04AF80AA090E811
:10018000000C82448344AAF10107DA4501D100F052
:100190003FF8AFF2090EBAE80F0013F0010F18BFD5
:1001A000FB1A43F001031847108D0100308D010048
:1001B0000A4410F8014B14F00F0508BF10F8015B5A
:1001C000240908BF10F8014B6D1E05D010F8013B43
:1001D0006D1E01F8013BF9D1641E03D0641E01F8C5
:1001E000015BFBD19142E4D370470000002300245F
:1001F00000250026103A28BF78C1FBD8520728BF37
:1002000030C148BF0B6070471FB51FBD10B510BD92
:10021000DFF80CD0FFF7F8FF04F020FC16F0FDFF2C
:100220000000012003B4FFF7F1FF03BC16F0FCFF50
:1002300000210028D8BF704700BF491C8842FBDC62
:100240007047704770477047704770477047017834
:10025000002908BF704710F8011F0029FBD1704723
:1002600082B0010F8DF80010C0F303618DF801100A
:10027000C0F303518DF80210C0F303418DF8031051
:10028000C0F303318DF80410C0F303218DF805107D
:10029000C0F303118DF8061000F00F008DF8070071
:1002A00000206A46115C0A2934BF303137311154BD
:1002B000401CC0B2082828BF0020F3D3401CC0B2A5
:1002C0000828FBD302B0704782B001098DF80010F6
:1002D00000F00F008DF8010000206A46115C0A2929
:1002E00034BF303137311154401CC0B2022828BF0E
:1002F0000020F3D3401CC0B20228FBD302B07047E9
:1003000082B0010B8DF80010C0F303218DF80110AD
:10031000C0F303118DF8021000F00F008DF80300F8
:1003200000206A46115C0A2934BF3031373111543C
:10033000401CC0B2042828BF0020F3D3401CC0B228
:100340000428FBD302B0704712484FF6FF710160DA
:1003500070471048104A0021016012681020506157
:100360000E48012203685A6003684022DA6003687D
:100370004FF40C621A6102685161026840F6FF7125
:1003800011620068EA21016305A010F8011F00292D
:10039000FBD1704700700020E4861100D486110064
:1003A00055415254204F50454E21210D0D00000063
:1003B0000B0ACAB2F849D1F800C0CCF81C0043F4CB
:1003C000FE400B6858610868006840F00103086847
:1003D00003600868C06810F0010FFAD008688068F0
:1003E0000B6840F00100986002F07F024FF400407B
:1003F00040EA022208684261086800680B6840F021
:10040000010018600868C06810F0010FFAD0086891
:1004100080680B6840F001009860086842610868D5
:1004200000680A6840F0010010600868C06810F0B9
:10043000010FFAD0086880680A6840F001009060F7
:1004400008688069C0B2704700F07F0041EA00216F
:10045000D1480268516101680968026841F00101F0
:1004600011600168C96811F0010FFAD0016889684C
:10047000006841F001018160704700F07F014FF496
:10048000004040EA0122C44801684A6101680968E5
:10049000036841F0010119600168C96811F0010F9A
:1004A000FAD001688968036841F001019960016828
:1004B0004A6101680968026841F001011160016840
:1004C000C96811F0010FFAD001688968026841F02B
:1004D0000101916000688069C0B2704710B58C4618
:1004E0000446FFF7CAFF20EA0C01E0B2BDE8104065
:1004F000AAE7704770B5A848002401210268C2F835
:10050000141302686FF0FE21C2F8201302689921CB
:10051000C2F8301300680321C161A048A04DA14E6C
:1005200000684FF0010390F8800190B935F823007E
:10053000C0F307217F20FFF787FFF01890F8C0165F
:1005400015F82300FFF780FF5B1CB3F5A67FEDDBFA
:1005500070BD35F82300C0F3072C644505D0644610
:100560000CF00F017F20FFF76FFFF01890F8C01616
:1005700015F82300FFF768FF5B1CB3F5A67FE8DBE7
:1005800070BD10B504F072FA834B84464FF004300E
:100590001968086219680014486219680120086126
:1005A000196888601968486000217F20FFF74CFFB8
:1005B00040210120FFF748FFBCF1050F18BF10BD17
:1005C00000201968C1F8100310BD734A00B5126805
:1005D0000321D16100284FF000014FF07F0006D0C9
:1005E000FFF732FF032100205DF804EB2CE7FFF753
:1005F0002BFF012100205DF804EB25E7664A00B5DA
:1006000012680321D16100284FF000014FF07F00F4
:1006100006D0FFF719FF012100205DF804EB13E776
:10062000FFF712FF03210020FFF70EFF002108460D
:100630005DF804EB08E7584900B509680320C86174
:1006400000217F20FFF700FF00205DF804EB14E796
:10065000514900B509680320C86100217F20FFF7D8
:10066000F3FE082102205DF804EBEDE64A490A6832
:10067000926C0123096803FA00F010438864704704
:10068000704745490968896D80F001000122801C8E
:1006900002FA00F0084070473F480168496C026860
:1006A00041F4006151640168496C006821F4006103
:1006B00041647047384A012303FA00F000291168A9
:1006C000096C03D0084311680864704721EA0000F0
:1006D000116808647047304900280868C06D0AD066
:1006E0000A6840F00200D0650868C06D096840F0F3
:1006F0001000C86570470A6840F00100D0650868BE
:10070000C06D096840F00800C86570472DE9F043E6
:10071000DFF8849080462025D9F8001009270220B0
:10072000C861002404217F20FFF78EFEA44611E05B
:10073000BCF1030F03D0BCF1060F0BD105E005217E
:100740007F20FFF781FE002404E006217F20FFF7D1
:100750007BFE00240023002D88BF08EB4C1608D92F
:10076000F15C2046FFF770FE601C5B1CC4B29D422A
:10077000F6D80CF1010C6745DAD8D9F80010012041
:10078000C861002404217F20FFF75EFEA446002FED
:100790001CD8BDE8F0830000E8861100E8060020C0
:1007A000000000209C5D0020BCF1030F03D0BCF1D1
:1007B000060F0BD105E005217F20FFF745FE002441
:1007C00004E006217F20FFF73FFE00240023002DD8
:1007D00088BF08EB4C160AD9F01890F82011204673
:1007E000FFF732FE601C5B1CC4B29D42F4D80CF1D2
:1007F000010C6745D8D8CCE770B5D449044603202E
:100800000968C8610425E9B27F20FFF71DFE0023B7
:10081000E1B2D8B2FFF718FE03F12000E1B2C0B296
:10082000FFF712FE03F14000E1B2C0B2FFF70CFE89
:100830005B1C202BECDB0CF087F9002808BF0024A0
:100840006D1C072DDFDB70BDC04803210268D1613C
:1008500002681121C2F8301300684FF00111C0F88E
:10086000201300217F20EFE5B84B00B51968032065
:10087000C86101467F20FFF7E7FD09210320FFF74C
:10088000E3FD01210F20FFF7DFFD19680120C1F80A
:10089000140319689920C1F8300319686FF0FE201D
:1008A000C1F8200303217F20FFF7CEFDFF210020A8
:1008B000FFF7CAFD03210120FFF7C6FD2121052016
:1008C000FFF7C2FD01217F20FFF7BEFD002175204B
:1008D000FFF7BAFD012176205DF804EBB4E59B4BF0
:1008E00000B519680320C86100217F20FFF7ACFD27
:1008F00040210120FFF7A8FD00210320FFF7A4FD00
:1009000002217F20FFF7A0FD15210220FFF79CFDAB
:1009100089210420FFF798FD0F217F20FFF794FD28
:1009200001210320FFF790FD19680120C1F814038D
:1009300019681120C1F8300319684FF00110C1F88F
:10094000200303217F20FFF77FFD01210020FFF717
:100950007BFD00210120FFF777FD21210520FFF716
:1009600073FD04216D20FFF76FFD08216E20FFF756
:100970006BFD10216F20FFF767FD01217F20FFF73E
:1009800063FD08210020FFF75FFD04210120FFF730
:100990005BFD1868406C196840F400604864186892
:1009A000406C196820F40060486400BD2DE9F047F0
:1009B000664E0546012730680024C0F8147304F021
:1009C00055F86FF0FE294FF0990A4FF003080228FE
:1009D00004D004F04BF805281DD028E00CF0B4F842
:1009E00038B130685A4CC0F820933068C0F830A352
:1009F0001DE03068574CC0F81C8031681120C1F8E8
:100A0000300331684FF00110C1F8200300217F202E
:100A1000FFF71AFD0BE009F024FA78B330684C4C6C
:100A2000C0F820933068C0F830A3FFF71DFF30688E
:100A3000406C316840F4006048643068406C316854
:100A400020F40060486404F011F8034630684FF069
:100A50000431016208143168486230680761306807
:100A600087603068476000217F20FFF7EDFC402160
:100A70000120FFF7E9FC052B09D104E0FFE7354C25
:100A8000FFF72DFFD3E731680020C1F8100330686D
:100A9000C0F81C80DFF8C0C001233CF82300C0F37D
:100AA00007217F20FFF7D0FCE95C1CF82300FFF74B
:100AB000CBFC1CB1E118E85C81F8C0065B1CB3F507
:100AC000A67FEADBBDE8F0877047244B00211A4679
:100AD000E0FB03214809C0EB0010800070470020B4
:100AE000704700207047002070470020704708467C
:100AF000704700207047704700207047704770476C
:100B000000207047704770470020704700207047F2
:100B100000207047002070477047704700207047E2
:100B2000704770477047002070470020704770473B
:100B300070477047002070470020704770470020C2
:100B4000704770477047704770470000E886110093
:100B50009C5D0020E2070020000000205BB0055BE8
:100B6000FF4910B509680320C86100217F20FFF705
:100B70006BFC02210020FFF767FC01210220FFF738
:100B800063FC0121BDE810400020FFF75DBCF44983
:100B900010B509680320C86100217F20FFF754FCCD
:100BA00002210020FFF750FC01210220FFF74CFC3E
:100BB0000121BDE810400020FFF746BCE94808B518
:100BC00001684969C1F30721009101684969009AE8
:100BD000C1F307219142F8D0E1480168D1F82C1304
:100BE000006841F00401C0F82C13FFF724FD002831
:100BF00008BF08BD0020BDE80840FFF7FFBCD9488A
:100C000008B501684969C1F3072100910168496984
:100C1000009AC1F307219142F8D0D1480168D1F878
:100C20002C13006841F00401C0F82C13FFF703FDFA
:100C3000002808BF08BD0020BDE80840FFF7DEBC63
:100C400010B503F013FF052809D0C5480068D0F897
:100C50002C0310F0040F0CBF0120002010BDC2486F
:100C60000068006810BD70B50546FFF7E9FF012870
:100C700018BF70BD03F0FAFEB94C0326052827D033
:100C8000FFF7BDFF012D18BF70BD2068406C2168C3
:100C900040F40060486400BF00BF00BF2068406CA3
:100CA000216820F4006048642068C66100217F202C
:100CB000FFF7CAFB02210020FFF7C6FB012102203B
:100CC000FFF7C2FBBDE8704001210020FFF7BCBB6D
:100CD0000020FFF793FCD8E710B5FFF752FC012086
:100CE000FFF7C1FF102004F026FA0121052002F0D1
:100CF0004AFA0121062002F046FA9C490120887038
:100D000010BD10B5602002F094FA602002F084FA61
:100D1000934903200968C86410BD944A014650797C
:100D2000002818BF0120002918BF01215171704708
:100D30008E4A11691061084670478C480021017184
:100D4000C17001898A4816F0CAB98848002101712A
:100D5000C1700189864816F0C2B900B583B0002081
:100D60008DF80000ADF8040003F080FE02281CBFDF
:100D700003B000BD0BF0E8FE02281CBF03B000BDAD
:100D8000012077490968C86103217F20FFF75CFBD8
:100D900089210520FFF758FB67210620FFF754FB48
:100DA00045210720FFF750FB23210820FFF74CFBCC
:100DB00003B0F12109205DF804EBFFF745BB2DE9F5
:100DC000F14F88B0002004464FF0100B02900090C5
:100DD00003F04CFE022806D003F048FE052808BFA9
:100DE00009F03FF801E00BF0AFFE03F03FFE614970
:100DF00005280BD0086890B1012808BF01240ED047
:100E000002280BD0032808BF032408E00868022842
:100E100014BF4FF0360B4FF0000BEBD102245648B5
:100E200056494FF0200900680969406BFF3100F511
:100E3000E03021F0FF01503004FB010512200026B4
:100E4000069001E0032E01D214271AE0F01E0328B9
:100E500038BF152715D3B01F032838BF162710D366
:100E6000A6F10900032838BF24270AD3A6F10C00F5
:100E7000032838BF252704D3A6F10F00032838BF65
:100E800026270298B84209D03548029739090068E8
:100E9000C16107F00F017F20FFF7D6FA0BF054FE77
:100EA00000280CBF4FF07F084FF048080024B9F12C
:100EB000000F35D9380905903148A0FB06104008CD
:100EC000A0EB800000EB060A2E48A0FB06104008AD
:100ED000404200EBC0008119089800EB41100490DB
:100EE000089800EB461003900598012820D0C4F123
:100EF0001F0000EB4A1080B201900122694628468B
:100F000001F0DEF86D1C03F0B1FD02284BD050E07B
:100F1000202C45F10005E7D3601CC4B24C45F7D343
:100F2000701CC6B2069886428CD309B0BDE8F08F1B
:100F300004EB4A1080B2019001226946284601F074
:100F4000BFF86D1C03F092FD022805D10098804582
:100F500002D880384F281BD203F088FD052813E003
:100F6000E886110004871100EC861100300500208E
:100F7000D0100020CC050020A4060020A8060020E8
:100F8000ABAAAAAA398EE33804BF0098FF2801D182
:100F9000CDF800B00098C1B2039801550198C0B2D5
:100FA000FFF752FAB8E70098804502D880384F28FA
:100FB00006D203F05BFD052804BF0098FF2801D18D
:100FC000CDF800B0049800992044C9B280F82011EF
:100FD0000198C0B2FFF738FA9EE7F749C86070473A
:100FE00010B503F043FD052802D0BDE8104006E629
:100FF000FFF726FE012818BF10BD0020BDE81040F5
:10100000FFF7FCBA70472DE9F041064682B00C4666
:101010000120FFF728FE03F029FDE84FE64D4FF0D1
:10102000000824B303F022FD052815D0FFF7E7FDE3
:10103000606800281CBF2168002918D0FFF7B6FCA3
:101040003868C0F82883EE600BF07EFD02280BD0D4
:101050000BF02AFC40B10AE0FFF7F2FD012804BFC3
:101060000020FFF7CBFAE3E7A068FFF7A8FE8DF8B2
:101070000080ADF8048003F0F9FC02281ED10BF0CB
:1010800063FD02281AD139680120C86103217F203D
:10109000FFF7DAF989210520FFF7D6F96721062045
:1010A000FFF7D2F945210720FFF7CEF923210820C9
:1010B000FFF7CAF9F1210920FFF7C6F985F8048086
:1010C00085F803802989BE4816F009F8C5F8108014
:1010D000687900206871602002F0ABF8602002F0AF
:1010E0009BF839680320C86402B0BDE8F081602035
:1010F00002F096B810B5602002F092F8BDE81040FA
:101100000120B0E5AC48C0687047AB4800780028C3
:1011100018BF0120704738B500240094FFF790FDF8
:10112000002818BF38BDA4480471C4700189A448C0
:1011300015F0D5FFDFF884C2DCF80000406CDCF865
:10114000001040F40060486400BFDCF80000406C10
:10115000DCF8001020F4006048649A4D9A48297821
:1011600000290168496914BFC9B2C1F30721009180
:1011700020D001684969009AC9B29142F9D000684B
:101180000221C161DCF80000D0F82C03DCF800106B
:1011900020F00400C1F82C03DCF80000C0F8104374
:1011A000FFF749FA002818BF38BD0120BDE83840D4
:1011B000FFF724BA01684969009AC1F307219142F7
:1011C000F8D0002301684969C9B2009101684969F2
:1011D000009AC9B29142F9D0591CCBB2042BF1D379
:1011E00001212970CBE770B503F040FC0025724C5B
:1011F000052803D02570BDE870408CE7FFF720FD7F
:10120000002818BF70BD2571E57021896C4815F064
:1012100066FF257069480168D1F82C13006821F039
:101220000401C0F82C13BDE870400120FFF7E6B9B7
:10123000614901200870704770B503F017FC5E4CDF
:101240000125052808D0FFF7FBFC002818BF70BD5A
:101250002570BDE870405EE7FFF7F2FC002818BF7C
:1012600070BD00202071E0702189554815F037FFCE
:101270002570BDE870400120FFF7C0B90120F2E4FD
:1012800070B54D4C0025E57003F0F0FB052803D048
:101290002570BDE870403EE7FFF7D2FC002818BF7C
:1012A00070BD2571E5702189454815F018FF25703E
:1012B00042480168D1F82C13006821F00401C0F8FD
:1012C0002C13BDE870400120FFF798B93A4A5169E4
:1012D00050610846704738498861704736488069D0
:1012E0007047354840787047334948707047012847
:1012F00088BF7047354900280868406E04D00968E7
:1013000040F0020048667047096840F001004866F6
:101310007047012888BF70472C4900280868406E34
:1013200004D0096820F0020048667047096820F080
:10133000010048667047002000F0F6BB012000F075
:10134000F3BB10B51C4CE069401CE0611B48016810
:10135000096D006841F004010165FFF79DF9FFF791
:1013600077F9207800281CBF0120FFF77CFC60691A
:10137000002818BF80471648016841F400610160E9
:1013800010BD10B50120FFF76EFCBDE8104000F065
:1013900014BC10487047104870470748006A7047EF
:1013A0000548406A70470448806A70470249002037
:1013B000086248628862704730050020E8861100A4
:1013C000D0100020AA05002004871100E486110037
:1013D00064050020A4100020AD100020F84900EBA7
:1013E000C00001EBC010704748434FF6FF7101EA9F
:1013F0004000F44908817047F34A107051707047FB
:10140000F149085C7047F0B50746A1B020240121DE
:101410000220FFF74FF9ED4D00216E46286830F8A5
:10142000110026F81100491CA142F7D30021022027
:10143000FFF740F901210020FFF73CF90021002CC3
:1014400009D9286806EB410230F81100491CA2F8BE
:1014500040008C42F5D800210846FFF72BF9A20086
:101460006946384615F09AFD21B0F0BD70B50E46BC
:10147000D4490500E0B04FF0800008814FF020040F
:101480004FF001010CBF05200420FFF713F9CF49ED
:1014900000206B46096801EB053101EB800202F583
:1014A0008052D2F800C043F820C003EB800CD2F881
:1014B0008020401CCCF88020A042EED3002D4FF0BD
:1014C000000114BF04200520FFF7F4F8E20069468C
:1014D000304615F063FD60B070BD70B50400B948CA
:1014E0000E464FF0010105890CBF05200420FFF7CF
:1014F000E1F8B6482A46006800EB043000F5805158
:10150000304615F04BFD4FF0000124B1BDE87040AE
:101510000420FFF7CFB8BDE870400520FFF7CAB838
:1015200010B590B020220021009101910291039109
:101530000491059106910791089109910A910B91E7
:101540000C910D910E91EC460F9100EB410430F897
:101550001130B4F8404223442CF81130491CC9B270
:101560009142F2D35200614615F018FD10B010BD43
:10157000F0B5944F954EADF2844D00243D89002C7A
:101580004FF001010CBF05200420FFF793F83068ED
:101590002A4600EB043000F58051684615F043FD03
:1015A000002C4FF000010CBF05200420FFF782F84B
:1015B000641C022CE2DB0020FFF7ABFE0120FFF7EA
:1015C000A8FE0DF2844DF0BD814A824900201368C7
:1015D00003EB8003D3F8C03021F81030401C0728FB
:1015E000F5D31068D0F8E40048827047784A7A4B07
:1015F000002818BF00201DD0116801EB8001D1F830
:1016000080110904090C18BF23F81010401C202871
:10161000F2D30020116801EB8001D1F88012090497
:10162000090C1CBF03EB400CACF84010401C2028F8
:10163000F0D37047116801EB8001D1F80011090463
:10164000090C18BF23F81010401C2028F2D30020EA
:10165000116801EB8001D1F800120904090C1CBFCC
:1016600003EB400CACF84010401C2028F0D370472E
:101670002DE9F84304460020009003F0F7F9012714
:10168000504EDFF84C81534D052809D00BF05CFA21
:101690000028204650D0FEF7F4FF002859D061E022
:1016A00008F0DFFB0228204603D0FEF7EAFF68B30C
:1016B00035E0FEF7E6FF40B984F001042046FEF76E
:1016C000E0FF002808BFBDE8F8833D492046FFF74A
:1016D00004FF0020D8F8001001EB8001D1F8C01001
:1016E00025F81010401C0728F4D3D8F80000D0F8D3
:1016F000E40068822046FFF779FF2046FFF709FEE5
:10170000377184F00100F070BDE8F88384F00104C3
:101710002046FEF7B6FF002808BFBDE8F883284939
:101720002046FFF7DAFE2046FFF7F3FD377184F01D
:101730000100F070BDE8F883FEF7A3FF0028EED1AA
:1017400084F001042046FEF79CFF0028E7D1BDE8A5
:10175000F88384F001042046FEF793FF002808BFB9
:10176000BDE8F88316492046FFF7B7FE0020D8F8F9
:10177000001001EB8001D1F8C01025F81010401CBA
:101780000728F4D3B1E770B50E4D044668790028F8
:1017900004BFE878FFF76CFF2879002808BF70BD08
:1017A000074AAB6902F5A060A0F18001A0610020AA
:1017B000C4E9021020616061C4E90032012070BDFB
:1017C000D010002030050020360500200C871100C5
:1017D000E8861100D015002050150020E8490020AF
:1017E000087170472DE9F14F82B00020009012205F
:1017F0004FF020080025019001E0032D01D21426AE
:101800001AE0E81E032838BF152615D3A81F0328A1
:1018100038BF162610D3A5F10900032838BF2426A7
:101820000AD3A5F10C00032838BF252604D3A5F15F
:101830000F00032838BF26260098B04209D0D148AF
:10184000009631090068C16106F00F017F20FEF7A4
:10185000FBFD0024B8F1000F28D902984FEA161BAF
:1018600000EB451AC848A0FB05104008A0EB80001B
:101870004719C648A0FB05104008404200EBC000D5
:101880000299284401EB4019BBF1010F16D0C4F1B5
:101890001F0000EB471080B2FEF7EFFD09EB0401DB
:1018A00081F82001601CC4B24445EDD3681CC5B268
:1018B00001988542A1D303B0BDE8F08F04EB471037
:1018C00080B2FEF7DAFD0AF80400EBE7012070476A
:1018D0007047002070472DE970431C4616460D46A0
:1018E0008046FFF7ADF95FEA00091CBF0120FFF752
:1018F000BAF92819A84288BF01210FD9002344460C
:10190000B34238BF202C06D201FA04F23A4218BF83
:101910005B1C641CF4E76D1C8542EFD3B9F1000F2A
:1019200008BFBDE87083BDE87043A9E42DE9F04726
:10193000994614460E460746089DFFF781F95FEA6F
:1019400000081CBF0120FFF78EF903F0EDF9DFF866
:1019500040C206EB0903B342CCF8000088BF381937
:1019600013D93C460AE0DCF80010097825F8021B80
:10197000DCF80010491C641CCCF80010844238BF0D
:10198000202CF0D3761C9E42EBD3B8F1000F08BF99
:10199000BDE8F087BDE8F04772E4704710B5FFF787
:1019A000ABF87749488110BD754AC1B200F4706345
:1019B0005289914288BF11464FF0640C01FB0CF133
:1019C000B1FBF2F11A0A02FB0C1189B210F4805F2C
:1019D00012BF08B2484200B270470028B8BF404268
:1019E00080B2B4BF00214FF4805100F47062114303
:1019F000634AC0B25289504341EA1020704708B58B
:101A00000921732000F030F9BDF8001000F01F002C
:101A100021F0FF010843ADF800000D21732000F014
:101A200023F9BDF8001000F01F0021F47F4141EAC6
:101A30000020ADF80000BDF8000008BD7047FFF7BA
:101A400071B854484FF41071006800F5405015F01B
:101A500046BB2DE9F84F12204FF0200800900BF004
:101A600073F8DFF82CB102280CBF4B484B4800F547
:101A700090600024CBF8000001E0032C01DA14266A
:101A80001AE0E01E032838BF152615D3A01F03282F
:101A900038BF162610D3A4F10900032838BF242626
:101AA0000AD3A4F10C00032838BF252604D3A4F1DF
:101AB0000F00032838BF2626B24509D03148310926
:101AC000B2460068C16106F00F017F20FEF7BCFC42
:101AD0000025B8F1000F1EDD31484FEA161980FBD2
:101AE0000410A0EBE070A0EB80000719B9F1010F22
:101AF0000EBF05EB4710C5F11F0000EB4710DBF8E8
:101B00000020C0B212F8011BCBF80020FEF79CFCAD
:101B10006D1C4545EADB0098641C8442ADDBBDE8E2
:101B2000F88F0020FEF7DDBF70B5044601280AD803
:101B30001C48002C0168496E14BF41F0020141F0BD
:101B40000101006841660E4DA869401CA861296921
:101B500000291CBF20468847287800281CBF012088
:101B6000FFF781F80748002C0CBF02210121006813
:101B700001650D48016841F02001016070BD000061
:101B800030050020E8861100ABAAAAAA398EE338F6
:101B9000E00500200C8711009C5D0020E20700207A
:101BA00056555555E4861100640500200549002866
:101BB00014BF0020012008707047704770477047BD
:101BC000704700005C050020704710B501F017FE5B
:101BD000234B244900224C6824B14A6001F014FED2
:101BE000204610BD1878002818BF0A80F3D1088855
:101BF000B0F57A7F87BF30BF0A80401C0880EAE7D3
:101C000010B501F0FCFD17484468002C08BF30BF38
:101C1000FAD00021416001F0F7FD204610BD70B5FB
:101C200001F0EDFD0F4D6C682CB10020686001F0F3
:101C3000EBFD204670BD30BF01F020FB0028F2D044
:101C400001F020FBA860EEE70020704730BF70472E
:101C500072B662B670477047704772B662B6704728
:101C60003406002060050020EE4BC2081B681A6491
:101C700001F0FC0141EA002040F4704040F0804057
:101C800000687047E74BC2081B681A6401F0FC0249
:101C900042EA002040F4704040F08040890700682C
:101CA000C90EC840C0B27047DF4900200870DD4946
:101CB0000E2009680864DD48007810F0800018BF25
:101CC0000120704710B44FEAD00CD64B1C68C4F802
:101CD00040C001F0FC0141EA002040F4704040F0B7
:101CE000804002601868006C10F4007F04BF10BCD4
:101CF000704700BF1868006C10F4007FF9D110BC69
:101D00007047DFF820C310B4DCF800C0C308CCF87B
:101D1000403001F0FC0343EA002343F4704343F0F6
:101D20008043FF24D3F800C08B07DB0E9C402CEAD5
:101D3000040C9A4010BC42EA0C02C3E7BC484FF4C2
:101D4000F4610268116101684968026841F00201AA
:101D500051600068032181617047B54810B5026881
:101D60001021116002684FF4F46111610168496843
:101D7000026841F00201516000680321816107227D
:101D800008217120FFF7BDFF0E2001F02BFABDE8FE
:101D900010400E2001F033BAA24910B50968A548D9
:101DA0000862072201217020FFF7ABFFA048102135
:101DB0000268116002684FF4F461116101684968BA
:101DC000026841F00201516000680321816107222D
:101DD00008217120FFF795FF0E2001F003FABDE8FE
:101DE00010400E2001F00BBA9148002102681160EA
:101DF00002684FF4E0611161006801218161704760
:101E00008B4900200A6810600A68106109688861BF
:101E100070478748062102681160026802215160FC
:101E20000068816170478248002102681160006883
:101E3000816170477E49002009680860704710B5CD
:101E40007B4C0820216808602168022088610722F5
:101E500008217120FFF755FF2068C06810F0080FB7
:101E6000FAD021680F20886010BD10B504460246E4
:101E70000021F020FFF726FF22460121F020FFF786
:101E800021FF22460021F120FFF71CFF22460121FD
:101E9000F120FFF717FF22460021FC20FFF712FF79
:101EA00022460121BDE81040FC200BE74FF4807171
:101EB00041EAD0025B490B681A645F4A42EA002299
:101EC00010600868006C10F4007F08BF704700BF06
:101ED0000868006C10F4007FF9D17047514A4FF444
:101EE000807141EAD00112681164534941EA00202F
:101EF0000068704708227020002102E7002270204D
:101F00001146FEE647480168496E026821F40071F7
:101F100051660168496E026841F48071516601683A
:101F2000496E026841F4806151660168496E00683B
:101F300021F480614166002270201146E1E63948B3
:101F40000168496E026841F4806151660168496E1A
:101F5000026821F4806151660168496E026821F4CB
:101F6000807151660168496E006841F400714166F4
:101F700070472C480168496E026841F480615166DF
:101F80000168496E006821F4806141667047254808
:101F90001B210268116400680164704710B5244C6D
:101FA0002068C0682549086025484FF6FF71006821
:101FB00001602068C06810F0100F0BD019491B2079
:101FC0000A6810640968086420688068216840F025
:101FD000100088602068C06810F0080F05D02068E5
:101FE0008068216840F0080088602068C06810F0B0
:101FF000040F0AD020688068216840F004008860DF
:10200000FF2200217020FFF77CFE2068C06810F0DE
:10201000010F08BF10BD20688068216840F00100F2
:10202000886010BDE48611006C05002000F20040BD
:10203000048711002222A26000F00040EC0600207C
:10204000CC861100704770B5FF4D0446C0F30741C0
:10205000286801F0CEFAC4F30721286801F0C9FA14
:10206000E1B22868BDE8704001F0C3BA2DE9F04143
:10207000F64F0446164638680D46806A396840F0C7
:1020800003008862DFF8C0830321D8F8000001F064
:10209000B0FA2046FFF7D7FF0024002E07D9D8F862
:1020A000000001F0D4FA2855641CA642F7D838681D
:1020B000806A396820F0030088620120BDE8F08161
:1020C00070B514460D46064601F0A3FB224629468C
:1020D0003046BDE87040C9E72DE9F0410024DC4DF1
:1020E000042601F096FB324629462046FFF7BEFF44
:1020F00004242F463D1D264601F08BFB324629461F
:102100002046FFF7B3FF08242D1D042601F081FBB4
:10211000324629462046FFF7A9FF202507F10C0487
:1021200001F077FB324621462846FFF79FFF0C3728
:1021300024243E1D042501F06CFB2A46314620462E
:10214000FFF794FF2824361D01F063FB2A46314631
:102150002046FFF78BFFBF4E07F10C0401F059FB3F
:102160002A4621463046FFF781FF371D25462C1DA4
:10217000042601F04EFB324621463846FFF776FF33
:102180003E1D0424083501F044FB22462946304612
:10219000FFF76CFF4FF4FC342D1D042601F039FBD2
:1021A000324629462046FFF761FF271D2C46251D94
:1021B00001F02FFB324629463846FFF757FFA64F5E
:1021C0002D1D01F026FB324629463846FFF74EFF0B
:1021D0003F1D2D1D01F01DFB324629463846FFF7F5
:1021E00045FF2E1D3F1D042501F013FB2A463146F5
:1021F0003846FFF73BFF351D3F1D042601F009FB64
:10220000324629463846FFF731FF3E1D0425183473
:1022100001F0FFFA2A4621463046FFF727FF8F4E8E
:102220008F4C012501F0F5FA2A4621463046BDE8DB
:10223000F0411BE77047F8B50E0005464FF000046B
:1022400017D0042269462846FFF710FF9DF80000CA
:102250009DF801109DF8032008409DF802101140E0
:102260000840FF2801D00020F8BD641C2D1DB44299
:10227000E7D30120F8BD2DE9F84391460D4680468D
:10228000002401F0C6FA0027B9F1000F88BF6E469E
:1022900019D9042269464046FFF7E8FE0023F05CA6
:1022A000E95C88421CBF601C84B25B1C042BF6D323
:1022B0002D1D7F1C08F104084F45EAD3002C1CBFDC
:1022C0000020BDE8F8830120BDE8F88301207047B5
:1022D00070B55E4C06462068806A216840F00300B5
:1022E0008862594D0521286801F083F9286801F0BA
:1022F000AEF92168896A226821F003019162307089
:10230000012070BD38B5514C2068806A40F003014F
:10231000206881624C4D0521286801F06AF928681F
:1023200001F095F92168896A226821F00301916220
:102330008DF8000010F0010018BF012038BD10B565
:10234000424C2068806A216840F0030088623E4861
:102350000621006801F04DF92068806A216820F0AC
:1023600003008862012010BD70B50546FFF7CAFF63
:1023700000281CBF022070BDFFF7E1FF334C20682E
:10238000806A216840F0030088622F48202100689D
:1023900001F02FF92846FFF756FE2068806A216871
:1023A00020F003008862FFF7ADFF28B100BF00BF37
:1023B000FFF7A8FF0028F9D1012070BD2DE9F84FE3
:1023C0008046032701F025FADFF88090DFF878A037
:1023D000FFF798FF10BBFFF7B2FFD9F80000806A43
:1023E000D9F8001040F0030088622021DAF80000DC
:1023F00001F0FFF84046FFF726FED9F80000806A9A
:10240000D9F8001020F003008862FFF77BFF28B1A5
:1024100000BF00BFFFF776FF0028F9D145464FF413
:1024200080660024042269462846FFF71FFE9DF8B7
:1024300000009DF801109DF8032008409DF802104F
:1024400011400840FF280DE000871100E4861100CC
:10245000F015002068C0010010F8010004300300EE
:102460007005002006D0381EA7F10107B0DC02205D
:10247000BDE8F88F641C2D1DB442D3D30120BDE804
:10248000F88F2DE9F04117460E460446FFF73AFF54
:1024900000281CBF0220BDE8F081FFF750FFDFF8E5
:1024A0000C84D8F80000806AD8F8001040F00300CF
:1024B0008862FF4D0221286801F09BF82046FFF753
:1024C000C2FD0024002F06D9315D286801F091F883
:1024D000641CA742F8D8D8F80000806AD8F8001029
:1024E00020F003008862FFF70DFF28B100BF00BF96
:1024F000FFF708FF0028F9D10120BDE8F0812DE9A0
:10250000F043C1B08846814603276E4601F081F949
:102510004FF4807241464846FFF7B3FF002445461A
:102520004FF4807269464846FFF7A0FD305D295D93
:10253000884205D07F1EE9D241B00220BDE8F08379
:10254000641CB4F5807FF1D341B00120BDE8F08375
:102550002DE9F041D74C0646D44FDFF8548360682C
:10256000C0B00D4650B1D8F8000001F042F86268E2
:10257000FF2AB8BF501C1BDA606035E001F049F952
:10258000FFF7DDFE3868806A396840F00300886232
:102590000221D8F8000001F02CF83046FFF753FD77
:1025A0002946D8F8000001F024F86068401CE3E7F1
:1025B000002060603868806A396820F00300886213
:1025C00000244FF4807269463046FFF74FFD68469D
:1025D0002A5D015D914203D040B00220BDE8F08148
:1025E000641CB4F5807FF3D340B00120BDE8F081D6
:1025F00070B50C46054601F00CF9B4F5807F88BF34
:1026000070BDAA490A68926A096842F003028A62A8
:10261000A7480321006800F0ECFF2846BDE87040A1
:1026200011E5A348006801F012B8A0480168896A62
:10263000006821F003018162704770B50C460546C1
:1026400001F0E7F821462846BDE870404FF480725B
:102650000CE570B5954D04462868806A296840F0FD
:1026600003008862924E9F21306800F0C2FF3068FC
:1026700000F0EDFF2070306800F0E9FF6070306816
:1026800000F0E5FFA0702868806A296820F0030048
:102690008862012070BD70B5044601F0BAF8834D20
:1026A0002868806A296840F003008862804E9F2174
:1026B000306800F09EFF306800F0C9FF207030687D
:1026C00000F0C5FF6070306800F0C1FFA07028689E
:1026D000806A296820F003008862012070BD2DE91E
:1026E000F047DFF8C89104461746D9F8000088463D
:1026F000806AD9F8001040F0030088626C4D032115
:10270000286800F076FF2046FFF79DFC0024B4EB1C
:10271000970F18D2286800F09AFF0646286800F044
:1027200096FF46EA0026286800F091FF46EA004638
:10273000286800F08CFF46EA006048F82400641C1A
:10274000B4EB970FE6D3D9F80000806AD9F80010EF
:1027500020F0030088620120BDE8F08770B51446C0
:102760000D46064601F055F8224629463046BDE89A
:102770007040B4E710B5FFF7C5FD00281CBF02206C
:1027800010BDFFF7DCFD494C2068806A216840F0ED
:102790000300886246486021006800F02AFF206834
:1027A000806A216820F003008862FFF7ABFD28B142
:1027B00000BF00BFFFF7A6FD0028F9D1012010BD22
:1027C00010B501F026F8FFF79DFD00281CBF022080
:1027D00010BDFFF7B4FD354C2068806A216840F0D9
:1027E0000300886232486021006800F002FF206820
:1027F000806A216820F003008862FFF783FD28B11A
:1028000000BF00BFFFF77EFD0028F9D1012010BDF9
:1028100070B50C46054600F0FCFF002600F0F9FFFD
:102820004FF4807221462846FFF720FC761C04F501
:10283000807405F58075102EF0D3012070BD2DE950
:10284000F047C0B08846814600F0E3FF4FF0000A31
:10285000464603276D4600F0DCFF4FF48072314698
:102860004846FFF70EFE00244FF480726946484642
:10287000FFF7FCFB295D305D814205D07F1EEAD267
:1028800040B00220BDE8F087641CB4F5807FF1D32E
:102890000AF1010A08F5807809F58079BAF1100F7C
:1028A000D6D340B00120BDE8F0870000E4861100D7
:1028B00000871100700500202DE9F04F81B005461A
:1028C000ADF5804D000514468846000DEB4633D02B
:1028D0002F466FF30B07BA465E4600F09AFF4FF0A3
:1028E000000900F096FF4FF4807231463846FFF73A
:1028F000BDFB09F1010906F5807607F58077B9F18E
:10290000100FEED3C5F30B00C0F58056A64288BF6A
:10291000264658443246414614F040FB5046FFF7E5
:102920004DFD022850D059465046FFF788FF022837
:102930004CD03544B044A41BB4F5805F19D34FF498
:1029400080524146584614F029FB2846FFF736FDD1
:10295000022839D059462846FFF771FF022835D0A2
:10296000A4F5805405F5805508F58058B4F5805FCE
:10297000E5D21CB3D9462E4600F04BFF002700F0ED
:1029800048FF4FF4807259463046FFF76FFB7F1CBB
:1029900006F580760BF5807B102FF0D3224641465A
:1029A000484614F0FBFA2846FFF708FD02280BD032
:1029B00049462846FFF743FF022807D0012001B00F
:1029C0000DF5804DBDE8F08F0A20F8E70B20F6E703
:1029D00010B5ADF5806D0446AAB1684614F0DEFA74
:1029E0002046FFF7EBFC022802BF0A200DF5806DA0
:1029F00010BD69462046FFF782FD022802BF0B206A
:102A00000DF5806D10BD01200DF5806D10BD70B508
:102A10000646FFF777FC00281CBF022070BDFFF7B9
:102A20008EFCB44C2068806A216840F00300886204
:102A3000B14D0121286800F0DCFD3146286800F026
:102A4000D8FD2068806A216820F003008862FFF7C3
:102A500059FC28B100BF00BFFFF754FC0028F9D192
:102A6000012070BDF8B500F0D4FEA24D2868806A40
:102A7000296840F0030088629F4E0521306800F00D
:102A8000B8FD306800F0E3FD2968896A2A6821F002
:102A90000301916240F040048DF80040FFF732FCE2
:102AA000002818BFF8BDFFF74AFC2868806A29682B
:102AB00040F0030088620121306800F09AFD214651
:102AC000306800F096FD2868806A296820F00300CD
:102AD0008862FFF717FC002808BFF8BD00BF00BFE1
:102AE000FFF710FC0028F9D1F8BD70B505460024A9
:102AF000FFF708FC40B1AC4201D9002070BD641C56
:102B0000FFF700FC0028F6D1012070BD70B5794CAC
:102B100006462068806A216840F003008862764D8E
:102B20000921286800F065FD286800F090FD216803
:102B3000896A226821F0030191623070012070BD22
:102B400038B5FFF7DFFB002836D1FFF7F8FB694CFB
:102B50002068806A40F0030120688162664D2F2161
:102B6000286800F046FD2068806A216820F0030094
:102B70008862FFF7C7FB28B100BF00BFFFF7C2FBA9
:102B80000028F9D12068806A216840F0030088623B
:102B90000921286800F02DFD286800F058FD216803
:102BA000896A226821F0030191628DF8000010F01B
:102BB000020F1CBF012038BD022038BD4E4810B5A1
:102BC0000421006800F015FD012010BD70B5FFF76D
:102BD00099FB00281CBF022070BD464C2068806A0B
:102BE000216840F003008862434D0521286800F009
:102BF00000FD286800F02BFD06462068806A2168E9
:102C000020F0030088622068806A216840F0030099
:102C10008862FFF794FB0121286800F0EAFC26F0A7
:102C20004001286800F0E5FC2068806A216820F0F7
:102C300003008862012070BD70B50546FFF762FB96
:102C400000281CBF022070BDFFF779FB294C2068CB
:102C5000806A216840F0030088622748522100689A
:102C600000F0C7FC2846FFF7EEF92068806A21686B
:102C700020F003008862FFF745FB28B100BF00BFCA
:102C8000FFF740FB0028F9D1012070BD10B50446C4
:102C9000FFF738FB00281CBF022010BDFFF74FFBD9
:102CA0001548D821006800F0A4FC2046FFF7CBF9B6
:102CB00010480168896A006821F003018162FFF70A
:102CC00021FB28B100BF00BFFFF71CFB0028F9D192
:102CD000012010BD084810B5B921006800F089FC3A
:102CE000012010BD044810B5AB21006800F081FC44
:102CF000012010BDE486110000871100012101FAB6
:102D000000F041490A6810430860404909680860BA
:102D10007047012101FA00F03B490A6822EA0000ED
:102D200008603A490968086070473749096821FA1C
:102D300000F000F001007047334A116821FA00F3F7
:102D400013F0010F4FF0010303FA00F02F4B05D0F1
:102D500021EA00001060196808607047084310609D
:102D600019680860704729490968096821FA00F064
:102D700000F00100704725490A685268012309687C
:102D800003FA00F010434860704720490A6852680F
:102D90000123096803FA00F022EA00004860704746
:102DA0001A490A68126A0123096803FA00F01043FD
:102DB0000862704715490A68126A0123096803FA14
:102DC00000F022EA00000862704710490868406875
:102DD0000A6840F001005060086840680A6840F0E6
:102DE00002005060084A106840F0010010600B6853
:102DF0001860106840F0020010600968086004491B
:102E000000200968C860704778050020DC86110042
:102E1000E486110070477047B24810B502683F2140
:102E2000D1600268002191640068C0F8B4100321E9
:102E30000A2000F0A8F9BDE810400A2000F0C7B948
:102E4000A84A13681860136859604843116888607D
:102E50007047A44A1368186013685960484310F01B
:102E6000010F18BF401C1168886070479D490968B0
:102E7000C1F8B40070479B4918B109680120886403
:102E80007047096800208864704796480168C968DF
:102E9000006841F00201C1607047DFF848C210B419
:102EA000DCF800402062DCF800004162DCF8000041
:102EB0008262DCF80000C362DCF8001001200863C5
:102EC000DCF80000406B10F0010F09D000BF00BF1C
:102ED00000BF00BFDCF80000406B10F0010FF5D11F
:102EE00010F0020018BF4FF0FF3010BC70477D4853
:102EF0000168C968006821F00201C1607047794823
:102F00000168C968006841F00101C1607047754BF4
:102F1000D3F800C0CCF820001868416218688262BB
:102F20001968012008641868406C10F0010F08D07F
:102F300000BF00BF00BF00BF1868406C10F0010F59
:102F4000F6D110F0060018BF4FF0FF30704765480B
:102F50000168C968006821F00101C16070476148DB
:102F60000168C968006841F00401C1607047027CD3
:102F7000017B02F03F0241EA02415A4A1368996517
:102F8000136801685962136841689962136881681F
:102F9000D9621368012119651168496D11F0010F9B
:102FA00008D000BF00BF00BF00BF1168496D11F01D
:102FB000010FF6D11368DB6D83821368DB6D1B0C88
:102FC000C38213681B6E038313681B6E1B0C438341
:102FD00013685B6E83831268526EC2F30E42C28323
:102FE00011F0020018BF4FF0FF3070473D480168F4
:102FF000C968006821F00401C160704701684FEAA8
:10300000314238490B68C3F89C200A684068C2F80E
:10301000A0000868C068096840F02000C8607047D8
:10302000304A136818621068416211680120C1F8C3
:1030300090001068D0F8980010F0010F09D000BF80
:1030400000BF00BF00BF1068D0F8980010F0010F5B
:10305000F5D110F0060018BF4FF0FF30704721483F
:103060000168C968006821F02001C16070471D48EF
:103070000168C968006841F01001C1607047A3F1A0
:10308000050C184B10B41C68C4F888C0D3F800C0F5
:10309000CCF8200018684262186881621968012023
:1030A000C1F880001868D0F8840010F0010F09D032
:1030B00000BF00BF00BF00BF1868D0F8840010F048
:1030C000010FF5D110F0060018BF4FF0FF3010BC13
:1030D000704704480168C968006821F01001C160A8
:1030E00070470000F0861100234810B502680121E6
:1030F0001166026810215167026841F206015166AB
:1031000002680021916602680A21C2F888100268EC
:103110009021C2F884100168D1F88410026841F04F
:103120000101C2F8841002684FF4817111660068D1
:103130000166032000F04BF80021032000F023F883
:103140000E49022009688862002010BD10B50320D6
:1031500000F048F808484FF4807102681166026870
:1031600000211166006810218167002010BD04490C
:103170000020087070470000E0861100EC86110006
:103180007C050020704700F00303DA004FF0FF0CCD
:103190000CFA02F24FF0050C0CEBC303994000F05F
:1031A0000C03002808DA30480068184443691140CD
:1031B00093431943416170472C4800681844D0F884
:1031C0000033114093431943C0F80013704700F0D7
:1031D0001F01012202FA01F1244A4009126842F853
:1031E0002010704700F01F01012202FA01F11F4A6E
:1031F0004009126802EB8000C0F88010704700F0B0
:103200001F01012202FA01F1184A4009126802EB7B
:103210008000C0F880117047144909680860704741
:1032200012490968C1F880007047104800680068BA
:1032300070470E490968C1F8800170470A48006864
:103240008068704708490A68926809688860104673
:103250007047054A1268926800F1100352F8230083
:1032600042F8231070470000D0861100CC86110070
:10327000704770477047704770477047002070472D
:103280000020704700207047704770471B4A116844
:10329000106008467047704718484068704710B57E
:1032A00000F0ACF8164804210268C2F888100268E1
:1032B0004FF6FF71C2F88C1072B600684FF40071BF
:1032C000016662B610BD72B60D484FF40031026857
:1032D000116662B60068D0F8040268B14FF6FF715B
:1032E000081A0649074A8860A0F50840B938904294
:1032F0003CBF4FF00110C86000F085B88005002089
:10330000F4861100372B1A001A48016849690268CF
:1033100041F40071516101680969026821F00601F8
:10332000116101680969006841F01001016170478D
:10333000104801680969026821F0060111610168FD
:103340000969026841F004011161016809690068B6
:1033500041F01001016170470649096888607047B3
:10336000BFF34F8F034904480968C860BFF34F8F0C
:10337000FEE70000D08611000400FA05022824BFF1
:1033800000207047874B53F8202043F82010104648
:10339000704770B5844C2068006F824D10F0010FAB
:1033A00006D021680120C8662868002818BF804719
:1033B0002068006F10F0020F08BF70BD0220216866
:1033C000C8666868002808BF70BDBDE87040004747
:1033D000754810B5026802211165036801221A665A
:1033E00003680322DA66006841650920FFF7EFFEF3
:1033F0000221BDE810400920FFF7C5BE6A4902203E
:10340000096808657047684902200968486570477F
:103410000020704764480168096F11F4007F04D0F0
:1034200000684FF440710166704700684FF4807186
:103430000166704710B55C4C2068C06F10F0020F39
:103440004FF0010018BF0320226850670520B1FB30
:10345000F0F022684FF405710009C2F8801014F0F2
:1034600007FB524A524B14F053FB14F0BDFA21688B
:10347000C1F884002068006F10F4007F04D0216838
:103480004FF44070086610BD21684FF480700866E4
:1034900010BD45480168096F11F4807F04D00068B1
:1034A0004FF440710166704700684FF40071016687
:1034B00070473D4B30B41A68D26F12F0010F1DBF38
:1034C0000322D3F800C0CCF874204FF0020C04BFE4
:1034D0001A68C2F874C04FF0020C00EB4005C5EB4F
:1034E000C0104FF49674C1EBC0004C4300EB800059
:1034F000304904EB4010A1FB0010C0080521B0FBCF
:10350000F1F00022B0F5803F05D3511C4008CAB24B
:10351000B0F5803FF9D242EA0C211A6841F010015F
:10352000C2F888101968C1F88C001868006F10F490
:10353000807F05D019684FF44070086630BC704732
:1035400019684FF40070086630BC7047164801686F
:10355000096F11F4003F04D000684FF44031016658
:10356000704700684FF48031016670470E4801686B
:10357000096F11F4803F04D000684FF440310166B8
:10358000704700684FF400310166704706480068D4
:10359000006FC0F30020704703480068006FC0F35D
:1035A0004020704794050020F48611007B14AE473C
:1035B000E17A843FCDCCCCCC30B40025DDE9024C9F
:1035C000056001F00F0141EA8C1101600168D2B27F
:1035D00041EA0221016023F47F4101611021416031
:1035E000416804F0040211436FF3CF11416030BC15
:1035F0007047C26812F0010F18BF8160C16811F0F6
:10360000100FFBD1C16811F0040F08BF704781682B
:10361000C16811F0040FFAD170470023002A0BDDB6
:1036200011F803C0C0F808C0D0F80CC01CF0100F8F
:10363000FAD15B1C9342F3DBC16811F0040F08BFA1
:1036400070478168C16811F0040FFAD17047FF22FA
:10365000C16811F0100FFBD18260C16811F0100F2A
:10366000FBD1C16811F0040FFBD08068C0B2704775
:103670000023002AD8BF704710B4FF24D0F80CC034
:103680001CF0100FFAD18460D0F80CC01CF0100FA1
:10369000FAD1D0F80CC01CF0040FFAD0D0F808C052
:1036A00001F803C05B1C9A42E7DC10BC704741681C
:1036B00041F002016FF3CF1141607047416821F47E
:1036C000C17121F47E41416070470000704702489B
:1036D0000068406870477047E48611002649002062
:1036E0000A6890600968086024494860704710B50E
:1036F000214C216848602168002088600221401E1A
:10370000FFF741FD21680720086010BD1A4900201D
:1037100009680860704719490870704717480078B1
:103720007047164901200870704714488068704738
:103730002DE9F041114C002705466780A0684FF441
:103740007A71B0FBF1F00C4E401E31684860306871
:1037500087600221C81EFFF716FD31680720086048
:103760006188A942FCD330680760BDE8F081044954
:103770004843024988607047C88611009C050020B4
:1037800040420F00704770B52C4C05464FF40D5069
:103790002168886621680320C86621682848486631
:1037A00021684CF27100086621682648C1F8800043
:1037B000216842F24630886602210020FFF7E3FCD0
:1037C0000020FFF704FD002D08BF70BD2068806E4B
:1037D00042F2413108432168886670BD174810B530
:1037E00002680121916700684FF40D518166002045
:1037F000FFF7F8FCBDE810400020FFF700BD0F49BF
:1038000001200968486770470C49012009688867EA
:1038100070470A494CF2710009680866704707480A
:1038200081B04CF27101026811660168096F02688B
:10383000D1660068006F009001B07047D886110013
:1038400007383937009C1C9110B500210A20FEF77B
:1038500045FB8B49887110BD024670200121FEF79F
:1038600050BA024670200021FEF74BBA2DE9F04114
:103870000024254672201421FEF7F6F9064610F0C2
:10388000010F18BF012416F0020F18BF44F0020404
:1038900016F0040F18BF44F0040416F0080F0DD002
:1038A000784844F008040168D1F82C13006841F00E
:1038B0000401C0F82C130020FCF7A0FE16F0100F36
:1038C00018BF44F0100416F0200F6D4F06D044F0DE
:1038D000200400210A20FEF701FBB87124B17020FA
:1038E00001212246FEF70DFA300A10F0010F18BF31
:1038F0001025040A14F0010F4FF0010607D045F01F
:1039000020053E7000210A20FEF7E8FAB871200A6F
:1039100010F0010F1CBF45F040057E7025B17020EE
:1039200000212A46FEF7EDF9B8799C281CBF00203B
:10393000B870BDE8F08199E710B500210A20FEF7C4
:10394000CDFAC0B200224E499C2804BFCA700A704A
:1039500008D0C878401CC0B2C870032882BFCA70A3
:10396000012010BD002010BD10B5454C6079401CF1
:10397000C0B26071142818D900210A20FEF7AEFAEF
:10398000A279C0B20021824204BF217161710CD0C2
:103990006079401E60712079401CC0B220710328FC
:1039A00003D921716171012010BD002010BD10B537
:1039B000C9200021FEF758F9002010BD70B574240D
:1039C000002133222046FEF79CF901210D462A46AC
:1039D0002046FEF796F902212A462046FEF791F985
:1039E00003212A462046FEF78CF970200121772218
:1039F000FEF787F90C20FFF7EAFB00210C20FFF708
:103A0000C2FBC82000211422FEF77BF91C4C0020C9
:103A10000146A0700A20FEF761FAA07170BD70B572
:103A2000FFF7A2FF20B10020FFF773F9FEF787FA36
:103A3000134C00252078B0B100210A20FEF74EFA81
:103A4000C0B29C2804BFE57025700CD0E078401C03
:103A5000C0B2E070032806D9E57025700020FFF79A
:103A600058F9FEF76CFA6078002808BF70BD6570E1
:103A70000020FFF74EF9BDE87040FEF760BA000085
:103A8000A8050020E886110070B5FE4C00254FF413
:103A9000906125706570FC4813F021FB4FF4906134
:103AA000FA4813F01CFB4FF49061F94813F017FB30
:103AB0006560A5708021F74813F011FBBDE87040E8
:103AC0008021F54813F00BBBEE488078002818BF22
:103AD00001207047EB484078002818BF012070474C
:103AE00070B50546ED48EE490078097800FB01F411
:103AF000FFF7A6F9E64A2B46A2F510610846FFF744
:103B0000CCF962002946E24813F048FADD49012069
:103B1000487070BD2DE9F0411D4616460F4680469F
:103B2000069C00F0A3FF022802D109F00DF830B185
:103B300000F09CFF052803D106F093F900B9022498
:103B4000FFF768F921462846FFF783F93A463146E0
:103B50004046FFF7DCF9BDE8F041FFF75CB9C94822
:103B600040687047CF4A10B5127801469200C948A4
:103B700013F014FAC3490120887010BD2DE9F04FED
:103B8000DFF800A3002689B09AF801809AF8027045
:103B9000B346FDF7EDFCC4480168496C026841F486
:103BA0000061516400BF0168496C006821F4006144
:103BB0004164BE490220096808660020FDF7ADF89F
:103BC000FDF711FB05F041FB01280BD06846FDF71E
:103BD000DAFD0028F6D0684605F061FF029870B162
:103BE0001FB10CE04FF0010B69E00146AD480078D1
:103BF0008200A84813F0D2F901208AF80200019847
:103C0000002854D0B8F1000F51D104469AF80000B2
:103C1000A8BBDAF8045095B3A04800780790A048F4
:103C200090F8009000F022FF022802D108F08CFFEB
:103C300030B100F01BFF052804D106F012F908B9D5
:103C40004FF00209FFF7E6F849460798FFF701F938
:103C500021462A460846FFF75AF9FFF7DCF8DFF855
:103C6000509299F80000022804BF284605F0AEFDE6
:103C700099F80000092804BF204605F0A7FD254655
:103C8000864887490078097800FB01F4FFF7D8F8E7
:103C90007F4A2B46A2F510610846FFF7FEF8620046
:103CA00029467B4813F07AF901208AF80100FDF7D4
:103CB00095FD761C042E85D3BBF1000F03D08AF846
:103CC00001808AF802700120FCF7CDFF77480221BD
:103CD0000068016609B05846BDE8F08F69480021C8
:103CE00001704BE738B50F2100F08CFF654C0128BF
:103CF00006D100202070FFF741FF009001F005F889
:103D0000607800281BBFA07800280020012038BD63
:103D10000F2138B500F076FF5A4C012806D100205B
:103D20002070FFF72BFF009000F0EFFF6078002875
:103D30001BBFA07800280020012038BD0021514879
:103D4000417081707047504870475048704770B557
:103D500005464FF490614C4813F0C1F94FF490615F
:103D60004B4813F0BCF9474C29464748227800F0ED
:103D700031FB22782946BDE87040454800F02ABB57
:103D8000F0B4464A404B002114788C4603F5106588
:103D90000022002C13D933F9116030F91170BE42A2
:103DA00053F81160B4BFB61CB61E43F8116033F966
:103DB000116045F81160491C521CA242EBD30CF172
:103DC000010CBCF1020FE3D3F0BC7047002818BF10
:103DD00001202C49487070472DE9F047DFF8A49086
:103DE00082B05FEA00087BD000254FF4107A2C46A1
:103DF00000F03CFE052808BF012505D008F0A4FE10
:103E000000280CBF2B4C2C4C2C482D4F0068796996
:103E1000806BFF3100F5E03021F0FF01503005FBF1
:103E2000010600F023FE022807D108F08DFE20B91C
:103E30007869FF3020F0FF00064400F017FE0228EA
:103E400002D108F081FEE8B300F010FE052802D18F
:103E500006F007F8B0B30025771C3046012269460A
:103E6000FEF72EF97E1C012201A93846FEF728F93B
:103E70000198C1B2009861F31F2000B2414628F8B2
:103E8000150021E0B005002034160020B41A0020EF
:103E9000341F0020B42C0020342D0020BE0500204B
:103EA000BF050020C5050020E8861100E48611004A
:103EB00031060020E20700209C5D0020A4060020BF
:103EC000A806002011E00BE0002C18BF24F8150014
:103ED0006D1C5545C0D30122FE4800F07BFAFD4819
:103EE000C9F8040002B0BDE8F087402300208446F2
:103EF000614628F810C0002C18BF24F81010401C90
:103F00009842F5D301224146F34800F063FAF248A3
:103F1000E6E710B508F018FE02284FF0010207D0BE
:103F2000EE49EC4800F056FAED49EA48486010BD09
:103F3000EC49E84800F04EFAF6E710B5E84C0028E6
:103F400004BF606010BD01220146E24800F042FA61
:103F5000E048606010BDE4487047002818BF0120A9
:103F6000DF4988707047DE49002200284A708A7055
:103F700018BF0120087001E610B54FF44C30142230
:103F8000DA49FEF79DF8D94810BD10B54FF44C3012
:103F90001422D649FEF794F8D448006810BD10B535
:103FA0004FF44C301422D149FEF78AF8CF4810BDA7
:103FB0000268B2F1FF3F15D0052904BFC07A7047EF
:103FC00028DC012904BF00797047022904BF007A68
:103FD0007047032904BF407A7047042904BF807AE0
:103FE000704727E0052913D007DC012922D00229D8
:103FF0001CBF032904290BD01CE0142912BF15296A
:104000002D207047162904BF28207047172911D189
:1040100000207047142904BF007B7047152904BF96
:10402000407B7047162904BF807B7047172904BF67
:10403000C07B7047FF20704770B5C0B000244FF4BC
:104040008071684613F04BF8FF224FF44C36511C38
:10405000684613F01AF8FF21254661F307052D2263
:10406000214662F3070162F30F2128224BF6BB3091
:1040700062F3174164F31F61CDE90005CDE9024108
:1040800004943046FEF722F969463046FEF737FAC7
:1040900040B070BD2DE9F04FC1B00446DDE94A984B
:1040A00093489A4693460D4601602068B0F1FF3F61
:1040B00008BFFFF7C1FFD4E901106BF307006AF3F3
:1040C0000F20266869F31740D4E9037465F30701EC
:1040D00068F31F600D468046FF22511C684612F0AF
:1040E000D4FFCDF80880CDE90374CDE900654FF425
:1040F0004C342046FEF762F969462046FEF7FFF988
:10410000012818BF002041B0BDE8F08F2DE9F04F25
:10411000174688468146C1B000244FF44C30142223
:104120007249FDF7CDFF714B1D68B5F1FF3F02BF2E
:10413000204641B0BDE8F08FFF22D3E902A4511C14
:104140006846D3F810B05E6812F09FFF69F3070469
:1041500068F30F2467F31744012060F31F64CDE96F
:1041600002A4CDE900564FF44C34CDF810B02046EF
:10417000FEF724F969462046FEF7C1F941B0BDE8D3
:10418000F08F2DE9F04F5B4F0024C1B07E42A14675
:104190004FF44C3014225549FDF792FF534D17212F
:1041A00028462B68FFF704FF844614212846FFF7B2
:1041B000FFFE40B2B3F1FF3F04D0BCF1000F09D1C4
:1041C0002D2807D0FFF738FF4FF44C301422474911
:1041D000FDF776FF14212846FFF7EAFE40B2039070
:1041E00015212846FFF7E4FE40B20290162128462A
:1041F000FFF7DEFE40B2019016212846FFF7D8FEF9
:10420000404240B20090FCF77DFF10F0020F79D0E1
:1042100039483B4A4FF0000890F800C03748007812
:104220000028C8BFACF1010A1EDD0021BAF1000F61
:1042300016DD01F1010B01FB00830BFB008B32F853
:10424000133032F81BB0A3EB0B031BB2002BB8BF2B
:104250005B421BB24B45C8BF9946491C5145E8DB40
:1042600008F101088045E0DB02994945B8BF44F0F8
:1042700002044FF00008C246BCF1000FC8BFA0F115
:10428000010B1BDD0021BBF1000F13DD0AFB001346
:1042900032F813E002EB43035B88AEEB03031BB27F
:1042A000002BB8BF5B421BB24345C8BF9846491CB0
:1042B0005945EBDB0AF1010AE245E3DB039941458D
:1042C000B8BF44F004044FF0000ABCF1000F2DDD2C
:1042D000002318E0B423002034280020E207002047
:1042E000B00500209C5D0020B42C0020B42D0020DF
:1042F00070050020F1D8FFFFBF050020BE0500209B
:10430000341600201AE000280CDD0AFB003132F9D7
:104310001110B942C8BF0F46B142B8BF0E465B1C70
:104320008342F2DB0AF1010AE245D1DB0198B8428F
:1043300002DB0098B04201DD44F0080409F0FF0000
:1043400040907042C6B2344808F0FF08FFB20460E3
:104350002868B0F1FF3F08BFFFF76EFED5E9020AFB
:10436000409968F3070061F30F20D5E9009B67F3DC
:10437000174066F31F600646FF222D6964F3070BA2
:10438000511C684612F081FECDF80090CDE903A5DE
:10439000CDE901B64FF44C352846FEF70FF86946D3
:1043A0002846FEF7ACF81D208DF8000041208DF85E
:1043B000010000208DF802408DF804008DF8030004
:1043C0008DF8050006226946072007F0F1FF41B08D
:1043D000BDE8F08F2DE9F041074610480E460478FD
:1043E0000F48057800F042FB022802D108F0ACFB30
:1043F00078B100F03BFB052802D105F032FD40B159
:1044000004FB05F0420031463846BDE8F04112F0A9
:10441000C5BD6000F6E7000070050020BE05002065
:10442000BF0500202DE9FF4FADF2B44D6FF0310014
:10443000CDF8AC040020CDF8A404CDF8A0041446B7
:104440004FF0320BCDF8A8048146CDF89004824697
:10445000CDF89C04CDF88C04FE484FF00008474688
:104460000678FD480078CDF88484CDF898044FF0A4
:10447000FF30CDF88884CDF8940400F0F7FA1E25BB
:104480006842CDF8B004FFF75EFCCDF88004DDF89B
:1044900098040023002840F3EF800022002E7BDDEB
:1044A00003FB062081B2DDF8B40430F91100A84204
:1044B00006DDDDF8A804401C00B2CDF8A80409E030
:1044C000DDF8ACC4604505DADDF8A404401C00B298
:1044D000CDF8A40434F91100A84217DD09F1010C4C
:1044E0000FFA8CF94045C8BF8046DDF894C460459A
:1044F000C8BF584521DD1FFA83FCCDF884C41FFADC
:1045000082FCCDF89404CDF888C416E0DDF8B0C480
:10451000844512DD0AF1010C0FFA8CFA8742C8BFFC
:104520000746DDF8ACC4604507DADDF8A0C40CF13D
:10453000010C0FFA8CFCCDF8A0C40028B4BFC0F168
:10454000000C8446DC4507DDDDF890C40CF1010C5D
:104550000FFA8CFCCDF890C4DDF880C43CF811C093
:10456000ACEB0000DFF8F4C200B23CF811C0ACEBD9
:10457000000C2DF811C0DDF8B4C43CF911E0BEF117
:10458000000F20DA0028B8BF4042DDF880C43CF9B3
:1045900011C0BCF1000F00E035E0B8BFCCF1000C59
:1045A000844510DA1EF11E0F04DADDF8C0C40220C3
:1045B000ACF80000DDF8B40430F811C0DDF8B80440
:1045C00020F811C005E0DDF8B8044FF0000C20F829
:1045D00011C03DF91100A84205DDDDF89C14491C0D
:1045E00009B2CDF89C140028B8BF4042584505DDFB
:1045F000DDF88C04401C00B2CDF88C04501C02B2D3
:10460000B242FFF64DAF581C03B2DDF89804834266
:10461000FFF643AFBAF10A0F03DBDDF8C004072150
:104620000180D145B8BFB8F1960F0DDA07F19500BA
:10463000B0F5957F08D8002FB4BF78423846404582
:10464000C8BF4FF0000919DCD145B8BFB8F1500F11
:104650000FDA07F14F009E280BD881494878401C9B
:10466000C0B24870C8283DD9C820487000200870E2
:1046700038E0002FB8BF7F42474533DCDDF8A8049F
:10468000012238B1B9F1000F10D075480078012827
:104690002DD042E0DDF8A40400280BDC70494878F6
:1046A000401CC0B24870C8281CD9DDE7DDF8A00462
:1046B000002810DD6A480021417002704FF49062BA
:1046C0006648DDF8801412F069FC0DF2C44D4FF01D
:1046D000FF30BDE8F08F62494878401CC0B2487096
:1046E000C828C1D800200DF2C44DBDE8F08FDDF818
:1046F0009014DDF88C0488420FDA32466946DDF802
:104700009834DDF8B40405F092FFDDF89C0400282D
:1047100004BF0DF2C44DBDE8F08F4FF00008DDF886
:104720009404A6F101091FFA89F70028C8BFBAF15D
:104730000F0F72DDDDF88414DDF8880401FB060E2E
:1047400034F91E3003EBD370B3F1FF3F4FEA600042
:10475000B8BF404202B201FB06F01FFA80FCDDF850
:10476000880400B28346012839DB0CEB000189B2D2
:10477000002B18DD34F911A004EB410131F9021CC2
:10478000BAEB010A06D50029B4BFC1F1000A8A4676
:10479000924504DB0029B8BF4942A9421BDA401EFA
:1047A0001FFA80F81BE016DA34F911A004EB41017E
:1047B00031F9021CAAEB010ABAF1000F06DD00294B
:1047C000B4BFC1F1000A8A469245E8DB0029B8BFB0
:1047D0004942A942E3DB401E00B20128C5DACB45BD
:1047E00037DA0CEB0B0080B2002B17DD34F9101018
:1047F00004EB4000B0F90200091A05D50028B4BF47
:1048000041420146914204DB0028B8BF4042A84221
:1048100019DA0BF1010087B21BE060E013DA34F91A
:10482000101004EB4000B0F90200091A002905DD60
:104830000028B4BF414201469142EADB0028B8BFDC
:104840004042A842E5DB0BF101000FFA80FBCB45AB
:10485000C7DB07E0BE050020BF050020B42E002006
:10486000B8050020DDF88404DDF8802400FB068014
:1048700083B2DDF8840432F9132000FB067034F8AB
:1048800013301FFA80FCD31ADDF880041DB21FFA22
:104890008EF1DDF8803430F9110034F8111033F95D
:1048A0001C3034F81CC0411A09B2A3EB0C0C0FFAEF
:1048B0008CFC4C1B48BF6C1AB1EB0C0548BFACEB31
:1048C000010561190FFA81FC811A48BF111AC21A39
:1048D00048BF1A1A881800B28445FFF603AF0120BA
:1048E00001E72DE9F05FDFF864A180460026DAF8E1
:1048F0000000374690F8241100291CBFB0F83001A1
:1049000000286CD0FCF7EAFCDAF8001091F82411CA
:10491000B0FBF1F201FB1200002860D101F070FC45
:104920005FEA00095BD04A480078102804BF484677
:1049300004F04CFF47484FF0000C444690F800B09C
:104940004548634690F800E0BEF1000F19DD34F9E8
:10495000020B0125BBF1010F10DD34F9022B101AF7
:1049600001B20029B8BF494208B2604502DD844661
:104970001E462F466D1C10465D45EEDB5B1C7345E5
:10498000E5DBDAF80020B2F83001844527DB06FBCE
:104990000B7008EB400338F8101033F8023CC91ACA
:1049A00039F8103009EB400009B230F8020C181A3F
:1049B000081A00B20028B4BF434203460029B8BF1A
:1049C00049428B420BDA0028B8BF4042B2F832119C
:1049D000884204DA01F01EFC0020BDE8F09F0120AF
:1049E000BDE8F09F70B515460E46044608F0ACF8D9
:1049F000002C18BF70BD042818BF052806D0134826
:104A0000006890F82400A84288BF70BD3046BDE819
:104A10007040FFF7A7B870B51546044608F094F843
:104A2000B4F1FF3F0AD0002C18BF70BD002D08BFA5
:104A300070BD2846BDE87040FFF752B8002D08BF92
:104A400070BD2846BDE87040FFF781B9E806002038
:104A500031060020BE050020BF05002010B506F07D
:104A6000E7FA06F081FB002010BD0000AB4800789B
:104A70007047AA480078022805D005281CBF0020EE
:104A8000704705F0EEB908F05FB8A44908707047A8
:104A900010B50446072C28BF10BDDFE804F013044E
:104AA0000810130C0800084600F040F90AE0084618
:104AB00008F03FF806E0084605F0C8F902E00846AD
:104AC00007F0E6FC9548047010BD95490020096880
:104AD000B1F8641011F4807F08BF7047FDF775B816
:104AE0008F4900200968B1F8641011F4807F08BF75
:104AF0007047FDF785B88A4900200968B1F864104D
:104B000011F4806F08BF7047FDF79EB8834948785D
:104B100000281CBF401E4870704710B572B6FEF7E3
:104B20005DFEBDE81040FEF71BBC10B57D48FDF7EB
:104B3000CDFB72B6FEF752FEBDE81040FEF710BC8A
:104B40007648006970477548C06870477349486186
:104B5000704772484069704710B5FCF741FAFBF79F
:104B6000C9FCFCF7CEF8FFF7D4F9BDE81040FCF71C
:104B700070BF10B5FCF734FAFBF7BCFCFBF774FE12
:104B8000FCF7BFF8BDE81040FCF763BF30B5ADF2ED
:104B9000844D05464FF49061684612F0A0FA5F4CD0
:104BA0002846256106F060F9E060F0B10278A27055
:104BB0004178E17083782371531C03F0FE03637125
:104BC0000023E37123724FF0120C84F806C004F145
:104BD0000A0C8CF800308CF80130007860721046B6
:104BE000FCF702FC0DF2844D30BD4D480068B0F872
:104BF000640010F4807F18BFFDF702F800200DF26A
:104C0000844D30BDF0B5ADF2CC4D0F4604464FF4A7
:104C10009061684612F063FA404D20462C6106F020
:104C200023F9E860002851D00278AA704178044640
:104C3000E97080782871501C00F0FE006871002037
:104C4000E87128721223AB7105F10A0318705870CD
:104C5000207868721046FCF7C7FB0DF5906120467E
:104C600006F01FF9608A6E6900281CBF7043060BAE
:104C7000002017F0040F18BF062017F0080F18BF08
:104C800040F00200616A0840DDF88014CDF8C014DD
:104C9000DDF89C14CDF8C414DDF89014CDF8C814D8
:104CA0000DF59861FCF7AFF9DDF88C0420B13346BF
:104CB000EA78A97805F0C4FB6421304605F073FC5E
:104CC000287802280FD0052810D017E01448006873
:104CD000B0F8640010F4807F18BFFCF791FF00204B
:104CE0000DF2CC4DF0BD07F02FFF01E005F0B9F853
:104CF000022804BFDDF89404FFF76EF8002001F0ED
:104D00007EFA0DF2CC4D0120F0BD10B5FCF7F2F9A2
:104D100002490020C860012010BD0000BC05002031
:104D2000E806002000FE1100F9487047F949487074
:104D30007047F84840787047F74810B4F74A016860
:104D4000914218D14168B1F5887F14D80022D0F87B
:104D500008C003461146B2EB9C0F24BF10BC70473D
:104D600053F82140491C2244B1EB9C0FF8D3002A90
:104D700004BF10BC7047002010BC70474FF4FC30DB
:104D8000FDF71CBB2DE9F0410446E3480E46E34F16
:104D90000168B94213D14168B1F5887F0FD800236B
:104DA000D0F808C001461A46B3EB9C0F08D251F860
:104DB0002250521C2B44B2EB9C0FF8D303B10020BD
:104DC000002558B1B0E80E10A4E80E10B0E80E109F
:104DD000A4E80E100FC884E80F0016E0FF2230216F
:104DE000204612F052F94FF48870C4E90070302068
:104DF000C4E90205AA20C4E904054FF0FF30E062CF
:104E0000A062A5616062C4E9075066B94FF4FC3046
:104E1000FDF7D4FAC248056045608560C56005614C
:104E200045618561C5610120BDE8F081B949012076
:104E300048707047B74900200870704770B5ADF5ED
:104E4000107D0446FFF77FFE054614F0020F04BFF5
:104E50000DF5107D70BD0426FFF70BFE002818BF6E
:104E6000B04C08D095F92C102246304606F03EF89A
:104E70000DF5107D70BD6C462046FCF7B3FCF1E7E4
:104E800070B50D4606461024FFF75DFE16F0020FC2
:104E900018BF05242A46102C28BF70BD002A08BF61
:104EA00070BD204490F928102046BDE8704006F0FF
:104EB0001DB82DE9F04F87B08146122000244FF035
:104EC000200A27460090FFF7D1FD022802D107F003
:104ED0003BFE30B1FFF7CAFD052804D104F0C1FF45
:104EE00008B9022000900098002500289CBF07B058
:104EF000BDE8F08F0026BAF1000F7CD98A4A681EFF
:104F0000A2FB00314908A1EB810108440590E81E8D
:104F10000490A81F0390C01E0290C01E0190A2FB27
:104F200005104008A0EB8000A5F10F0B00EB050871
:104F3000FFF79CFD022803D107F006FE00283AD0B7
:104F4000FFF794FD052803D104F08BFF002832D031
:104F5000032D38BF142417D30498032838BF152411
:104F600012D30398032838BF16240DD302980328C0
:104F700038BF242408D30198032838BF252403D33D
:104F8000BBF1030F38BF2624A7420AD06748C4F3F9
:104F9000031127460068C16104F00F017F20FBF771
:104FA00053FAC4F3031001281CBFC6F11F0000EB25
:104FB000481018D127E0002D0CBF14242424A74248
:104FC00009D05A48210927460068C16104F00F0141
:104FD0007F20FBF739FA2009012814D00598C6F183
:104FE0001F0101EB401019F8011BC0B2FBF72CFAAE
:104FF000761C56459CD300986D1C8542FFF47AAF11
:1050000007B0BDE8F08F06EB4810ECE72DE9F84F4C
:10501000834640484FF0000A0C46B0F904804FF038
:105020001209202750460091FCF7D8F90546CBF12C
:105030000706FFF71BFD022802D107F085FD30B1FE
:10504000FFF714FD052804D104F00BFF08B94FF059
:105050000209BBF1000F1CD0002E55DB4FF0000CF5
:10506000B9F1000F49D9012101FA06F3701E01FAC6
:1050700000FB0021002F3CD935F8020B2278A0EB71
:10508000080000B25FEAD21E23D0002827DA2EBB28
:105090001BE00023B9F1000F2FD90021002F10D9F8
:1050A00035F8022B2078A2EB080212B2502AC8BFB2
:1050B00040F0800040F04000491C04F8010BB94268
:1050C000EED35B1C4B45E8D317E010F1280F05DB4E
:1050D0000AE0002803DD0EB9282805DD9A43002EDA
:1050E000C4BF4BEA0200C2B204F8012B491CB9420A
:1050F000C2D30CF1010CCC45BBD30098FFF7D9FE0D
:10510000002E08BF4FF0010A5046BDE8F88F00009E
:1051100034330020D405002000F8110054435246D7
:105120001416002074350020ABAAAAAAE886110044
:10513000FD498880704770B5FB4EFC49F0800968D6
:105140000320C8610425E9B27F20FBF77DF9002424
:10515000B179E0B2FBF778F904F12000B179C0B27F
:10516000FBF772F904F14000B179C0B2FBF76CF9BA
:10517000641C202CECDB6D1C072DE4DB70BD2DE9DD
:10518000F04F89B00026FBF72BFFE849072009689C
:105190000865E748016841F0200101600020FFF741
:1051A000CAFFE1494FF4006088804FF41071E14874
:1051B00011F095FF0020FBF7B0FDFCF73DF800254E
:1051C0002C460795FFF755FC04F03FF801281DD049
:1051D0006846FCF7D8FAB8B10120FBF79EFD684697
:1051E00004F05DFC6D1C012D0ED00025D149204638
:1051F000FFF70CFF072C1ED00020FBF78EFDFCF7FD
:10520000EDFAFCF719F8641C002EDDD0FFF731FC35
:10521000C54AC948C74BD0600020D16813F800C008
:10522000401C01F801CBD160B0F5107FF5D3079891
:1052300000283CD135E012200890BB4800274FF0F1
:10524000200BB0F904603846FCF7C8F80546BA46AA
:105250000024BBF1000F18D9304612F0F2FBB74A18
:10526000B74B12F055FC8946804635F9022B901B4E
:1052700048BFB01A12F0E5FB42464B4612F046FD1D
:1052800038BF7F1C641C5C45EFD308980AF1010A03
:105290008245DDD3002F4FF001061CBF012007908F
:1052A000B4E7002E1EBF002009B0BDE8F08F01203A
:1052B00009B0BDE8F08FF0B587B000260120FBF7FC
:1052C000D2FC9B48016841F0200101600020FFF7FB
:1052D00032FF95494FF4006088809A490020C1F858
:1052E0008000C1F88400C1F88800C1F88C00C1F8C2
:1052F0009000C1F89400C1F89800C1F89C00C1F872
:10530000A000C1F8A400C1F8A800C1F8AC00C1F821
:10531000B000C1F8B400C1F8B800C1F8BC00FBF798
:10532000FCFCFBF789FF00252C462F4603F08DFF80
:10533000012835D06846FCF726FA78B30120FBF740
:10534000ECFC6D1C012D24D000257F492046FFF781
:105350005DFE072C06D00020FBF7DFFCFBF76CFF9F
:10536000641C1BE0002420252046FCF737F80021B0
:1053700030F9022BA2F26662B2F54D7F88BF641C41
:10538000491CB1EB450FF3D3002C08BF01260DD10A
:1053900006E00020FBF7C1FCFBF74EFF002EC5D056
:1053A00027B9002E1EBF002007B0F0BD012007B0B6
:1053B000F0BD2DE9F04F82460021ADF5137D634825
:1053C00090910C4600780F460D46022808BF022730
:1053D00003D0052804BF02240427DFF85091DFF82A
:1053E00070B100F09AB9204605F03EFD002800F0AB
:1053F0009381008900EA0A0626F0CC0030F47C4054
:1054000000F08A81DFF84C81D8F800004069D8F8B4
:10541000001040F400704861D8F800000069D8F826
:10542000001020F006000861D8F800000069D8F8E4
:10543000001040F0100008613CB1012C35D0022C66
:1054400071D0032C55D000F0FBB802210846FFF7BD
:105450001FFB0120FBF707FC05F06BFB0F2120462B
:10546000FFF7D0FB002800F05781D9F80000406C0E
:10547000D9F8001040F40060486400BF00BF00BFCE
:10548000D9F80000406CD9F8001020F4006048649E
:10549000FBF77DFB05F039FB012007F00FFC002036
:1054A000FBF73BFCFCF79AF9CAE000210220FFF76A
:1054B000EFFA0120FBF7D7FB0F212046FFF7A2FBF5
:1054C000002800F02981D9F80000406CD9F80010BC
:1054D00040F40060486400BF00BF00BFD9F800007E
:1054E000406CD9F8001020F400604864FBF74FFBD3
:1054F000A6E000210520FFF7CBFAFBF771FDD8F8F5
:1055000000000069D8F8001020F006000861D8F803
:1055100000000069D8F8001040F004000861D8F8D5
:105520000000006918E03EE0D4050020E886110084
:105530006405002074350020343300209A9999992D
:105540009999B93F34370020B4370020290600204C
:10555000EC861100D0861100D8F8001040F0100041
:10556000086109F01CFA0F210220FFF74BFB00280D
:105570007ED0DBF8001007208860DBF800100420E4
:10558000486002212020FBF72FFF0020FBF7C5FB1E
:10559000FBF729FEDBF800000068DBF8001040F0A4
:1055A000010008604CE002210520FFF771FAFBF7CB
:1055B00017FDD8F800000069D8F8001020F00600A8
:1055C0000861D8F800000069D8F8001040F0040025
:1055D0000861D8F800000069D8F8001040F0100009
:1055E000086109F0DCF905F090FA0F210320FFF7BC
:1055F00009FB00283CD0DBF800107F208860DBF836
:10560000001002204860D9F80000406CD9F8001062
:1056100040F400604864012007F049F9D9F800001F
:10562000406CD9F8001020F400604864FBF7DBFD03
:10563000DBF800000068DBF8001040F001000860B3
:105640009098002864D116F0010F23D00120FBF7B9
:105650000AFBFFF70EFA88B1FBF78AFFFF210F2044
:10566000FFF78DFD012121EA00000543002000E045
:1056700052E0FBF752FB909890BB0BE0FBF778FFF2
:10568000FF210F20FFF717FE012121EA000045EA64
:105690004005EBE716F0060F22D0FFF7EAF90228E3
:1056A0001ED1FEF7F1F90020FEF75DFC0120FBF7AB
:1056B000DAFAFEF748FB0646FFF745FA0523320003
:1056C00004D090F92D10184605F010FCFEF73BFBB6
:1056D000FEF733FCFEF737FB4FF4906111F0DDFC71
:1056E000FFF731FA804604209190FFF7C2F90028B5
:1056F00018BFFE4E1FD098F92C103246919805F035
:10570000F5FBFB4900200870FA490870FBF76BFDB8
:10571000FFF7ACF9FFF7F9FA641CBC4203D290988A
:1057200000283FF460AEF449002008700DF5137DA9
:105730002846BDE8F08F6E463046FCF753F8DAE7AE
:1057400070B5ED48CCB04578FFF790F901287DD1D0
:10575000EA480068B0F93610B0F9340004F096FF5A
:1057600015F0020F73D0002140A8FFF70BFB4598FE
:10577000401C459040F27770FFF71BFEC0B2032833
:1057800010D0002804BF45F25000449012D00128E8
:1057900008BF4AF250100CD0022808BF45F2A10001
:1057A00007D007E04AF2A11044904698401C46906A
:1057B00008E0449047980022401C47902121072090
:1057C00006F0CDFD40AC05F040FB40B18169489149
:1057D000C169499141694A91C0684B9005E04FF019
:1057E000FF304B904A9049904890C54840904FF404
:1057F000887041903020429000204390A368224658
:10580000014652F820C0401C6144B0EB930FF8D31E
:105810004E42FF22511C6846E66011F036FCA26839
:10582000F4E804018DE847000FCC04AE86E80F00D1
:1058300094E80F0008AE203C86E80F004FF4FC30DF
:105840006946FCF75CFEAF49226801E022E00DE00A
:105850000A6062684A6022698A606269CA60A269F5
:105860000A61E2694A61226A8A610CE015F0010F5F
:1058700009D040F22220FFF79CFD20B9002221210F
:10588000072006F06CFDFEF759FA2A464021072052
:1058900006F065FD4CB0BDE8704003F0D2BC70B5B9
:1058A0000C469949054603200968C86101217F20FB
:1058B000FAF7CAFD00217520FAF7C6FD012176200E
:1058C000FAF7C2FD60210820FAF7BEFD0021092089
:1058D000FAF7BAFD30210A20FAF7B6FD00210B20B5
:1058E000FAF7B2FD06210E20FAF7AEFDE1B226204E
:1058F000FAF7AAFDE1B22720FAF7A6FDE1B22820C7
:10590000FAF7A2FDE1B22920FAF79EFDE1B22A20C2
:10591000FAF79AFDE1B23020FAF796FDE1B23120B4
:10592000FAF792FDE1B23220FAF78EFDE1B23320B0
:10593000FAF78AFDE1B23420FAF786FDE1B23620AB
:10594000FAF782FDE1B23720FAF77EFDE1B23820A6
:10595000FAF77AFDE1B23920FAF776FDE1B23A20A2
:10596000FAF772FDE1B24020FAF76EFDE1B2412094
:10597000FAF76AFDE1B24220FAF766FDE1B2432090
:10598000FAF762FDE1B24420FAF75EFDE1B246208B
:10599000FAF75AFDE1B24720FAF756FDE1B2482086
:1059A000FAF752FDE1B24920FAF74EFDE1B24A2082
:1059B000FAF74AFDE1B25020FAF746FDE1B2512074
:1059C000FAF742FDE1B25220FAF73EFDE1B2532070
:1059D000FAF73AFDE1B25420FAF736FDE1B256206B
:1059E000FAF732FDE1B25720FAF72EFDE1B2582066
:1059F000FAF72AFDE1B25920FAF726FDE1B25A2062
:105A0000FAF722FDE1B26020FAF71EFDE1B2612053
:105A1000FAF71AFDE1B26220FAF716FDE1B263204F
:105A2000FAF712FDE1B26420FAF70EFDE1B266204A
:105A3000FAF70AFDE1B26720FAF706FDE1B2682045
:105A4000FAF702FDE1B26920FAF7FEFCE1B26A2042
:105A5000FAF7FAFC02217F20FAF7F6FC6A2102200D
:105A6000FAF7F2FC8E210420FAF7EEFCF121072070
:105A7000FAF7EAFC15B1012D05D008E00421062053
:105A8000FAF7E2FC03E008210620FAF7DDFC032127
:105A90007F20FAF7D9FC21211020FAF7D5FC00214C
:105AA0001120FAF7D1FC00211220FAF7CDFC0021D9
:105AB0001320FAF7C9FC00211420FAF7C5FC0021D5
:105AC0001520FAF7C1FC01211620FAF7BDFC0221CE
:105AD0001720FAF7B9FC00211820FAF7B5FC0021CD
:105AE0001920FAF7B1FC00211A200FE074350020CC
:105AF0001607002017070020D4050020E806002024
:105B00005443524614160020E8861100FAF79CFC14
:105B100000211B20FAF798FC01212020FAF794FCC1
:105B200020212120FAF790FC00212220FAF78CFC9A
:105B300000212320FAF788FC00212420FAF784FCB6
:105B400000212520FAF780FC01212620FAF77CFCB1
:105B500000212720FAF778FC02212820FAF774FCAC
:105B600000212920FAF770FC00212A20FAF76CFCAA
:105B700000212B20FAF768FC01213020FAF764FCA1
:105B800000213120FAF760FC20213220FAF75CFC7A
:105B900000213320FAF758FC00213420FAF754FC96
:105BA00000213520FAF750FC01213620FAF74CFC91
:105BB00000213720FAF748FC00213820FAF744FC8E
:105BC00002213920FAF740FC00213A20FAF73CFC88
:105BD00000213B20FAF738FC01214020FAF734FC81
:105BE00000214120FAF730FC00214220FAF72CFC7A
:105BF00020214320FAF728FC00214420FAF724FC56
:105C000000214520FAF720FC01214620FAF71CFC70
:105C100000214720FAF718FC00214820FAF714FC6D
:105C200000214920FAF710FC02214A20FAF70CFC67
:105C300000214B20FAF708FC01215020FAF704FC60
:105C400000215120FAF700FC00215220FAF7FCFB5A
:105C500000215320FAF7F8FB20215420FAF7F4FB37
:105C6000BDE8704000215520FAF7EEBB10B50322C5
:105C7000FD49062828BF10BDDFE800F00327FDFC22
:105C8000FBFA0868C26101217F20FAF7DDFBAF2132
:105C90000820FAF7D9FB73210A20FAF7D5FB0A216D
:105CA0000E20FAF7D1FB02217F20FAF7CDFB00216D
:105CB0000720FAF7C9FB1F210120FAF7C5FB1021C5
:105CC000BDE810400620FAF7BFBB0868C261012199
:105CD0007F20FAF7B9FB0F210E20FAF7B5FB8721D9
:105CE0000820FAF7B1FB6E210A20FAF7ADFB02217A
:105CF0007F20FAF7A9FB71210720FAF7A5FB6A219B
:105D00000220FAF7A1FB8E210420FAF79DFB032164
:105D10007F20FAF799FB61211020FAF795FB00210B
:105D20001120FAF791FB00211220FAF78DFB0021D8
:105D30001320FAF789FB00211420FAF785FB0021D4
:105D40001520FAF781FB01211620FAF77DFB0621C9
:105D50001720FAF779FB00211820FAF775FB0021CC
:105D60001920FAF771FB00211A20FAF76DFB0021C8
:105D70001B20FAF769FB01212020FAF765FB60215F
:105D80002120FAF761FB00212220FAF75DFB0021B8
:105D90002320FAF759FB00212420FAF755FB0021B4
:105DA0002520FAF751FB01212620FAF74DFB0021AF
:105DB0002720FAF749FB06212820FAF745FB0021A6
:105DC0002920FAF741FB00212A20FAF73DFB0021A8
:105DD0002B20FAF739FB01213020FAF735FB00219F
:105DE0003120FAF731FB60213220FAF72DFB002138
:105DF0003320FAF729FB00213420FAF725FB002194
:105E00003520FAF721FB01213620FAF71DFB00218E
:105E10003720FAF719FB00213820FAF715FB062185
:105E20003920FAF711FB00213A20FAF70DFB002187
:105E30003B20FAF709FB01214020FAF705FB00217E
:105E40004120FAF701FB00214220FAF7FDFA602118
:105E50004320FAF7F9FA00214420FAF7F5FA002175
:105E60004520FAF7F1FA01214620FAF7EDFA03E0AE
:105E70003FE039E033E02DE000214720FAF7E4FA73
:105E800000214820FAF7E0FA00214920FAF7DCFA6D
:105E900006214A20FAF7D8FA00214B20FAF7D4FA63
:105EA00001215020FAF7D0FA00215120FAF7CCFA5C
:105EB00000215220FAF7C8FA00215320FAF7C4FA59
:105EC00060215420FAF7C0FA0021BDE810405520A7
:105ED000FAF7BABAAA21BDE810400020DFE4552144
:105EE000BDE810400020DAE4AA21BDE810400120FE
:105EF000D5E45521BDE810400120D0E410B5FDF7F0
:105F000022FF0446FDF721FF2146BDE810404FF473
:105F1000906211F043B82DE9F04154480478544898
:105F20000578FDF712FF0646FDF70DFF0022002D54
:105F300098BFBDE8F0810021002C10D902FB04FCC1
:105F400006EB4C0300EB4C0C11F0010F1CBF33F8B7
:105F500011702CF81170491CC9B2A142F4D3511C24
:105F6000CAB2AA42E7D3BDE8F08100B5ADF2844DD4
:105F7000FDF7EBFE01464FF49062684611F00EF813
:105F80006846FDF7E4FE0DF2844D00BD2DE9F04FAB
:105F900083B012200190384836494FF02009002480
:105FA000C16001E0032C01DA14261AE0E01E032888
:105FB00038BF152615D3A01F032838BF162610D3C7
:105FC000A4F10900032838BF24260AD3A4F10C0049
:105FD000032838BF252604D3A4F10F00032838BFB7
:105FE0002626B34509D020483109B3460068C1616F
:105FF00006F00F017F20FAF727FA0025B9F1000F0C
:106000002ADD1E484FEA161A80FB0410A0EBE07050
:10601000A0EB800000EB0408BAF1010F0EBF05EB06
:106020004810C5F11F0000EB481087B21249C8683C
:1060300010F8012B0092C860F8B21146FAF704FA82
:1060400000BF00BF00BF00BF00BFF8B20099FAF761
:10605000FBF96D1C4D45DFDB0198641C8442A1DB1C
:1060600003B0BDE8F08F0000E8861100BE050020F7
:10607000BF05002034330020D40500205655555567
:106080002DE9F84FDFF8D8B174484FF02008CBF86D
:106090000C0012200024009001E0032C01DA1426E9
:1060A0001AE0E01E032838BF152615D3A01F0328C9
:1060B00038BF162610D3A4F10900032838BF2426C0
:1060C0000AD3A4F10C00032838BF252604D3A4F179
:1060D0000F00032838BF2626B24509D06148310990
:1060E000B2460068C16106F00F017F20FAF7ACF9F3
:1060F0000025B8F1000F1EDD5B484FEA161980FB42
:106100000410A0EBE070A0EB80000719B9F1010FBB
:106110000EBF05EB4710C5F11F0000EB471080B222
:10612000FAF7ABF9DBF80C106D1C454501F8010BD3
:10613000CBF80C10EADB0098641C8442ADDBDBF882
:106140000C00BDE8F88F4648C08870472DE9F04341
:10615000002787B0B946FAF743FF41494FF4006082
:106160008880FAF7EAFD0020FAF7D7FD00254FF006
:106170005A082846FEF7DFFFFBF735F803F065F80D
:106180006846FBF700FB28B3684603F088FC002450
:1061900020262046FBF722F9002130F9022BA2F23B
:1061A0006662B2F54D7F88BF641C491CB1EB460F97
:1061B000F3D3ACB1454515D2FAF712FFA8B26D1C66
:1061C000FEF7B9FFFBF70FF806F0BEFC002808BF8A
:1061D000FBF70AFE002FD1D0B9F1000F0BD104E07C
:1061E0000127F9E7FAF7FCFE05E0002F1EBF0020AB
:1061F00007B0BDE8F083012007B0BDE8F083704729
:106200001748816800291BBF017811F0020F002098
:10621000C068704715481249006890F825218878B1
:10622000401CC0B28870824228BF7047002088702E
:1062300001210846FEF72CBC10B506F085FC074985
:1062400002284FF4107204D0BDE81040084810F046
:10625000A5BEBDE81040074810F0A0BE34330020B2
:10626000D4050020E886110056555555E806002053
:10627000620C00201C6200201FB513F0070F069867
:1062800004D003F00702022A08D004E0012202A988
:106290000F2002F0B6FF04B0002010BDF84B5A7971
:1062A000052A0DD1DA8982423CBF521CDA8192B2B2
:1062B000824205D10020D881012008700320587146
:1062C00004B0012010BD1FB513F0070F04D003F078
:1062D0000700022808D004E0012202A90F2002F0E2
:1062E00090FF04B0002010BD0120087004B010BD64
:1062F0001FB513F0070F04D003F00700022808D0E1
:1063000004E0012202A90F2002F07BFF04B000206C
:1063100010BD0120087004B010BD1FB513F0070FA9
:1063200004D003F00700022808D004E0012202A9EB
:106330000F2002F066FF04B0002010BD012008709D
:1063400004B010BD1FB513F0070F04D003F0070011
:10635000022808D004E0012202A90F2002F051FF18
:1063600004B0002010BD0120087004B010BD2DE95C
:10637000F00703F007050027C14EDDF81CC0012D12
:1063800008BFF7810DD013F0070FBD4BDFF8F48283
:10639000DFF8F492DB8903F10104A4B205D0022DE9
:1063A00016D0BDE8F0070020704763453CBFD9F820
:1063B0000000C254F481644524D1D9F80000D9F812
:1063C00000104078097800EB0120A8F80E0019E0D1
:1063D000B8F80E20D9F80050120A63452A70D9F88F
:1063E000005098F80E206A7004D2D9F80020D25CD0
:1063F0000270F481F089604504D1F78101200870B2
:1064000003207071BDE8F007012070471FB513F03D
:10641000070F04D003F00700022808D004E001228F
:1064200002A90F2002F0EDFE04B0002010BD0120F3
:10643000087004B010BD1FB513F0070F04D003F0AF
:106440000700022808D004E0012202A90F2002F070
:10645000D8FE04B0002010BD0120087004B010BDAB
:106460001FB513F0070F04D003F00700022808D06F
:1064700004E0012202A90F2002F0C3FE04B00020B4
:1064800010BD0120087004B010BD1FB513F0070F38
:10649000069804D003F00702022A08D004E0012283
:1064A00002A90F2002F0ADFE04B0002010BD744B15
:1064B0005A79052A0DD1DA8982423CBF521CDA8111
:1064C00092B2824205D10020D881012008700320B9
:1064D000587104B0012010BD0020704708B503F0CA
:1064E0000700012806D18DF80000024669460B20FE
:1064F00002F087FE002008BD08B503F00700012860
:1065000007D100208DF80000012269460B2002F01F
:1065100078FE002008BD10B503F00700012808BF71
:10652000FEF7FBFA002010BD08B503F007000128B4
:1065300007D103208DF8000001226946002002F0F7
:1065400060FE002008BD08B503F00700012807D150
:1065500003208DF8000001226946002002F051FE60
:10656000002008BD70B403F007020024444BDDF89E
:106570000CC0012A02D0022A08D004E0052058717C
:10658000DC811C639C8270BC002070475A79052A0C
:1065900011D1DA89624506D23C4DAD68D600F5408E
:1065A0000570501CD881D889604504D1DC81012058
:1065B00008700320587170BC012070471FB513F09C
:1065C000070F08D19DF80800F02807D0012202A982
:1065D000072002F016FE04B0002010BDFEF7CEFB2F
:1065E000F9E71FB513F0070F04D1012202A91046E5
:1065F00002F007FE04B0002010BD2DE9F00103F009
:1066000007041F4E059D012C04BF0020F0811ED001
:1066100013F0070F1A4B1E4FDB8903F1010C1FFA11
:106620008CFC02D0022C16D011E01749022B3CBF83
:106630000868C254A6F80EC0AC4508D108680278B4
:10664000386880F8EB200968497880F8EA10BDE8DE
:10665000F001002070470E4A002B126804BF92F828
:10666000EB10017006D0012B04D192F8EA200270E1
:1066700001200870A6F80EC0BDE8F00101207047A7
:10668000EC050020F80F00201487110014160020DC
:10669000E806002030B403F0070CF84CBCF1010F01
:1066A00004BF0020E08118D013F0070FF34BDB8903
:1066B00003D0BCF1020F13D00FE073B9A271082A06
:1066C0000BD2DFE802F004070704040404044FF4CB
:1066D000906001E04FF41070E06230BC0020704721
:1066E000E64A002BD26A04BF110A017004D0012BC4
:1066F00002D1027001200870581CE08130BC0120DA
:106700007047F8B5054603F007000026DB4C0F463E
:10671000012807D013F0070F2346DB8906D0022893
:1067200028D025E005206071E68121E003BBA2713D
:106730004FF49060A0824010082A19D2DFE802F0DE
:1067400004060A0E10121416CD4810E0CD4921633C
:10675000A0820DE0CC492163A08209E0CB4806E08D
:10676000CB4804E0CB4802E0CB4800E0CB482063B4
:106770000020F8BD6079052847D1206B002844D05F
:10678000C749BE4A0968928A91F8EB10012918BFDF
:10679000032906D0694693422DD213F0030F21D16D
:1067A00018E0934227D213F0010F07D094F82C0081
:1067B0002870E06A000AE062581C1BE0AF49A0792B
:1067C000C989042821F0010214BFB648B648805E8A
:1067D000E062EBE70422FBF773FC0098E062206BB9
:1067E000001D206394F82C002870E06A000AE06223
:1067F000E089401CE081E089A18A884205D1E681D8
:10680000012026633870032060710120F8BD2DE956
:10681000F84303F007020026984D089C0F46804677
:10682000012A02D0022A06D002E005206871EE811A
:106830000020BDE8F883687905281CD1E889A042CA
:1068400011D2FCF744FFAC208DF800007A208DF8BF
:10685000010070208DF80200EA891DF8020088F816
:106860000000501CE88180B2A04204D1EE810120DA
:106870003870032068710120BDE8F8832DE9F041EC
:1068800082B003F0070200267C4D089C0F4680462C
:10689000012A02D0022A07D002E005206871EE81A9
:1068A00002B00020BDE8F0816879052821D1E8898F
:1068B000A04216D2FCF70BFF53208DF800004520B4
:1068C0008DF801007A208DF8020070208DF8030009
:1068D0008DF80460EA891DF8020088F80000501C59
:1068E000E88180B2A04204D1EE81012038700320FB
:1068F000687102B00120BDE8F0812DE9F00388B095
:1069000003F007020027DFF87481DDF838C0012AA0
:1069100009D04446E489651CAEB2022A0DD013F0BA
:10692000070F2FD004E0052088F80500A8F80E70A6
:1069300008B00020BDE8F003704798F80520052A4C
:106940001BD164450ED2594D00226B4615F80290BA
:1069500003F80290521CD2B2202AF7D31A5D0270BB
:10696000A8F80E60B8F80E00604506D1A8F80E70C1
:1069700001200870032088F8050008B00120BDE858
:10698000F0037047644538BFA8F80E60B8F80E00F1
:10699000604508BFA8F80E70CAE72DE9F007DFF8D8
:1069A00000C183B003F0070ADCF800C00A9A002790
:1069B000BCF81640BCF81450DFF8C080BAF1010FE3
:1069C0000ED0C4464FF00109BCF80EC0BAF1020F58
:1069D0000CF10106B6B20DD013F0070F40D004E061
:1069E000052088F80500A8F80E7003B00020BDE867
:1069F000F007704798F80530052B2CD194451FD22D
:106A0000230A8DF800308DF804304FEA152A12233E
:106A10008DF808308DF801408DF8054020238DF861
:106A200002A08DF806A08DF809308DF803508DF87E
:106A300007508DF80A701DF80C300370A8F80E602E
:106A4000B8F80E00904206D1A8F80E7081F80090B8
:106A5000032088F8050003B00120BDE8F007704767
:106A60001348944580F8009038BFA8F80E60B8F835
:106A70000E00904208BFA8F80E70B6E7EC050020A3
:106A800054B0020054D8020054DC020054C8020082
:106A900054D0020054C0020054B8020054EC02006A
:106AA000E8060020006D002000750020F43700206B
:106AB000440700202DE9F04383B0804603F007002F
:106AC0000026FF4D0A9C0F46012802D0022807D05D
:106AD00002E005206871EE8103B00020BDE8F0837C
:106AE000687905282DD1E8894FF00109A04220D20C
:106AF0000021B220FBF7B8F88DF80000010A8DF8EC
:106B00000110010C8DF80210000E8DF803007A20A0
:106B10008DF804001F208DF8050004208DF8070073
:106B20008DF80690E8891DF8001088F80010401CC8
:106B3000E88180B2A04204D1EE8187F80090032062
:106B4000687103B00120BDE8F0832DE9F84303F03C
:106B500007020026DA4D089C0F468046012A02D023
:106B6000022A06D002E005206871EE810020BDE80F
:106B7000F8836879052814D1E889A04209D26846CB
:106B8000FBF789FDEA891DF8020088F80000501C17
:106B9000E88180B2A04204D1EE8101203870032048
:106BA00068710120BDE8F88310B403F00701DFF835
:106BB00010C3012906D013F0070FC24B08D00229D9
:106BC00010D00CE00020ACF80E00ACF8100006E08D
:106BD000BCF80E0019680A54401CACF80E0010BC3A
:106BE00000207047BCF810101A68525C0270481CF4
:106BF000ACF8100010BC01207047F0B583B003F072
:106C0000070201270025AF4CAD4EDDF820C0012A58
:106C100004D0022A00F0C68000F09DB8FCF757FDB2
:106C2000012202A912200295FBF74AFA0520707191
:106C300021687A20087020684770216821208870B8
:106C4000A14822680168897CD17000682268017CB3
:106C50001171017E11F0040F0ED0C18A2268090A59
:106C600051712268817D9171818A2268090AD171EE
:106C70002168007D08720DE0818A2268090A51713D
:106C80002268017D9171C18A2268090AD171216847
:106C9000807D08720422694610460095FBF710FAC1
:106CA0002168009848722268010A91722268010CDA
:106CB000000ED172216804220873694614200095E1
:106CC000FBF7FEF92168009848732268010A917366
:106CD0002268010C000ED173216808740298009597
:106CE00000283BD0042201A948200195FBF7E8F9D0
:106CF000019804225030019069461C30FBF7E0F9FE
:106D00002168009848742268010A91742268010C75
:106D1000000ED174216804220875009501A948204D
:106D20000195FBF7CDF90198042250300190694696
:106D30002C30FBF7C5F92168009848752268010AD4
:106D400091752268010C000ED175216808762168C2
:106D5000FF204876F58103B00020F0BD042269468B
:106D60005A48FBF7ADF92168009848742268010A77
:106D700091742268010C000ED174216804220875F8
:106D8000694653480095FBF79BF9216800984875C0
:106D90002268010A91752268010C000ED1752168E4
:106DA0000876D4E77279052A0ED1F289624504D2B9
:106DB00023689B5C0370501CF081F089604503D10F
:106DC000F5810F700320707103B00120F0BD30B465
:106DD00003F007043B4B3A4D029A4FF0000C012C94
:106DE00002D0022C38D034E0022068713948A5F86E
:106DF0000EC00168880A444211EB842418BF401C6D
:106E0000404201EB8000C01C20F003003249B0F585
:106E1000003F014414D8CC78086864F31F602F4CFD
:106E2000A0420DD10020002A13D901EB000C1C68F0
:106E30009CF804C004F800C0401C8242F5D808E069
:106E40000020002A05D9196801F800C0401C8242C0
:106E5000F9D830BC002070476C79022C10D1EC8935
:106E6000944204D21B681B5D0370601CE881E889B2
:106E7000904205D1A5F80EC001200870032068716A
:106E800030BC0120704738B503F007020D4C0025D7
:106E90000B4BDDF810C0012A02D0022A7ED086E01A
:106EA000022058710E48DD8100680E49884245D1A4
:106EB0000D4801682268117001682268090A15E00E
:106EC000EC05002014871100E80600205CC00100DA
:106ED0006CC0010000FE1100E8FF0F0034CD12ABC2
:106EE000F015002054464953FC15002051700168EC
:106EF0002268090C917001682268090ED1704168FE
:106F00002268117141682268090A5171416822683A
:106F1000090C917141682268090ED171816822685B
:106F2000117281682268090A517281682268090C0D
:106F3000917280682168000EC87238E004226946A8
:106F400020200095FBF7BCF8216800980422087007
:106F500000982168000A487000982168000C887029
:106F600000982168000EC87069462420FBF7A8F835
:106F70002168009808712268010A51712268010C89
:106F8000000E917121680422C87169462820FBF720
:106F900097F8216800980872010A00E009E0226869
:106FA00051722268010C000E91722168C872002093
:106FB00038BD5A79022A0FD1DA89624504D2246891
:106FC000A45C0470501CD881D889604504D1DD814F
:106FD0000120087003205871012038BD70B503F0FE
:106FE00007020025FA4CFB4BDDF810C0012A03D044
:106FF000022A0DD0002070BD02205871DD8103F0FF
:10700000E3FE002814BF8020402021680870F1E7CB
:107010005A79022A0FD1DA89624504D22468A45C25
:107020000470501CD881D889604504D1DD810120CD
:10703000087003205871012070BD70B503F007027D
:107040000025E34CE34BDDF810C0012A02D0022AF0
:1070500010D00DE002205871DD810020FBF783FE87
:1070600005460120FBF77FFE216845EA0010087005
:10707000002070BD5A79022A0FD1DA89624504D204
:107080002468A45C0470501CD881D889604504D160
:10709000DD810120087003205871012070BD30B4DB
:1070A00003F007020024CA4DCA4BDDF808C0012ACC
:1070B00002D0022A09D005E002205871DC8129683B
:1070C0005520087030BC002070475A79022A0FD131
:1070D000DA89624504D22D68AD5C0570501CD881F8
:1070E000D889604504D1DC810120087003205871E3
:1070F00030BC012070472DE9F84303F00702002659
:10710000B34DDFF8D082089C4FF00109012A02D06C
:10711000022A2CD028E003F098FE8769022088F824
:107120000500A8F80E60042269460020FAF7C8FF9F
:10713000A948009981420FD1286880F800902968F9
:1071400004204870286887702968380AC870286841
:1071500046712868867107E00020002C04D9296850
:107160000E54401C8442FAD80020BDE8F88398F8F9
:107170000520022A14D1B8F80E20A24205D22B68AD
:107180009B5C0370501CA8F80E00B8F80E00A042DB
:1071900006D1A8F80E6081F80090032088F8050059
:1071A0000120BDE8F883F8B503F00702884C0025FC
:1071B000884EDDF818C0012A02D0022A70D06CE097
:1071C00003F043FE00282ED0844801682268117025
:1071D00001682268090A517001682268090C9170DF
:1071E00001682268090ED1704168226811714168F6
:1071F0002268090A517141682268090C917141683D
:107200002268090ED1718168226811728168226832
:10721000090A517281682268090C9172806821689C
:10722000000EC87236E0042269466D480095FAF7F0
:1072300047FF216800980422087000982168000A1E
:10724000487000982168000C887000982168000E32
:10725000C87069466348FAF733FF216800980871DF
:107260002268010A51712268010C000E9171216897
:107270000422C87169465C48FAF722FF2168009829
:1072800008722268010A51722268010C9172010E83
:107290002068C17202207071F5810020F8BDFFE7FF
:1072A0007279022A0FD1F289624504D223689B5C6D
:1072B0000370501CF081F089604504D1F5810120F4
:1072C0000870032070710120F8BD38B503F0070283
:1072D0003F4C00253F4BDDF810C0012A02D0022AA6
:1072E0004FD04CE0022058714048DD8101683A4A95
:1072F00091421ED141682268117041682268090AD2
:10730000517041680A0C21688A7041682268090E30
:10731000D17081682268117181682268090A5171EF
:1073200081682268090C917180682168000EC8711B
:1073300025E00422694610460095FAF7C1FE21684F
:1073400000980422087000982168000A487000988C
:107350002168000C887000982168000EC87069468A
:107360000820FAF7ADFE2168009808712268010A2A
:1073700051712268010C000E91712168C8710020C2
:1073800038BD5A79022A0FD1DA89624504D22468BD
:10739000A45C0470501CD881D889604504D1DD817B
:1073A0000120087003205871012038BD2DE9F04FED
:1073B00085B0934603F00702DFF81890DDF838C077
:1073C000012A15D013F0070F19D0022A76D070E0E9
:1073D00014871100EC05002054464953081600207C
:1073E00068C001006CC0010070C00100F0150020F1
:1073F000022089F805000020A9F80E0059E00024B9
:1074000040274FF001081BF0010F28D0BA46042294
:1074100003A95046FAF754FE042201A94820FAF7BE
:107420004FFEFB490398884240D101980025B5EBF7
:10743000900F10D20AEB850004226946FAF740FE4D
:107440000098032D044408BF06466D1C0198B5EB57
:10745000900FEFD304B93446B8F1000F26D01BF0DB
:10746000020F1DD00020042202A9FBF777F9E94999
:10747000029888421AD10025B5EB970F0DD2A800CB
:1074800004226946FBF76AF90098062D044408BFF8
:1074900006466D1CB5EB970FF1D3002C08BF3446A0
:1074A000B8F1000F18BFC9F82C4002D10020C9F86C
:1074B0002C0005B00020BDE8F08FFFE799F805200B
:1074C000022A1AD1B9F80E2062450AD2C2F103038A
:1074D000D9F82C40DB0024FA03F30370501CA9F800
:1074E0000E00B9F80E00604507D10020A9F80E0083
:1074F00001200870032089F8050005B00120BDE8CF
:10750000F08F10B503F00700012804D100221146C6
:107510001C2001F076FE002010BD70B5044603F07B
:107520000700BD4D0E46012804BF0020E88119D098
:1075300013F0070F02D0022816D013E0E889B74BEA
:1075400003283CBF19680A54401C80B2E881032814
:1075500008D1186890F9022090F9011090F9000004
:10756000FCF7D4FD002070BDFCF719FD0246E88948
:1075700030B101280AD002280ED0032812D018E01A
:1075800014211046FCF714FD207012E0152110465E
:10759000FCF70EFD20700CE016211046FCF708FDEC
:1075A000207006E017211046FCF702FD2070012034
:1075B0003070E889401CE881012070BD13F0070F8E
:1075C00004D003F00702022A05D002E0924900200D
:1075D000C88100207047924A12680270012008702A
:1075E000704730B403F007030024DFF82CC2029A7E
:1075F000012B02D0022B0BD007E005208CF80500F0
:10760000ACF80E4020208CF8060030BC00207047FB
:107610009CF80530052B14D1BCF80E30934205D2EE
:107620009CF806500570581CACF80E00BCF80E0013
:10763000904206D1ACF80E400120087003208CF86F
:10764000050030BC012070472DE9F04383B003F002
:107650000705724E704FDDF828C04FF00008012D6D
:107660000AD013F0070F3B46DB8903F10104A4B2F3
:1076700011D0022D22D01DE001A9684601F092FF31
:107680000520787131680198087031680098487059
:10769000A7F80E800EE0634502D23068C254FC8128
:1076A000F889604506D1A7F80E80306801784078E7
:1076B00001F06FFF03B00020BDE8F0837A79052A5E
:1076C0000ED1634503D23268D25C0270FC81F88926
:1076D000604505D1A7F80E8001200870032078715D
:1076E00003B00120BDE8F08370B503F0070000246B
:1076F000494D4A4EDDF810C0012803D013F0070FA2
:1077000006D043E0EC8130680470306844703DE09E
:10771000E889604503D233681A54401CE88180B27E
:10772000604533D13FA001220068EC810A703168C6
:10773000C2B20978914229D13168C0F30720497853
:10774000814223D11C2600244FF4801505EB043020
:10775000FAF734FE022808BF70BD601CC4B2B44200
:10776000F4D3032600244FF48E1505EB0430FAF70A
:1077700025FE022808BF70BD601CC4B2B442F4D319
:107780002948FAF71BFE022808BF70BD002070BD13
:1077900010B503F00700012808BF02F0D5F900205A
:1077A00010BD70B503F007041B4D012C09D013F078
:1077B000070F2B46D3F82CC0DB8908D0022C17D03A
:1077C00014E00020E88104F0C4FDE8620EE0002B24
:1077D00004BF1002E86206D0012B04D14CEA02007B
:1077E000E86204F0AFFDE889401CE881002070BD2C
:1077F000002B04BF4FEA1C21017005D0012B03D1DF
:1078000080F800C001200870581CE881012070BD7C
:107810005446435354464953EC0500201487110045
:107820007005002055AC000000FE110070B5064642
:1078300003F00700F84C0D46012808BF00200DD0CA
:1078400013F0070F02D002280BD008E0E0890028CF
:1078500004BF104607F0ACF8E089401CE08100202E
:1078600070BD07F0A2F830700120287070BD70B5AF
:1078700003F0070CE84D0E460446BCF1010F06D09C
:1078800013F0070F07D0BCF1020F1CD019E0002045
:10789000E881288215E0E889002804BF1002E86228
:1078A0000CD001280AD1E86A1043E862F9F798FB86
:1078B000A88D80B2FDF73FFCF9F795FCE889401CE4
:1078C000E881002070BD288A02280CD2FEF73BFC1C
:1078D0002A8A002A04BF000A207004D0012A02D19B
:1078E000207001203070288A401C2882012070BD41
:1078F00010B513F0070F04D003F00702022A08D0D6
:1079000005E0002A14BF0120002006F046F90020FF
:1079100010BDC24A92F85420D208027001200870AB
:1079200010BD0020704770B503F007020026BC4C64
:10793000B94DDDF810C0012A02D0022A15D012E09C
:1079400005F02BF921680870FDF790F82168487060
:1079500003F0FAF821688870FDF78BF82168C87089
:1079600005206871EE81002070BD6A79052A0FD16B
:10797000EA89624504D223689B5C0370501CE8814D
:10798000E889604504D1EE81012008700320687108
:10799000012070BD70B5064603F007000D460228B1
:1079A0001CBF002070BD01F046FC002814BF01245C
:1079B000002401F043FC002814BF022200222243CD
:1079C00032700120287070BD30B403F00703944A70
:1079D0000024914DDDF808C0012B02D0022B4AD0C3
:1079E00046E090490868904B98422FD14868B0F51E
:1079F000887F2BD8C868FF282EBFFF20C868C0B278
:107A0000136818700869FF283ABF0869C0B2FF20E0
:107A1000136858704869FF283ABF4869C0B2FF2010
:107A20001368987088681368000AD87088691368AA
:107A3000187188691368000A58718869030C106806
:107A4000837188691168000EC87110E010680470B5
:107A500010684470106884701168FF20C870116845
:107A6000087111684871116888711168C871EC81DA
:107A700030BC00207047EB89634504D21268D25CA9
:107A80000270581CE881E889604502D1EC81012030
:107A9000087030BC012070472DE9F04103F0070168
:107AA00000255D4C0646012904BFE561E58101D052
:107AB000022902D00020BDE8F081207F584F00F05D
:107AC0000701E1812078084304D1386802F0BAF850
:107AD00001202070E189052928BF25703868405CA5
:107AE0003070E069401CE0610120BDE8F08170B5B4
:107AF00003F0070200254A4B474CDDF810C0012A6D
:107B000002D0022A08D005E0186802F09BF8052090
:107B10006071E581002070BD6279052A0FD1E2898C
:107B2000624504D21B689B5C0370501CE081E089B5
:107B3000604504D1E58101200870032060710120B7
:107B400070BD70B503F007020025334C012A02D046
:107B5000022A11D00EE0052060710021E58108465F
:107B600001F020FD4FF6FF7101EA4000608201F054
:107B700025FDA061002070BD6279052A16D1E28939
:107B8000B4F812C0624507D212F0010F1CBFA379EE
:107B900003700DD0501CE081E089604506D1E5817D
:107BA000012008700320607101F016FD012070BDF6
:107BB000A66922F00103F35A1E0A0670A371E9E7D1
:107BC0007FB51C460E46054613F0070F08D103F09B
:107BD000FBF828B1012202A91D2001F012FB03E0ED
:107BE00004F00700022802D004B0002070BD01F0AC
:107BF000B2FD28700120307004B070BD2DE9F04155
:107C000003F007020027044E88460546012A0DD0DE
:107C1000022A16D012E00000EC050020F80F002028
:107C20001487110014160020544352460520707129
:107C3000F7810A20708201F0C1FCB0610020BDE82C
:107C4000F0817079052818D1F289708A824208D2B1
:107C500012F0010F1CBFB079287011D0F089401CC0
:107C6000F081F089718A884207D1F781012088F874
:107C700000000320707101F0AFFC0120BDE8F0812D
:107C8000002401F068FD012804D1F089B16920F0D9
:107C900001000C5A200A2870B471DFE77FB50D4649
:107CA000044613F0070F04D003F00700022808D0A1
:107CB00004E0012202A90A2001F0A3FA04B0002086
:107CC00070BD04F06AFF20700120287004B070BD00
:107CD000F8B503F007020025FF4C0E460746012ABF
:107CE00002D0022A0ED00BE00520607103F079FA71
:107CF000206300281ABF44F26440A082A582E58177
:107D00000020F8BD6079052822D1E289A08A694661
:107D1000824214D212F0030F08D10422206BFAF72A
:107D2000CFF90098E062206B001D206394F82C00CE
:107D30003870E06A000AE062E089401CE081E08976
:107D4000A18A884204D1E58101203070032060714E
:107D50000120F8BD10B513F0070F04D003F007029F
:107D6000022A0DD00AE0012A05D0002A04BF012012
:107D7000FAF7CFFF02E00120FAF7C0FF002010BDA4
:107D8000D64A1268126802F00202027001200870DE
:107D900010BD70B50D46044613F0070F04D003F074
:107DA0000700022808D005E0002A14BF01200020A7
:107DB00001F0BCFE002070BD01F0BFFE002814BF22
:107DC0000122002222700120287070BD70B503F0DE
:107DD0000700C14D1446012808BF002016D013F03B
:107DE000070F14D1E889002808BFAA710CD0012818
:107DF0000AD1A879FAF7BFFFA8792040FAF77EFFE9
:107E0000A879A043FAF785FFE889401CE8810020A3
:107E100070BD2DE9F00103F00704AF4E059F012C62
:107E200004BF0020F08135D013F0070FAA4BAC4DF2
:107E3000DB8903F1010C1FFA8CFC02D0022C2DD03F
:107E400028E0A8490868C254781E834220D10868F7
:107E5000007830B101280AD002280ED0032812D0B1
:107E600016E008682968407881F8800110E0086809
:107E70002968407881F881010AE00868296840781B
:107E800081F8820104E008682968407881F883015C
:107E9000A6F80EC0BDE8F00100207047904A1268B5
:107EA00013B1012B0AD014E092F8801101F00F03F6
:107EB00092F8811163F31F1101700AE092F8823188
:107EC00092F8832103F00F0363F31F120270012065
:107ED0000870A6F80EC0BDE8F0010120704710B48C
:107EE000DFF804C213F0070F04D003F00702022AE0
:107EF00018D014E0012A01D04AB110E0DCF80000EB
:107F0000806ADCF8001020F00300886207E0DCF8EB
:107F10000000806ADCF8001040F00300886210BCAA
:107F200000207047DCF80020926A0270012008707F
:107F300010BC704770B503F007000025664C0E4674
:107F4000012806D013F0070F04BF6079022805D07E
:107F500019E002206071E581E56214E0E089A18A00
:107F6000884207D2614811460068FBF742FBE0896E
:107F7000401CE081A18A80B2884204D1E5810120C1
:107F8000307003206071002070BD2DE9F04103F0D6
:107F900007020025504C0E460746012A02D0022A4D
:107FA00006D002E002206071E5810020BDE8F0818A
:107FB0006079022814D1E189A08A814207D24B4816
:107FC0000068FBF744FB3870E089401CE081E089E1
:107FD000A18A884204D1E5810120307003206071BC
:107FE0000120BDE8F08110B503F007023A4C012AE8
:107FF00002D0022A27D024E003F0F6F8002300285C
:1080000004BF2363A3821BD000F1540121634168A4
:10801000B1F5887F90F820100CD390F8212001EB67
:10802000020C01FB02C190F8222090F823001044BA
:10803000084404E090F822000A1801FB0020A08206
:10804000E381002010BDE289A38A9A4207D2D4F8C6
:1080500030C01CF802C080F800C0501CE081E089EC
:10806000984204BF01200870012010BD10B513F024
:10807000070F04D003F00702022A05D002E01046E1
:1080800001F0B7FA002010BD194A127802700120E1
:10809000087010BD1FB513F0070F04D1012202A90B
:1080A000092001F0AEF804B0002010BD70B503F057
:1080B00007000949012804BF0020C88130D013F00F
:1080C000070F2DD1C889074C03283CBF23681A54D9
:1080D000401C80B2C8810DE0EC050020DC86110058
:1080E000E806002014871100E486110000871100C3
:1080F00031060020032813D1F8F784FF2068B0F878
:10810000010045BAF8F79CFD040018BFF9F7B6F86E
:1081100029460020F8F7EBFC002C18BFF9F7B0F85F
:10812000002070BD70B503F00700F949012804BFB5
:108130000020C88124D013F0070F21D1C889F54D44
:1081400002283CBF2B681A54401C80B2C881022808
:1081500016D1F8F757FFF8F773FD040018BFF9F7C9
:108160008DF82868007818B128684078F8F7C3FCC3
:1081700028684078F8F7BFFC002C18BFF9F780F8A2
:10818000002070BD13F0070F04BFE148C27000204B
:1081900070477FB50D46044613F0070F04D003F077
:1081A0000700022808D004E0012202A90E2001F0F5
:1081B00028F804B0002070BD04F0B6FC002814BFFD
:1081C0000122002222700120287004B070BD7FB50A
:1081D0000D46044613F0070F04D003F007000228F1
:1081E00008D004E0012202A90F2001F00AF804B02F
:1081F000002070BD04F089FC20700120287004B0BC
:1082000070BD10B503F00700DFF804C30299012820
:1082100004BF0020ACF80E001AD013F0070F17D1DE
:10822000BCF80E00BB4B03283CBF1C682254401C0A
:1082300080B2ACF80E0088420AD118681968B0F80C
:108240000100097840BA00B2002908BFFCF770FFAE
:10825000002010BD10B503F00700DFF8B4C202998A
:10826000012804BF0020ACF80E0017D013F0070F50
:1082700014D1BCF80E00A74B03283CBF1C68225445
:10828000401C80B2ACF80E00884207D11868B0F8E4
:10829000010041BA18680078F9F77FFB002010BD93
:1082A00070B503F007029A4CDDF810C0012A02D025
:1082B000022A07D004E00020E081FAF7EDFFE06237
:1082C000002070BDE289624506D2C2F10303E56A6F
:1082D000DB0025FA03F30370501C80B2E081604597
:1082E00004BF01200870012070BD70B5044603F082
:1082F000070C0020864DBCF1010F06D013F0070FCC
:1083000007D0BCF1020F13D010E0E8812882A871D9
:108310000CE0E889002808BFAA7104D001227E4938
:10832000102000F06EFFE889401CE881002070BD3D
:108330002A8A3AB1207001200870288A401C2882BD
:10834000012070BD04F075FC2070F6E770B50D4695
:10835000044613F0070F04D003F00700022805D0ED
:1083600002E0104606F0AEF8002070BD06F0ADF851
:1083700020700120287070BD10B513F0070F1FD1B9
:10838000500048F6B801B1FBF0F4644903200968D5
:10839000C86101217F20F8F757F8E1B24FF48470EB
:1083A000F8F752F820460FF04CFB5D4A5D4B0FF09A
:1083B000AFFB0FF019FBC1B24FF48570F8F744F82A
:1083C000002010BD10B513F0070F4ED1122A4CD269
:1083D000DFE802F0090E132B2B2B2B303336393C00
:1083E0004B4B4B3F424750490020096808773CE01F
:1083F0004D4901200968087737E04849032009689A
:10840000C86101217F20F8F71FF815214FF487700C
:10841000F8F71AF875214FF48470F8F715F84D2124
:108420004FF48570F8F710F81FE00021D01E04F01B
:10843000FCFC1AE0F9F783FD17E0F8F7D4FE14E02E
:10844000F8F7CEFD11E004F0F4FA0EE004F004FBBE
:108450000BE0FDF715FE08E03349022009680886A5
:1084600003E03149002009680886002010BD10B5DE
:10847000144613F0070F16D1072C14D827490320F0
:108480000968C86102217F20F7F7DEFF052040EA76
:10849000041140F20220F7F7D7FF04F188014FF4EE
:1084A0000170F7F7D1FF002010BD7FB50C460546DF
:1084B00013F0070F04D003F00700022808D004E0EF
:1084C000012202A9062000F09CFE04B0002070BD2D
:1084D000FCF7CCFA022808BF00200BD0032808BF05
:1084E000022007D0042808BF032003D0052814BFAA
:1084F000FF20012028700120207004B070BD10B54D
:10850000104613F0070F08BF04F029FB002010BD30
:10851000EC05002014871100F2050020E886110008
:108520001F85EB51B81EE53FE806002010B5104648
:1085300013F0070F08BF04F01EFB002010BD70B53C
:10854000044603F007000D4602281CBF002070BD42
:1085500004F01EFB20700120287070BD70B403F081
:1085600007020024FE4BDDF80CC0012A05D0022AC8
:1085700004BF5A79022A0AD01BE002205871F94838
:10858000DC816FF07F410068081AD86211E0DA8957
:10859000624506D2DE6AD50026FA05F50570501C44
:1085A000D881D889604504D1DC810120087003207E
:1085B000587170BC0120704713F0070F04BFEA48E0
:1085C00002700020704710B5944603F00700E4499C
:1085D000029A012804BF0020C88112D013F0070FAF
:1085E0000FD1C889E14B90423CBF1C6804F800C021
:1085F000401C80B2C881904203D10D20196800F060
:1086000000FE002010BD70B503F00704D44D012C0E
:108610000AD0AC4613F0070FBCF81230DCF830C0BB
:1086200006D0022C21D01EE00020E88128821AE02A
:10863000E889002808BF2A6312D0012804BF501C13
:1086400068820DD0022816BFC11EAA82994207D2A5
:10865000297D0844C01EC1B20CF0FF00F9F751FBA0
:10866000E889401CE881002070BDFF22027093B1B0
:108670002A8A9444521CBCF5807F0BD20CF5801CD6
:108680000CF5F83C9CF800C080F800C09A4204BF8A
:10869000012008702A82012070BD2DE9F04103F00D
:1086A00007050026AE4C9446012D04BFE6812682C4
:1086B00024D013F0070FAA4B5A8A1B6B02D0022D4D
:1086C00028D01BE0E089002808BFC4F830C012D0D1
:1086D000012816D0A549801E90423CBF0D6805F8C0
:1086E00000C0401C904206D103F58010096800F5D7
:1086F000F830FAF7E1F8E089401CE0810020BDE89D
:10870000F0810CF1010060821844B0F5807F88BFD1
:108710006682F0E74FF0FF0C80F800C09AB1258A1E
:1087200003EB050C6B1CBCF5807F0BD20CF5801C99
:108730000CF5F83C9CF800C080F800C0934204BFE0
:108740000120087023820120BDE8F08110B5944615
:1087500003F007008249029A012804BF0020C88163
:1087600012D013F0070F0FD1C889804B90423CBF45
:108770001C6804F800C0401C80B2C881904203D13C
:108780000220196800F03DFD002010BD10B5944690
:1087900003F007007249029A012804BF0020C88133
:1087A00012D013F0070F0FD1C889704B90423CBF15
:1087B0001C6804F800C0401C80B2C881904203D1FC
:1087C0000320196800F01DFD002010BD13F0070FF5
:1087D00005D003F00700022804BF012070470020E5
:1087E00070471FB513F0070F04D1012202A9112011
:1087F00000F007FD04B0002010BD03F00701DFF812
:1088000060C10098012907D013F0070F04BF9CF83E
:108810000510012909D01FE001208CF80500002077
:10882000ACF80E00CCF8280014E0BCF80E10814221
:1088300008D2DCF82830491C42EA0322CCF8282070
:10884000ACF80E1089B2814206D103208CF80500E5
:10885000DCF82800CCF830000020704703F0070057
:108860003F494FF0010C012806D013F0070F04BF59
:108870004879012807D014E081F805C00020C8819C
:10888000087148620DE0C889002804BF0A71A1F888
:108890000EC006D0012806D00323022818BF4B7152
:1088A00006D000207047100248620220C881F8E715
:1088B000486A104348624B71F3E770B5154613F0F0
:1088C000070F0FD12A49264C09682079C861A08C6E
:1088D000C0F307217F20F7F7B7FD94F8240029465D
:1088E000F7F7B2FD002070BD70B5044603F0070035
:1088F0000D4602281CBF002070BD1948818C0079EC
:1089000089B2F7F755FD20700120287070BD03F083
:1089100007011348012904BF0021C18103D013F0CE
:10892000070F08BF827200207047F8B503F00702F6
:1089300000230E4E0A4F012A02D0022A2FD02CE02B
:108940000024022000937871FB81B87A4FF44835F7
:10895000834222DA042269462846F9F7B1FB09E08E
:10896000EC050020A005002032050020148711002E
:10897000E886110031680098085531680098214454
:10898000000A48700098000C88700098000EC870AB
:10899000B87A241D2D1D8442DCDB0020F8BD7A79D5
:1089A000022A15D1FA8997F80AC0624507D2D6F88B
:1089B00000C01CF802C080F800C0501CF881F88983
:1089C000BA7A904204D1FB810120087003207871AB
:1089D0000120F8BD10B503F00700FC49012804BFD1
:1089E0000020C88118D013F0070F15D1C88991F85D
:1089F0000AC0F74B604505D2D3F800C00CF8002040
:108A0000401CC8818A7A80B2904205D18A7A4FF49C
:108A100048301968F9F750FF002010BD70B54FF4C9
:108A200044324FF4407101FB00240120F8F71BF998
:108A3000FDF726FBFCF778F90546F8F7D4FBE34B86
:108A40004FF4107220461C639A822946BDE870409C
:108A5000F9F732BF70B513F0070F18D14FF4443156
:108A60004FF4407000FB02140120F8F7FCF8FDF70A
:108A700007FBFCF759F90546F8F7B5FBD34B4FF464
:108A8000107220461C639A822946F9F715FF0020D0
:108A900070BD13F0070F04BFCC484272002070472E
:108AA000F8B503F007020027C94EDFF820C3012AFA
:108AB00002D0022A2DD02AE09CF80900002400EB05
:108AC00040004FF4443101EB0025022000978CF860
:108AD0000500ACF80E704FF41070ACF814000422CE
:108AE00069462846F9F7ECFA316800982D1D0855BB
:108AF000316800982144000A48700098241D000C39
:108B000088700098000EC870B4F5107FE7DB002075
:108B1000F8BD9CF80520022A16D1BCF80E20BCF83E
:108B200014309A4205D23468A45C0470501CACF82E
:108B30000E00BCF80E00984206D1ACF80E70012071
:108B4000087003208CF805000120F8BD03F0070130
:108B5000DFF878C20098012907D013F0070F04BF8F
:108B60009CF80510022909D01FE002208CF80500AE
:108B70000020ACF80E00CCF82C0016E0BCF80E106B
:108B8000814208D2DCF82C30491C42EA0322CCF89E
:108B90002C20ACF80E1089B2814206D1BCF82C0012
:108BA000ACF8140003208CF805000020704770B565
:108BB00003F007000025854C0E46012806D013F06F
:108BC000070F04BF6079022805D023E002206071FE
:108BD000E581E5621EE0E089A18A884211D2E16A5E
:108BE000090A41EA0261401CE162E08110F0030FD2
:108BF00007D104227749206BF9F75EFE206B001D38
:108C00002063E089A18A884204D1E5810120307087
:108C100003206071002070BDF8B503F00702002545
:108C20006A4C0E460746012A02D0022A05D002E00D
:108C300002206071E5810020F8BD6079022822D110
:108C4000E289A08A824215D212F0030F09D10422D0
:108C50006946206BF9F734FA0098E062206B001D3A
:108C6000206394F82C003870E06A000AE062E08922
:108C7000401CE081E089A18A884204D1E58101207D
:108C80003070032060710120F8BD70B403F007025A
:108C900000254E4C012A02D0022A06D002E0022012
:108CA0006071E58170BC002070476279022A1CD196
:108CB000E289B4F814C062450FD212F0030F04D158
:108CC000236B53F8046BC4E90B6394F82C300370E6
:108CD000E06A000AE062501CE081E089604504D14E
:108CE000E581012008700320607170BC012070478D
:108CF00030B403F007000024DFF8D0C0012807D00B
:108D000013F0070F04BF9CF80500022808D025E0E7
:108D100002208CF80500ACF80E40CCF82C401DE089
:108D2000BCF80E00BCF8143098420CD2DCF82C5081
:108D30002D0A45EA0262401CCCF82C20ACF80E004B
:108D400010F0030F0DD0BCF80E00984206D1ACF81D
:108D50000E400120087003208CF8050030BC002074
:108D60007047DCF83000B0F5002F28BF0260001D0E
:108D7000CCF83000E7E730B403F007040025DFF853
:108D80004CC0012C08BFACF80E503ED013F0070FBA
:108D900002D0022C3CD038E0042A08BF4FF42C301B
:108DA00031D01DDC002A08BF4FF480102BD0012ADF
:108DB00008BF094827D0022A08BF4FF48E1022D0DE
:108DC000032A08BF05481ED01AE00000EC05002069
:108DD000148711001806002000FE110000F8110091
:108DE000052A08BFF8480ED0F848102A00680AD0B3
:108DF000112A08BFF64806D0202A08BFB43002D096
:108E0000CCF8285001E0CCF8280030BC0020704796
:108E1000BCF80E20042A07D2C2F10303DCF8284074
:108E2000DB0024FA03F30370501C80B2ACF80E0090
:108E3000042824BF01200870012030BC704710B501
:108E400003F00700012804D1002211460C2000F095
:108E5000D8F9002010BD2DE9F04103F0070CDD4EDC
:108E6000069D0F460446BCF1010F04BF0020F081AF
:108E700017D0D84913F0070FCB8903D0BCF1020FEC
:108E800012D00EE0D449022B3CBF0868C254581CD3
:108E900080B2F081A84204D102220968052000F0C6
:108EA000B0F90020BDE8F08113B1012B04D008E037
:108EB000FBF7DCFD207004E0FBF7DBFD20700120F8
:108EC0003870F089401CF0810120BDE8F08170B558
:108ED00003F00700BF4D012803D013F0070F05D0A2
:108EE00024E00020A862E862A8711EE0B949EC897C
:108EF00091F806C0886A0CEB0201CBB2022C03D2B7
:108F000042EA0020A86206E0B249042CC96A04D2F1
:108F100042EA0120E862AB7105E0052C03D262450C
:108F200008BF00F051FFE889401CE881002070BDB7
:108F300010B503F007011046012905D013F0070F03
:108F400008BF00F01BF904E0A24900208862887184
:108F5000C881002010BD10B5104613F0070F08BFE0
:108F600000F00CF9002010BD70B5032600244FF46A
:108F70008E1505EB0430F9F721FA022808BF70BD01
:108F8000601CC4B2B442F4D3012070BD30B403F00D
:108F900007030024DFF83CC2029A012B02D0022B07
:108FA0000CD008E005208CF80500ACF80E409CF8C9
:108FB00008008CF8060030BC002070479CF8053093
:108FC000052B14D1BCF80E30934205D29CF8065004
:108FD0000570581CACF80E00BCF80E00904206D18B
:108FE000ACF80E400120087003208CF8050030BC5E
:108FF000012070472DE9F04778A0DDF820C0006817
:1090000003F007050027734E734C012D03D013F0B6
:10901000070F06D034E0F78120680770206847709A
:109020002EE0F389634503D22568EA545A1CF28185
:10903000F289624524D1F7814FF0010881F8008060
:109040002168C2B2097891421AD12168C0F3072081
:109050004978814214D1032500244FF48E1909EB7D
:109060000430F9F7ABF9022804D0601CC4B2AC425A
:10907000F5D34046012806BF86F80880F77137729D
:109080000020BDE8F0872DE9F0414FF0000C03F01F
:109090000700534E4F4C6546012803D013F0070FCD
:1090A0000CD068E06570A5812562A570002046F8A7
:1090B0002050401CC0B24028F9D35CE060780528FD
:1090C0003CBF401C6070C0B2012808BF100222D013
:1090D00040490228CB8A08BF98181CD024BFA18918
:1090E0008B4248D93F4F01F0030001F101083A5487
:1090F000A7F134004FF48E12006A984502EB00206D
:1091000008BF002109D1491CC9B20429FBD3344945
:10911000F9F7F5F926E0E0822DE0032232EA0101B9
:1091200020D17A5CCB009A40491CC9B242EA0C0CAF
:109130000429F6D3A17801F03F02491CC9B246F8D0
:1091400022C0A17040290DD12549F9F7D8F9A570A1
:10915000206A401C2062002046F82050401CC0B20B
:109160004028F9D3A089401C80B2A081E18A8842BE
:1091700004BF0120E0710020BDE8F08110B5154C5E
:109180002146E2898B6A8979022A05D240EA0322C4
:109190000844A262A07112E0B2F5817F08D20E49A4
:1091A0000968114401F8020CA1790844A07106E095
:1091B00008BF884203D10A49184600F01FFEE08923
:1091C000401CE08110BD000000F01100E806002006
:1091D000F80F0020EC0500201487110055AC0000AA
:1091E0001438002020060020D94800210170417069
:1091F000C1700171D74A08461154401C0428FBD3A2
:10920000704710B4D24C6378002B1EBF002010BCF6
:109210007047E07022710020002A88BFCD4B06D92C
:1092200011F800C003F800C0401C8242F8D80120A9
:10923000607010BC7047C64840787047C44880785A
:109240007047C34900208870704770B50024FAF752
:10925000E0FABF4D6878012806D100F012F8044604
:109260001E20E87000206870FBF700FC022802D185
:1092700001F066FD18B9002C04BF002070BD01206C
:1092800070BD2DE9F05FB2480024C0781E2880F040
:109290005B81DFE800F0121E2C350F41FD4597A0E1
:1092A000A6ABE4FCB9C7CCD19797979797979797B8
:1092B0009797FBFAFBF739FC16E0FBF7D7FBA44CBA
:1092C0006071A01D01780120FBF7E2FB0120A07076
:1092D0000AE0A048007801F081FF01210320FBF79C
:1092E000D7FB9B4901208870012400F02DB99948D3
:1092F0004178007841EA002003F0CAFA00F024B96E
:109300009448007803F0C9FA04210320FBF7C0FB5E
:109310008F4901208870E7E78E48417800789BE00C
:10932000DFF82C8200264FF0010A08F1060BB14647
:10933000012788F802A088F8019098F80000D0BBB7
:109340009BF8005088F800A015F0100F11D00120F4
:10935000F7F789FCFBF78DFBA8B3F8F709F9FF21B4
:109360000F20FBF70CFF074645F001050020F7F73B
:10937000D4FC15F0010F1CD0FAF786FB0020FAF799
:10938000F2FD0120F7F76FFCFAF7DDFC0146022041
:10939000FBF776FD0220FBF751FDF7F724FFFAF704
:1093A000D2FCFAF7CAFDFAF7CEFC4FF490610DF04B
:1093B00074FE88F8009088F80290002F1CBF761C7D
:1093C000032EB5DBC0E0FFE7F8F7D2F8FF210F204E
:1093D000FBF771FFC7E75F480078401E01F016FCFD
:1093E00082E75C48007803F0DDFB7DE759480078B0
:1093F000002804BF0021032003D003F0AAFB01468C
:109400000220FBF745FB9FE0524D2878002818BF4B
:10941000012003F07FFB2878002818BF012000F00E
:109420000BFD91E04B48007803F065FB5CE7494891
:10943000007803F0CAFB87E04648007820B1012895
:1094400056D0022804D07FE04348F8F73FFF7BE086
:1094500001F0F7FC00210420FBF71AFB44E73C482D
:109460004FF0000880F801804646454672B6F9F78D
:10947000CFFF48B1FAF78AF80646FAF767F8FAF725
:109480008BF80546FAF772F803E059E055E043E03F
:109490002FE0F7F7B7FDF7F7D3FB8146F7F771FF3A
:1094A000F9F7ECFE070018BFF9F7E7FE4FF4187064
:1094B000F9F7BFFE62B62948C0F80080F8F7C4FB90
:1094C00072B6B9F1000F03D0F7F79CFDF7F78BFEEA
:1094D000F9F79EFF38B1002E18BFF9F79BFF002D5A
:1094E00018BFF9F7D6FF002F18BFF9F7C4FE62B610
:1094F0002AE018480078012804BF02210520ABD0DB
:10950000022804BF00210320A6D0032819BF02218E
:109510000846002104209FE70E480178427841EA7E
:1095200002218278C078120442EA006041EA000217
:109530006221072002F013FF06E0FAF722FED3E6CD
:109540000448007800F0F3F82046BDE8F09F0000E2
:10955000240600202A06002000FE110064050020D9
:1095600002460020022928BF704752B1012A18BFC5
:10957000704701EB810000EBC100FE4901EB0010D8
:10958000704701EB410000EBC100FB4901EBC0104B
:10959000704700FB01F2B2F5307F9CBFF74AC2E989
:1095A000020170470028F54A926818BF0260F3482C
:1095B0000029C06818BF086050437047EF48012178
:1095C0000171007880F0010000EB400101EBC00068
:1095D000E94901EBC0107047E8488278002132B1B8
:1095E000C27822B9027882F00102027081700171A2
:1095F0007047E24910B54C7848701E2808BF00201B
:1096000008D01F2808BF012004D00E2808BF8120E1
:1096100002D000E00870012003F0D7FA204610BD08
:10962000F0B4D64E96F800C0B5680CEB4C0404EBD1
:10963000CC0CD14C8D4204EBCC1C03FB05F40CEBA1
:10964000440C34BF2C460C46F768FE1A964228BFDD
:1096500016461A44974224BF0023002E9CBFF0BC3C
:1096600070470022002C06D930F812702CF81270C6
:10967000521C9442F8D85B1C0CEB450C00EB4100EB
:10968000B342EED3F0BC70472DE9F041BB4F144616
:109690008C4601467A7806981D468A4218BFBDE876
:1096A000F0810121F970012802D0022825D02AE09A
:1096B0003878BE6800EB400101EBC000AE49A6421D
:1096C00001EBC01134BF32462246F868A84238BFC9
:1096D00005460023002D16D90020002A06D91CF8C3
:1096E000007021F81070401C8242F8D85B1C01EB1E
:1096F0004601A444AB42EFD305E000232A462146AD
:109700006046FFF78DFFBDE8F04100F0EBB910B502
:10971000002808BF10BD01229849CA70497800236B
:109720000821FFF77DFFBDE8104000F0DBB9934A48
:1097300001281146D071497808D000280CBF24298F
:10974000704730205070012003F03FBA2420507041
:10975000012003F03ABA8948C079704770B4DFF845
:1097600020C2DCF800C0DCF818C01CF0040F1ABFDF
:10977000012424EA0C060CF0010605680C68002E92
:109780001CBF1B1B5C1E1CF0020F1CBF521B551E76
:109790001CF0040F19BF04600D6005600C6070BC04
:1097A000704710B5002808BF10BD01227349CA7068
:1097B0004A787449DFF8D0C102220B789CF8001077
:1097C000FFF72EFFBDE8104000F08CB92DE9F04303
:1097D0006A498BB00122CA706C4A49781578694A87
:1097E0002529147824BF0BB0BDE8F083DFE801F031
:1097F000134D4D4D134D4D4D4D4D4D4D4D4D4DFD5D
:109800004D555555FDFDFDFDFDFDFDFDFD4DFDFDE0
:10981000FD7D7DFD8500002800F0028106460027C1
:10982000F7F7BEFD5FEA000C16D0544908788F6840
:1098300000EB400202EBC0004F4ABD4202EBC010F9
:1098400094BF2B463B46C968A14238BF0C46002155
:10985000002C06D800F0E4B83B46224629463046A4
:1098600048E00022002B08D91CF9028036F8188045
:1098700020F81280521C9342F6D8491C00EB470096
:1098800006EB4506A142ECD3CAE0002870D00023C5
:1098900022462946FFF7C4FEC2E03D480078012871
:1098A00084BF3C480478F7F72DFC10F0020F18BF76
:1098B000641CFBF739FA002205FB04F3002BC4BF3C
:1098C000DFF8B8C02C4C53DD10F8015B9CF8001099
:1098D00001EB410606EBC10104EBC11121F8125066
:1098E000511C8AB29342EFDC9AE0002840D000235A
:1098F000A21C2946FFF794FE92E0002838D00646C5
:109900001F480068007E10F0040F0EBFA946A14654
:109910002C464FEA9902A1080591A9EB99000691FE
:1099200000924FEA5901401ECDE9010161080791FB
:10993000A4EB9401491E08910991CDE90320234627
:109940004A4605A96846FFF709FF23464A4605AF80
:1099500006A9E84601A8FFF701FF23464A4607F19A
:10996000080108F10800FFF7F9FE23464A4613E014
:1099700056E0000014470020143C00203006002070
:10998000E8060020BF050020C5050020BE05002018
:10999000C0050020C205002007F10C0108F10C00F1
:1099A000FFF7DCFE23464A4607F1100108F11000DC
:1099B000FFF7D4FE58480078002200EB400101EB8D
:1099C000C0005649914601EBC01020F8129058F89B
:1099D0002210A1F1010C491C61451ED357F8221039
:1099E0004B1E491C994211D300E01EE003FB05C148
:1099F00036F9114030F912108C42C8BF20F81240DD
:109A000057F822105B1C491C9942EDD258F82210DD
:109A10000CF1010C491C6145E0D2521C052AD4D33B
:109A20000BB0BDE8F04300F05DB80BB0BDE8F083CB
:109A300039491E288A79887108BF002003D01F2861
:109A400008BF012000D148711046704770B50D461F
:109A500031490122CA70324A49781678314A21299F
:109A600014781EBF2229232970BD002818BF002D9D
:109A700011D0002322463146FFF7D2FD631C01229C
:109A800021462846FFF7CCFD05EB4400A31C01222C
:109A90003146FFF7C5FDBDE8704000F023B810B5B2
:109AA0001D4C6178002904BF4068FFF78FFE607885
:109AB000112804BF0020FFF789FE6078122804BF38
:109AC0000020FFF783FE6078132803D1FCF798FB92
:109AD000FFF77CFE60781D2818BF10BD1248BDE856
:109AE000104073E670B5F9F7A0FB00F008060820F7
:109AF000F9F796FB084C20790025002801BF207853
:109B000080F001002070A5701CBF0120A0703046BD
:109B1000F9F782FBE57070BD30060020143C002090
:109B2000BE050020BF05002080680020A349002852
:109B300014BF0020012008707047A048007800285A
:109B40000CBF01200020704710B59C4C20780028E5
:109B50001CBF0120F9F7D2F800206060A060E0602F
:109B60002061606110BD10B5944C207800281CBFA6
:109B70000120F9F7C3F800206060A060E060206178
:109B8000606110BD70B50446F9F74FFB00F00805A1
:109B90000820F9F745FB894A89490023106901EB40
:109BA000C001401C1061B0F5807F28BF1361207890
:109BB000087060784870A0788870E078C870207964
:109BC000087160794871A0798871E079C87150692D
:109BD000B0F5807F3CBF401C506116D31D2008703B
:109BE00001204870207888706078C870A07808716B
:109BF000E0784871207988716079C871D068401C1C
:109C0000D060B0F5807F28BFD360506840F001007D
:109C10005060107800281CBF0120F9F77AF8284618
:109C2000F9F7FAFA012070BD10B50178022211F09F
:109C300003011CBF0129022902D1FFF7A3FF02463D
:109C4000104610BD2DE9F0415C4E04463046726866
:109C500003780025002A1CBF00204FF0010C54D0CF
:109C6000B1680CFA01F7174207D1491CB1600D2900
:109C700028BFB560401C0D28F2D3B16809B3514824
:109C800000EBC1000CFA01F122EA01010838716011
:109C9000317D02782270427862708278A270C27838
:109CA000E27002792271427962718279A271C0797F
:109CB00001F03F0100F0C0000843E0717068D8B9BE
:109CC00015E0716909B33E48D6F80CC000EBCC0032
:109CD0000CF1010CC6F80CC0BCF5807F28BFF56004
:109CE000491E716104BF22F001017160D0E7002BB1
:109CF0001CBF0120F9F702F8B068401CB0600D28C5
:109D000028BFB5600120BDE8F081002B1CBF0120F9
:109D1000F8F7F4FF25706570A570E5702571657121
:109D2000A571E5710220BDE8F081244910B44A68AC
:109D300000204C69002A19BF01210B4610BC704756
:109D400003FA01FC1CEA020F18BF401C491C0D2934
:109D5000F6D312F0010F18BF204410BC704700B5B5
:109D60000178427883B0890102F0070241EA82015A
:109D70008DF80010418809098DF8011081880909C2
:109D80008DF80210817801F00F02017962F31F1142
:109D90008DF80310017A8DF80410417A8DF80510C2
:109DA000807900F03F008DF8060000208DF8070054
:109DB0006846FFF7E7FE03B000BD00004006002044
:109DC00014490020B448002070B50E4680280CD2FB
:109DD0008119491E802908D205030024002E04D9C8
:109DE0002846F8F7EBFA012801D0002070BD641C6A
:109DF00005F58055B442F3D3012070BDB0F5006F76
:109E000024BF0020704710B50002F8F778FB012846
:109E100018BF002010BD10B5064CFFF716FA012838
:109E200008BF10BD206801F0D7F8002818BFFAF766
:109E300057FEF2E7E8060020FC4A0028516814BFEC
:109E400041F0010021F0010050607047F74B596864
:109E50000A0E120721F07F4142EA00600843586071
:109E60007047F2484068C0F30360704770B5EF4D2B
:109E7000AA68521CAA604FF0000C0028C8BFC5F8A1
:109E80000CC00ED06A6812F0010F40D0E84BC2F34C
:109E9000036214001B6808D0022A18BF002413D0E4
:109EA00028E0EA68521CEA60ECE70028C8BF0224F8
:109EB00022DC93F81601A96888421BD802240120ED
:109EC000C5F808C0286117E0002918BF0A2402D08D
:109ED00004F069FD10E068B9B3F81201E96888423E
:109EE00038BF0024F4D32869012804BF0024C5F832
:109EF00010C001D094420AD06868010E090720F012
:109F00007F4041EA046108436860012070BD002081
:109F100070BD2DE9F041C54D04460026E86937467D
:109F2000012806D16068F9F712FF286A032808BFE4
:109F3000EF616068B0B103F0E2F90028C8BF012604
:109F40000FDC2888401C2880B9480068017F11F088
:109F5000010F07D0807F2988814203D96068F9F713
:109F6000F6FE2F803046BDE8F04100217EE72DE966
:109F7000F04F06468DB00020AC4F05900024786865
:109F8000A046C0F303654FF0FF308246049070682E
:109F90000DF11809A346D8B1CDE902BACDF800B049
:109FA00000234A4604A9CDF804B000F0C3FB804664
:109FB00000F0BAFB04469F480078012804BF204601
:109FC000FFF704FC04980028C8BFA7F800B002DC23
:109FD0003888401C388096480068017F11F0010FD6
:109FE00015D0B0F814013988814202D838690128A7
:109FF0000DD15B46A7F800B0CDE900B4CDF808B0AC
:10A0000042465146CDF80CB00498FAF704FD84B1ED
:10A01000022D04D0042D04BF0498012809D1306812
:10A02000CDE90004CDF80C906846049904F0C3FC17
:10A0300005900498012818BF00200599FFF716FF26
:10A040000DB0BDE8F08F7C4801680969006841F0F7
:10A0500001010161794801684969026841F40071B0
:10A06000516101680969026841F0040111610168E8
:10A070000969006841F010010161714801680968CF
:10A08000006841F0010101606E48007800226749D4
:10A0900000281CBF4A8070474888B0F57A7F87BF88
:10A0A0004A8030BF401C488070472DE9F04F87B090
:10A0B00004460025052700F0D7FE002804BF07B09E
:10A0C000BDE8F08FFAF7D2FC8146FAF7D2FC804661
:10A0D0000F212046FAF796FD002804BF07B0BDE81F
:10A0E000F08F0420DFF860A1DAF800108860DAF859
:10A0F0000010486002212020F7F776F90020F6F7DB
:10A100000CFE524C2068406C216840F400604864AA
:10A11000012002F0CCFB2068406C216820F4006034
:10A120004864F7F760F8DAF800000068DAF8001021
:10A1300040F00100086030BF3C4C01200026266240
:10A14000E061DFF8ECB0FFF780F8012844D0FAF7BF
:10A150008DFC484540D1FAF78CFC40453CD168461F
:10A16000F7F711FB002833D0206A401C20626846B4
:10A17000FFF795FCE0690025012806D10198F9F761
:10A18000E6FD206A032808BFE6610198B0B103F03C
:10A19000B6F80028C8BF01250FDC2088401C2080AD
:10A1A000DBF80000017F11F0010F07D0807F2188CC
:10A1B000814203D90198F9F7CAFD2680002128467B
:10A1C000FFF754FE0546F7F709FBFAF79FFC01E09D
:10A1D000FAF77BFC002DB6D0DAF800000068DAF858
:10A1E000001020F0010008600020F7F76FF8F6F784
:10A1F00053FAFAF73BFC052805D0FAF737FC074677
:10A200000520FAF742FCFAF780FD052F1CBF3846FF
:10A21000FAF73BFCFBF7A9FE0D4801780D480078E2
:10A22000F7F7E2F807B0BDE8F08F0000580600200D
:10A23000E806002031060020E4861100D0861100D7
:10A240000487110034060020EC861100E886110016
:10A25000BF050020BE0500202DE9F04F87B0F6F7BE
:10A26000BFFEF9F765F85C4D0124A86910B9F7F74E
:10A27000E6FDAC61DFF864A1DAF80000B0F90E1178
:10A28000B0F90C0100F002FA04F089FB6C61FAF7F6
:10A29000EDFB052804BF4FF0000B514F26D1DAF833
:10A2A00000006A68C2F30361D0F8F8008B00D84060
:10A2B00000F00F00C5F808B0C5F80CB0002970D048
:10A2C000022918D004296DD00A2922F07F404FEAD4
:10A2D000017118BF41F0007108436860FEF7B5FFD7
:10A2E000012803D0FAF7C2FB0528D8D007B0BDE893
:10A2F000F04F04F056BB064600244FF00508FAF76D
:10A30000B8FB81460F213046FAF77CFC0028E5D0E7
:10A3100000F0FBFB396870208860396802204860D3
:10A32000304E3068406C316840F400604864012071
:10A3300002F0BDFA3068406C316820F40060486477
:10A34000F6F751FF38680068396840F0010008608E
:10A3500030BFFEF77AFF012806D06868C0F30360BB
:10A36000484508BF002C1ED000F0CFFBFAF77EFB5B
:10A37000052805D0FAF77AFB80460520FAF785FB19
:10A38000FAF7C3FCB8F1050F1CBF4046FAF77DFB96
:10A3900038680068396820F001000860FBF7AEFDFE
:10A3A0009CE713E015E06846F7F7EDF958B1684609
:10A3B000FFF775FB6846FFF7DAFD0446F7F70EFA7C
:10A3C000FAF7A4FBC5E7FAF780FBC2E7FFF76DFEDB
:10A3D00084E702F043FF81E758060020E8060020EA
:10A3E000EC861100E8861100F0B4FF4EDDE905C4EB
:10A3F0003668049DB66916F0010F04D01F464B1B4A
:10A40000CD1BDBB2EDB216F0020F06D06746A2EB11
:10A41000040CD21B0CF0FF0CD4B216F0040F08D0C1
:10A4200080F800C04A1B84704270C91AC170F0BC29
:10A4300070470370857080F801C0C470F0BC70472D
:10A440002DE9F043164601FB06F90D46014685B09D
:10A450001F464A46E5480CF0A1FDE44C02F00FFC13
:10A460004FF0000818B104F030F801281AD002F0BB
:10A4700006FC18B104F029F8082842D0B7F5805F2F
:10A480001CBF0020B9F1000FDCBF05B0BDE8F083B0
:10A490002156794309132154401C8145F8DC05B04D
:10A4A000BDE8F08300210B46002ECEBFDFF838C395
:10A4B00005B0BDE8F0830020002D1CDDDCF8002095
:10A4C00092F83E919945DCBF92F83F914B450CDCE8
:10A4D00092F83C918145DCBF92F83D21904204DC2A
:10A4E00062567A431213625401E004F80180401C62
:10A4F000491CA842E2DB5B1CB342DCDB05B0BDE8D3
:10A50000F083AE428CBF701E681EC2B2B54234BF2B
:10A51000681E701EC1B20420CDE90002002303A80A
:10A520000292FFF761FF00210A46002EDCBF05B052
:10A53000BDE8F0830020002D19DD9DF80D30934219
:10A54000DCBF9DF80F309A4209DC9DF80C30834245
:10A55000DEBF9DF80E30984204F8018003DD63569B
:10A560007B431B136354401C491CA842E5DB521C6F
:10A57000B242DFDB05B0BDE8F0832DE9F0411C46B7
:10A5800015460E460746F8F745FC21462846F8F7DB
:10A5900060FC0623954A31463846F8F770FDBDE861
:10A5A000F041F8F738BC924A5060916070472DE94D
:10A5B000F00F0024DDE90875B7F5805F08BF642D52
:10A5C0002AD00026002B87BFA5F16409C5F16408D5
:10A5D000BDE8F00F70470020002A17D9B0FBF2FA4F
:10A5E00031F914C0642D0CFB07FC4FEA2C3C27BF4B
:10A5F0000AFB09FA0CFB0ACC0AFB08FA0CFB1ACC82
:10A6000021F814C0401C641C9042E7D3761C9E4283
:10A61000E1D3BDE8F00F7047884204BFBDE8F00FFA
:10A6200070475A43BDE8F00F52000CF0B7BC2DE95B
:10A63000F04180466C4882B00F4600681D461646C1
:10A6400090F84C10ADF8001090F84D10ADF80210D5
:10A65000B0F84A10ADF80410B0F848000024ADF886
:10A660000600F8F7D7FB6846F8F7C8FC29463046DD
:10A67000F8F7E6FB39464046F8F7D2FCF8F7CBFB93
:10A680005B48C46002B02046BDE8F08158490880AC
:10A6900070472DE9F041574E8AB005465448CDE940
:10A6A0000056A6F148080C46CDF80880B0F9001015
:10A6B00003913F29C8BF3F2005DC11F1400FB8BF0F
:10A6C0006FF03F0000DA039000200490F8F7A2FB3F
:10A6D00049484A4F01783878F8F7B2FB6846F8F7EE
:10A6E00046FC0890F8F797FBC4E90068BDF8140031
:10A6F0002081BDF816006081BDF81800A081BDF86A
:10A700001A00E081BDF81C002082BDF81E006082A6
:10A71000BDF81C00BDF81E103A7801FB020035F9A7
:10A7200010000AB0BDE8F081314800697047304838
:10A73000406970472DE9FF4FADF2A44D00208A46D5
:10A74000CDF89C04ADF88C048346471E9146DDF895
:10A75000E0844FF4906102A80CF0C1FCB8F1000F46
:10A7600018BF98F800B02548254E0578224804788F
:10A770001D480068008ECDF8940406F59060CDF871
:10A780009804DDF8A404CDF89004FAF76FF90228D4
:10A790001ED1FAF76EF902281AD1F9F7E0F9019003
:10A7A000B0B1DDF8A4242B46009410460199F9F7C6
:10A7B000B1F914480078022804BF0198FFF706F8A1
:10A7C00010480078092804BFDDF8A404FEF7FEFF56
:10A7D000DDF89004CDF8880405480661F9F7B3FA6E
:10A7E000CDE900402B460FE0E80600201451002080
:10A7F0007C0600209C530020BF050020BE050020E1
:10A800001C54002031060020024602A8DDF88814FE
:10A81000F9F780F9BE480078032804BF0198FEF7D5
:10A82000D5FFBB480078052804BF02A8FEF7CEFF7D
:10A83000B7480078062804BF02A8FEF7C7FF02A8A1
:10A84000CDF88804B2480078222803D1002102A85C
:10A85000FFF7FCF8DDF8940410F0010F15D0DDF8D7
:10A8600088040090F8F7D6FA21462846F8F7F1FA5E
:10A870000623A84A30460099F8F701FCF8F7CBFA0E
:10A88000A3480078082810D012E064214FF48050CB
:10A89000CDE9000123462A463046DDF88814FFF74B
:10A8A00086FE9B480078082802D13046FEF78EFFCE
:10A8B000DDF8940410F0060F31D002F0ADF870BB53
:10A8C0000020CDF894049448006890F84C10ADF83E
:10A8D000001090F84D10ADF80210B0F84A10ADF825
:10A8E0000410B0F84800ADF80600F8F793FA68468F
:10A8F000F8F784FB21462846F8F7A2FA31460846C5
:10A90000F8F78EFBF8F787FA8449DDF89404C860FD
:10A910007F4800780A2804BF3046FEF757FFBAF197
:10A92000000F23D0B9F1000F29D0DDF89C0400906E
:10A930000DF28C433046DDF88824DDF89814F9F7E1
:10A9400071FD0746BDF88C04072807D1680000FB9D
:10A9500004F23046DDF888140CF020FBB7F1FF3F1D
:10A9600012BF002F0020ADF88C0402E0B9F1000FF7
:10A9700005D049463046FFF78CFEA9F8140064481C
:10A980000078072804BF3046FEF720FFBAF1000F19
:10A9900018BFCAF80070DDF8D80400281CBFBDF845
:10A9A0008C140180B8F1000F18BF88F800B0DDF8F2
:10A9B00090040DF2B44DBDE8F08F594870472DE971
:10A9C000F05F81465748174688460078544C460049
:10A9D000F9F7C1FADFF838B1824600259BF800008C
:10A9E000042804BF4846FEF7DCFE9BF8000005285B
:10A9F00004BF4846FEF7D5FE9BF80000032804BFBD
:10AA00005046FEF7CEFE9BF80000232804BF4846C0
:10AA1000FEF7C7FE0020002E09D939F810103AF8C9
:10AA20001020891A24F81010401C8642F5D89BF893
:10AA30000000062804BF2046FEF7B3FE9BF8000086
:10AA4000222804BF2046FEF7ACFE0020711E18BF6E
:10AA50000A4612D004EB400134F810304988C91A74
:10AA600009B224F810100029B8BF494209B2A9421E
:10AA7000C8BF0D46401C9042ECD304EB460020F8C2
:10AA8000025C9BF800000A2804BF2046FEF789FEFE
:10AA90009BF80000082804BF2046FEF782FE9BF8C2
:10AAA0000000072804BF2046FEF77BFE9BF800004D
:10AAB000012804BF2046FEF774FE9BF800000E2814
:10AAC00004BF2046FEF76DFE9BF80000212804BF5E
:10AAD0002046FEF766FEB8F1000F10D00E494FF089
:10AAE000FF300968B1F97220AA42B8BF012004DB27
:10AAF000B1F970108D42B8BF0020C8F80000002FD7
:10AB000018BF3D804846BDE8F09F70477047000081
:10AB10003106002014510020E80600207C060020A9
:10AB20001C5D0020C505002008283CBF9C4908701A
:10AB3000704700209A49C8609A48006890F88100E0
:10AB4000082838BF0870704795480078704710B5DE
:10AB50000446F6F745FA944A03211268D161052CA0
:10AB60004ED2DFE804F0031221303F0001217F20A4
:10AB7000F5F76AFC8C214FF48470F5F765FC5C21D5
:10AB80004FF48570F5F760FC3AE001217F20F5F77E
:10AB90005BFC87214FF48470F5F756FC59214FF484
:10ABA0008570F5F751FC2BE001217F20F5F74CFC77
:10ABB00075214FF48470F5F747FC4D214FF48570F3
:10ABC000F5F742FC1CE001217F20F5F73DFC6721F1
:10ABD0004FF48470F5F738FC43214FF48570F5F796
:10ABE00033FC0DE001217F20F5F72EFC58214FF4B6
:10ABF0008470F5F729FC3A214FF48570F5F724FCB1
:10AC0000F9F76CF8F6F7EFFA012010BD0120704754
:10AC1000644863490068B0F876004242C8688242DE
:10AC2000BCBF401EC86070472DE9F04FA1B09346ED
:10AC3000884604464FF0000901F0AFFF594E8246A6
:10AC4000574D3068B0F96E00A0420DDAA868401E7A
:10AC5000A86009D26420A860686803280CBF00209F
:10AC6000401C6860FFF773FF504F3878072829D1E0
:10AC70004F4859460078820068460CF08FF9ADF8CD
:10AC80000040ADF80280ADF804A0A889ADF8060038
:10AC9000A888ADF808003068B0F87210ADF80A1056
:10ACA000B0F87410ADF80C10B0F86E10ADF80E10CE
:10ACB000B0F87600ADF810003878072804BF684671
:10ACC000FEF76FFD484621B0BDE8F08F344880782C
:10ACD000002818BF012070470020DFF8C4C09CF88E
:10ACE0000210002914BF012200229CF80110002943
:10ACF00018BF01218A4208BF70470A1C18BF0122F1
:10AD000010B48CF80220274A1368D3F8A42012F05C
:10AD1000040F0FD021B1C2F30310082809D206E0B6
:10AD20000020CCF80C0093F88100082801D28CF8A0
:10AD30000000012012F0020F18BF012010BC704764
:10AD40002DE9F041174F00263868D0F8A40010F420
:10AD5000807F21D0124D69780C1C18BF0124C0F3EC
:10AD60000330012101FA00F0F7F7FDFF3968B1F86F
:10AD7000A41011F4007F01D028B103E0002818BF0F
:10AD8000002000D10120844206D0002818BF0120F5
:10AD90006870FFF7A1FF06463046BDE8F08100006D
:10ADA00094060020E8060020E88611003106002005
:10ADB000C50500207148006800F5407070476F4875
:10ADC000006800F58070704770B56C4C6C49226863
:10ADD0001068884204BF5068B0F5087F24D1D2F8CB
:10ADE00008C0BCF5405F1FD86649D06888420DD0C6
:10ADF000002311461846B3EB9C0F07D251F8045BB1
:10AE0000401C6B40B0EB9C0FF8D36BB902F580701F
:10AE100000F0E2F840B1206800F5407000F0EBF877
:10AE200000281CBF012070BD002070BD534910B523
:10AE30004FF48E100860FFF7C7FF002818BF0120ED
:10AE400010BD4FF48E10F7F741BA4C484C4A0068D9
:10AE50000168914206BF4168B1F5087F0020704744
:10AE60004648006800697047444909680A69824297
:10AE70009CBF00207047C0EBC00001EBC00000F594
:10AE8000806070473D4A126802EB80035B6A1A4497
:10AE90003D4B53F82000FF3020F0FF0000FB012065
:10AEA00070472DE9F0010022344D17462E1D8318FE
:10AEB00093F92840002CB8BF41F8227010DBD5F878
:10AEC00000C0D3B20CEB830856F82330D8F82480A6
:10AED000FF33C44423F0FF0303FB04C341F82230D3
:10AEE000521C102AE3D3BDE8F00170472DE9F04170
:10AEF0000025174604460029B8BFBDE8F081042CA0
:10AF000002D0052C10D014E0F9F7B0FD052810D1BF
:10AF1000FEF7A7FF022808BF03250AD0FEF7A1FF0E
:10AF2000002808BF022504E0F9F7A0FD052808BFA6
:10AF300001251248144E006856F8241000EB8400D6
:10AF4000FF31406A21F0FF0100F5E030503005FB91
:10AF50000105F9F78BFD022808D101F0F5FD28B9AC
:10AF600056F82400FF3020F0FF00054456F8242056
:10AF700039462846BDE8F041F7F79EBCA4060020FC
:10AF800054465053EFBEADDEA806002010B51F4C4E
:10AF9000FFF74CFFA0B1FFF70DFF0146AC221C48A4
:10AFA0000CF041F8FFF70BFF01464FF4C472206824
:10AFB0000CF039F82068406DBDE8104001F025BD67
:10AFC0004FF4C47120680CF08AF800210420F9F7CE
:10AFD0005FFDFEF720FFDBE758B10E4A01689142A2
:10AFE00007D1406820F00F00B0F5087F04BF0120B2
:10AFF00070470020704738B1006820F00F00B0F5AE
:10B00000907F04BF0120704700207047E8060020B1
:10B01000F80F002041505352002808BF7047401ECF
:10B0200000BF00BF00BF00BF00BF0028F7D17047BE
:10B0300070B5614D82B00024286804665F480168DD
:10B04000D1F82C13006841F00801C0F82C13F8F770
:10B050005BF928680069296840F001000861601EFA
:10B06000F8F7DEF8564880234FF48012002152F89A
:10B0700021C040F821C0491CB1EB930FF7D3F8F77A
:10B08000E1F8F8F77FFBF8F7A9FB0020F8F77BFB66
:10B090002320F8F76CFBF7F798FEF8F71FFBF8F79B
:10B0A00097F9F7F7B9FEF6F777FEF5F715FEF8F71B
:10B0B0005EF8F8F719F8434E009401940423002237
:10B0C00007213068F8F778FA3068F8F7F0FA0420CA
:10B0D000CDE900043C4C0346002207212068F8F724
:10B0E0006BFA2068F8F7E3FAF6F729FFF6F7F4FFB2
:10B0F000364800683649884218BFF6F7EDFFF8F782
:10B100005DFCFEF771F8FEF72EFD62B6FFF73EFF1D
:10B11000304803F0B6FA304C2068B0F90C0103F067
:10B120003CFCF8F7B1FCF9F781FE2068418A008AFF
:10B13000FEF72FFA2068806EC0F34E0161F35F00C6
:10B1400001F000F9FFF7E2FC00221146022001F0B5
:10B1500006F900226421072001F001F92968012085
:10B16000086602B0002070BD01F0F3FC0146022029
:10B17000F9F78EFCF9F77AFC06281AD2DFE800F01E
:10B1800019090313160602F06CFAF3E7FFF764F8E7
:10B19000F0E7FAF7D5FAF9F769FC012804BF0220B5
:10B1A000F9F773FCE6E701F0FCFAE3E7FEF733FE9C
:10B1B000E0E7F9F7B2FCDDE7E4861100E88611006C
:10B1C0000068002000871100FC861100F0150020A7
:10B1D00054464953F80F0020E8060020FE49087045
:10B1E00070474FF42C30704770B54FF42C3044F258
:10B1F00064422146F6F764FFF84A216820469142EE
:10B200001BD16168B1F5007F17D3D4F808C00023C3
:10B2100044F264418C4588BF44F2644C0022B2EB96
:10B220009C0F28BF70BD54F82250521C2B44B2EB27
:10B230009C0FF8D3002B08BF70BD002070BDE749FC
:10B2400001604FF40071416044F26441816000216B
:10B25000C16080F8201080F8211080F8221080F85A
:10B26000231040F2FF72C0E904218161C1610165D0
:10B2700000F580404FF6FF71A0F85414A0F8561462
:10B28000A0F85814A0F85A14A0F85C14A0F85E14A2
:10B29000A0F86014A0F862140120704770B5002176
:10B2A000C1600B46D0F808C044F2644104468C45A6
:10B2B00088BF44F2644C0022B2EB9C0F06D254F8D3
:10B2C0002250521C2B44B2EB9C0FF8D35942C16060
:10B2D0004FF42C3044F264422146F7F7EDFA01288E
:10B2E00018BF002070BD2DE9F04F05468FB00E4607
:10B2F0000020F6F773F80C90F9F716FD8046B84871
:10B30000DFF8E4B2032490F800A0B6480778DBF831
:10B310000000C46102217F20F5F796F840F2022078
:10B32000F5F7ABF8C0F30219012E7DD0002006908E
:10B33000AE480390AE480890AE480490AE48002650
:10B3400001960090DBF80000C46101217F20F5F731
:10B350007BF84FF48770F5F790F8C0B20D9002219A
:10B360007F20F5F771F840F20720F5F786F8C4B2B0
:10B370004FF40270F5F781F80CF066FF07909F48D4
:10B3800014F0100F50F8290002909D4850F8290041
:10B39000059018BF974E14F0200F04D03046049942
:10B3A0000CF000FE064614F0400F04D03046009921
:10B3B0000CF0F8FD0646E00904D0304600990CF088
:10B3C000F1FD064614F0010F1CBF8A48019014F0ED
:10B3D000020F04D0049901980CF0E4FD019014F0E0
:10B3E000040F04D0DDE900100CF0DCFD019014F036
:10B3F000080F04D0DDE900100CF0D4FD019016F127
:10B40000FF4F2CBF86F0004030467E4CA042D8BF94
:10B410002646314601980CF039FE01904FF0FF317D
:10B4200003980DF03AF900E018E0814608990CF015
:10B4300057FF8346594648460CF0B4FD0B905946D9
:10B4400048460DF055F80A900AFB07F04FF0000946
:10B45000049000281ED80FB0BDE8F08F00240AFB2E
:10B4600007F6002E8EBF684F0FB0BDE8F08FB5F91C
:10B4700000000CF0E9FE57F829100CF031FF0CF039
:10B48000C7FE25F8020B601C84B2A642EFD80FB0AD
:10B49000BDE8F08F002000900C98B0F900000990F2
:10B4A0000C98801C0C9018F801BB1BF0800F1CBF7F
:10B4B0004FF07E50069000242BFA04F010F0010F9C
:10B4C00013D00120A0400CF0BCFA504A504B0CF0B5
:10B4D0001FFB07468A4600980CF038FD3A46534653
:10B4E0000CF0C6F90CF092F90090601CC4B2072C65
:10B4F000E2D3059902980CF0FBFF0446DDE90A103F
:10B500000CF0F6FF089009980CF09EFE6FF00A010F
:10B510000DF0C3F84FF07E510CF0EAFF8346DDE9F1
:10B5200002100CF03FFD06990CF0DAFE07464FF0D2
:10B530007E5006990CF0DCFF8246059903980CF0CA
:10B5400031FD51460CF0CCFE39460CF0D1FF82465D
:10B550000D98401E0CF078FE074610F1FF4F28BFF3
:10B5600087F0004027498842D8BF264F4FF08041DE
:10B5700007980CF017FD0990394608980CF086FDE5
:10B5800009990CF0ADFE59460CF0AAFE03990CF097
:10B59000A4FF834614F1FF4F2CBF84F000402046E7
:10B5A00018498842D8BF0C4616F1FF4F2CBF86F0D1
:10B5B000004030468842D8BF0E46DDE901010CF05C
:10B5C0008FFE0CF0C3FCCDE90801314600980CF069
:10B5D0005DFD51461EE00000F006002053454C463C
:10B5E000BE050020BF050020E88611000000B04025
:10B5F000CDCC4C3FC3F5A04048E1DA40F08A1100C1
:10B60000108B11000AD7233C308B11009A9999991D
:10B610009999A93F0CF064FE0CF098FC07468A4605
:10B6200058460CF093FC4FF0FF320DF008F83A4604
:10B6300053460CF01DF9DDE908230CF019F9074613
:10B640008A4621464FF07E500CF020FD0CF07EFC27
:10B650003A4653460CF05CFA0022FE4B0CF08CFB91
:10B6600004460F4630460CF071FC22463B460CF077
:10B670004FFA0CF0CBF8F8490CF032FEF7490CF019
:10B6800091FC0CF0C5FD25F8020B09F101001FFA31
:10B6900080F9049848453FF6FDAE0FB0BDE8F08F45
:10B6A0002DE9F043ADF2844D0C4681464FF0000881
:10B6B0004FF4906168460BF012FDE94FF5F745FB3A
:10B6C0000020F5F735FB0020F5F727FBF5F719FB10
:10B6D0006846F8F732FCE3480578E3480678002E20
:10B6E00018BF002D47D02068002119F0030F80F803
:10B6F000205080F8216080F8221080F8231038D084
:10B70000F5F771FD0020F8F72EFC0120F5F7ABFAF4
:10B710002046F5F762FCFAF7B3FC24680020F5F741
:10B720005DFE0146754343F254006A0020440BF06D
:10B7300035FCF9F7F9FA014643F654002A4620444D
:10B740000BF02CFCC948807810F0010F11D0F6F7EF
:10B7500010FC002104F15400FFF7C5FD386890F893
:10B76000EB00012805D1C20204F15401C0480BF0DE
:10B7700015FC4FF00108F5F7BDFC0DF2844D404675
:10B78000BDE8F0832DE9F04FADF5117D0E4604467E
:10B7900017464FF4107168460BF0A1FCB3484FF008
:10B7A00000084FF0FF39807810F0020F43F2540088
:10B7B00007EB000504FB06F090904ED06946AC46BE
:10B7C000C246002E88BFA4F1010B2ED90020002C08
:10B7D00025D9584508BF81F800801CD03CF91020BD
:10B7E000002AD8BF81F8009015DD0CEB4003B3F9B7
:10B7F0000230934207DCD31A4FF0640E03FB0EF3C2
:10B8000093FBF2F206E09A1A4FF0640E02FB0EF27E
:10B8100092FBF3F20A70401C491CA042D9D30AF1F2
:10B82000010A0CEB440CB245D0D342F65400384424
:10B8300069468246909A0BF0F6FB8948006890F8BA
:10B84000EB00012804D1C202514689480BF0A6FB47
:10B850004FF4107168460BF042FC8448807810F079
:10B86000040F04BF0DF5117DBDE8F08F68464FF061
:10B87000000A002C88BF06FB04FB36D900221146C3
:10B88000BBF1000F05D829E0112A08BF80F800801D
:10B890001FD00AEB010C35F91C30002BD8BF80F803
:10B8A000009016DDA44435F91CC09C4508DCA3EBD0
:10B8B0000C0C4FF0640E0CFB0EFC9CFBF3F307E04A
:10B8C000ACEB03034FF0640E03FB0EF393FBFCF3AE
:10B8D00003702144521C20448B45D5D804FB16002C
:10B8E000401C0AF1010A5445C8D842F65440384475
:10B8F00069460446909A0BF096FB5948006890F808
:10B90000EB00012804D1C202214659480BF046FB46
:10B910000DF5117DBDE8F08F2DE9F041504D064643
:10B92000144628680F4690F8E8205248028000F03C
:10B93000EAFD002306FB07F1002984BFDFF838C1C8
:10B940004E4A12D9DCF8000041F6540730F8136073
:10B9500004EB43003E52166800F5005036F81360C1
:10B960005B1CA0F854609942ECD8286890F8EB0072
:10B9700001280ED1C20241F6540021183C480BF0B8
:10B980000DFB42F2540021184FF400623C480BF0CA
:10B9900005FB364901204860BDE8F08130B5054619
:10B9A00091B000240120F5F75EF92046FFF75CFA1C
:10B9B0006946FFF776FA00990798F4F7F7FF3149DF
:10B9C00001200968C1F814032846FAF74FF9FF204F
:10B9D000F9F7B1FBF5F7B9F90020F5F7A9F900205F
:10B9E000F5F79BF9F5F78DF90020F8F7F5F9002048
:10B9F000FAF705FC0120F8F7B6FA11B030BDF0B542
:10BA0000ADF2C44D0D460646144600274FF4906132
:10BA100068460BF064FB2020F9F78DFB0120F5F759
:10BA200022F93846FFF720FA070008BFF9F758F85F
:10BA30000DF590613846FFF734FADDF88014DDF833
:10BA40009C04F4F7B3FF0F4901200968C1F81403FF
:10BA50001AE000000000F03F00007A440080CE436E
:10BA6000E8060020BE050020BF050020F0060020EB
:10BA7000006D0020040700200C07002008070020AC
:10BA800000750020E8861100FAF7F0F8F5F75DF987
:10BA90000020F5F74DF90020F5F73FF9F5F731F9FA
:10BAA0000120F8F760FA6846F8F747FA0020FAF73D
:10BAB000A6FB0020F5F792FC06FB05F14A000146C3
:10BAC00041F25400204404460BF068FAFE48006836
:10BAD00090F8EB0001281CBF0DF2C44DF0BD4FF4EF
:10BAE00000622146F9480BF059FA0DF2C44DF0BD41
:10BAF00070B515460E460446F8F725F904FB06F125
:10BB00004C0021460BF0C9FA0220FFF747FFFAF775
:10BB1000F5F90320FFF742FFFAF7FDF9F8F713F9FB
:10BB20000146224605F654000BF038FAE648006854
:10BB300090F8EB00012805D1C20205F65401E34854
:10BB40000BF02CFAF8F7FFF82146BDE870400BF037
:10BB5000A4BA2DE9F14FADF5065D4FF00109C846D5
:10BB60004FF410610DF6D8500BF0B9FA14204FF0D5
:10BB7000000A14901390129011905446CDF840A0F2
:10BB80000120F5F770F82046FFF76EF96946FFF7D8
:10BB900088F900990798F4F709FFDFF834B301201A
:10BBA000DBF80010C1F81403122720247D010020C7
:10BBB000F5F7B3F8F5F712FEDBF800100320C861C3
:10BBC00001217F20F4F740FC11210E20F4F73CFC0A
:10BBD0005A210820F4F738FC36210A20F4F734FC07
:10BBE00002217620F4F730FC02217F20F4F72CFCB0
:10BBF0006A210220F4F728FC8E210420F4F724FCAB
:10BC0000F1210720F4F720FC07210820F4F71CFCA1
:10BC100000211620F4F718FC03217F20F4F714FC10
:10BC200089210520F4F710FC67210620F4F70CFCAD
:10BC300045210720F4F708FC23210820F4F704FC31
:10BC4000F1210920F4F700FC68004FEA570B04FBD0
:10BC500007F6009002E0B8F1000F50D00120F5F790
:10BC600002F8F5F785FC0020F9F765FAF5F7BBFA5D
:10BC70000120F4F7F8FFF5F77BFC1198F9F75BFA70
:10BC8000F5F7B1FAB9F1000F34D042F26010684410
:10BC9000F5F779FD58B30020F5F73FF8F5F79EFD6D
:10BCA000B8F1000F26D00AF101001FFA80FABAF1AC
:10BCB000010F4FF000000BD0F5F790FB014641F665
:10BCC00058306844009A0BF069F94FF0000811E011
:10BCD000F5F784FB014641F2D8606844009A0BF006
:10BCE0005DF914991198084480B2119002E0B9F1FD
:10BCF000000FCAD14FF00109B8F1000FAED10020FA
:10BD0000002D18D941F2D8636B4403F590620DF50C
:10BD10009B6C32F9101033F91080A1EB08014FF041
:10BD2000640801FB08F101EBD17149104CF82010B7
:10BD3000401CA842EDD34FF000084346002C25D903
:10BD400041F6D87A0DF59B69EA4409F5DC5E0021DD
:10BD50000A464046B8EB560F0BD259F820C0624451
:10BD600000EB560C204459F82CC0B0EB560F614440
:10BD7000F3D3B2FBFBF04AF82300B1FBFBF04EF823
:10BD800023005B1C08F10108A342E0D30020002D32
:10BD90001FD941F6D8730DF59B626B4402F5DC5C4C
:10BDA0000DF15808B0FBF4F104FB1101B0EB550F95
:10BDB00034BF53F821105CF8211052F82090A1EB09
:10BDC00009010029B8BF494228F81010401CA842B8
:10BDD000E8D34FF00008002F82BF42F22019E94457
:10BDE000A9F1480A23D916A800EB88114022484639
:10BDF0000BF0D4F80020002F15D90021002C09D910
:10BE000039F811305AF82020491C1A444AF82020E9
:10BE10008C42F5D85AF8201091FBF4F14AF8201022
:10BE2000401CB842E9D308F10108B845DBD3002033
:10BE3000002D82BF42F2D808E8440DF1580C0CD90D
:10BE400041093CF8103058F82120D11A48BF991AFE
:10BE50002CF81010401CA842F2D30020002D84BF03
:10BE600016AA0DF6D85109D951F8203032F810C071
:10BE7000634441F82030401C8542F5D8109813994E
:10BE8000401CC0B210901298119010984FF0010809
:10BE90004FF0000AC14681423FF6DDAE0024002D7E
:10BEA00021D9DFF8308016AE0DF6D857109857F824
:10BEB0002410B1FBF0F00BF0DBFD4FF0663243468F
:10BEC0000BF026FE08E00000E8060020006D0020D0
:10BED000E88611006666E63F0BF086FD26F8140042
:10BEE000641CAC42E2D30DF5005316A9D3F88001CF
:10BEF00043F654431844009A04460BF094F8FE4865
:10BF0000006890F8EB0001281EBF61B00DF5005DE0
:10BF1000BDE8F08F4FF400622146F8480BF03EF880
:10BF200061B00DF5005DBDE8F08F2DE9F05FADF576
:10BF3000924D44F270476F444FF4906138460BF0D5
:10BF4000CEF803ADFF2244F2644128460BF09DF881
:10BF5000DFF8AC834FF0FF300290D8F804000DF109
:10BF6000080A4FF0FF0928B9FF224FF40061E548A5
:10BF70000BF08BF828460295FFF761F9DE4E346826
:10BF800094F8EA00A8F80200B4F9D8000CF05CF9C3
:10BF9000019094F8EB00032804D1012088F80000F8
:10BFA000A8F802900120F4F75EFE514698F80000D0
:10BFB000FFF776FB3846F7F7C0FF9DF82C409DF859
:10BFC0002D70002C12BF002F0DF5924DBDE8F09F93
:10BFD0004FF0000B2A4639462046CDF81CB0FFF73B
:10BFE000D1FB98F8020010F0080F04D02A46394619
:10BFF0002046FFF791FC98F8000010F0010F39D0AF
:10C0000098F8020010F0200F04D02A463946204646
:10C01000FFF7F5FC98F8020010F0400F2AD0F7F770
:10C0200092FE04FB07F14FEA410949460BF035F84F
:10C030000220FFF7B3FCF9F761FF0320FFF7AEFC26
:10C04000F9F769FFF7F77FFE01464A4605F6540007
:10C050000AF0A4FF306890F8EB00012805D1C20275
:10C0600005F65401A5480AF099FFF7F76CFE49461A
:10C070000BF013F898F8020010F0800F1CBF284650
:10C08000FFF767FD98F8000010F0400F40F02581A1
:10C090000898401C08900798002814BF0A9809982F
:10C0A00000F1010014BF0A90099004FB07F0441E40
:10C0B00058BFDFF854A27CD498F8020010F0010FAA
:10C0C0002FD0924901980BF0E1FF4FF07E51009084
:10C0D0000CF003FA51460CF003F905EB44078146D6
:10C0E000B7F954000CF0B0F849460CF0C5F810D37D
:10C0F0004FF07E5100980BF055FF51460CF0F0F8D0
:10C100008146B7F954000CF09FF849460CF0B4F999
:10C1100007D217980DF5804140F001001790A1F863
:10C120006844B8F8020010F0020F15D029193268DF
:10C1300001F5005191F95418B2F9C8308B4203DC73
:10C14000B2F9CA208A4207DA17990DF5804241F008
:10C1500002011791A2F8604410F0040F15D02919BC
:10C16000326801F5005191F9541CB2F9CC308B4280
:10C1700003DCB2F9CE208A4207DA17990DF5804226
:10C1800041F004011791A2F8624410F0080F18D092
:10C1900005EB4401326801F58051B1F95418B2F948
:10C1A000D0308B4203DCB2F9D2208A4209DA1799E7
:10C1B00000E06EE041F008010DF580421791A2F811
:10C1C000644410F0100F16D005EB4401326801F5FD
:10C1D0000051B1F95410B2F9D4308B4203DCB2F9FA
:10C1E000D6208A4207DA17990DF5804241F01001F6
:10C1F0001791A2F8664410F0200F16D005EB440109
:10C20000326801F58051B1F95410B2F9DC308B423B
:10C2100003DCB2F9DE208A4207DA17990DF5804275
:10C2200041F020011791A2F86A4410F0400F14D099
:10C23000326805EB4401B1F95418B2F9E0308B4291
:10C2400003DCB2F9E2208A4207DA17990DF5804241
:10C2500041F040011791A2F86C4410F0800F15D006
:10C2600005EB440043F65441415E3068B0F9E420E8
:10C270008A4203DCB0F9E600884207DA17980DF528
:10C28000804140F080001790A1F86E44641E7FF555
:10C2900013AF306890F8EB00F8B90598002144F22C
:10C2A00064422B46CDF818B0904294BF024644F247
:10C2B00064420020B0EB920F06D255F820C0401C1B
:10C2C0006144B0EB920FF8D34842D8604FF42C3061
:10C2D00044F264422946F6F7EFFA306890F8EB0032
:10C2E000032802D10549179808801D208DF8000009
:10C2F00041208DF801000BE0E8060020006D0020D1
:10C30000F00600200075002000803B450000C84278
:10C310009DF85C008DF802009DF85D008DF803002B
:10C320009DF85E008DF804009DF85F008DF8050013
:10C3300006226946072000F03BF80DF5924DBDE856
:10C34000F09F00005149C2B2C0F307200A80488024
:10C3500070474E484188008861F31F20704710B530
:10C360004A4C012303FA00FC248882B01CEA040F23
:10C3700004BF02B010BD00F00F0043EA80008DF84A
:10C3800000008DF801108DF80220100A8DF80300CE
:10C39000100C8DF80400100E8DF8050000208DF8AB
:10C3A00006008DF807006846FDF73EFC02B010BDA0
:10C3B000012303FA00F000B5344B83B01B88184208
:10C3C00004BF03B000BD072A88BF072200206B46C8
:10C3D000002A08D911F800C003F800C0401C9042A0
:10C3E000F8D3082804D200211954401C0828FBD394
:10C3F0001846FDF719FC03B000BDDFF890C001231B
:10C400008340BCF802C013EA0C0F08BF704710B598
:10C4100082B000F03F0040F080008DF80000072A55
:10C4200088BF072200206B46002A09D911F800C0F6
:10C430001C18401C84F801C09042F7D3072805D28D
:10C4400000211A18401C51700728FAD31846FDF72E
:10C45000EBFB02B010BD10B40C4C40EA01230228E3
:10C46000A288944602D0052805D009E0002918BF0B
:10C47000022905D103E0002918BF022900D11A467C
:10C48000944518BFA28010BC70470000F806002039
:10C49000F74908707047F64800B5C07848F6B8010B
:10C4A00083B0484301218DF8011000214A1E8DF808
:10C4B00007108DF80010ADF804208DF80810ADF8C5
:10C4C00002208DF806108DF80910F7F710F9FCF727
:10C4D000BCFE01280DD00120F6F710FCF7F71EF97D
:10C4E0000028F4D06846FDF73AFC0020F7F713F96E
:10C4F000EDE7F7F70BF903B000BDDD494870704771
:10C50000DB48407870472DE9F04FADF2F44D4FF421
:10C51000906104A80AF0E3FDDFF8548302210020B3
:10C5200088F80110FEF7A0FC040008BFF8F7D8FA5D
:10C53000F4F756FD0DF592612046FEF7B2FCDDF8EA
:10C540009014DDF8AC04F4F731FACA490120096807
:10C55000C1F81403F4F7F9FB0020F4F7E9FB00201D
:10C56000F4F7DBFBF4F7CDFB04A8F7F7E6FCF4F7F0
:10C57000C9FDCDF8EC0498F8020010F0100F18BFB8
:10C58000F5F75CFABC4890F80090BC480778BC48C6
:10C59000002F0578BB48067818BFB9F1000F0ED000
:10C5A000FEF7B3FA0020F7F717FC98F8020010F036
:10C5B000100F0AD00120F7F7D6FC012009E0002E69
:10C5C00018BF002DECD100F0E6B80020F7F7CBFC47
:10C5D0000020F7F7C8FC0120F4F783FAF4F703FE14
:10C5E0001E20FDF706F800210846FCF7B9FFC8F841
:10C5F000080001210020FCF7B3FFC8F80C00002060
:10C6000009FB07F4DFF880A2002C88BF47F6FF7112
:10C610000AD9D8F8082022F810A0D8F80C2022F85F
:10C620001010401C8442F4D81E20FDF701FA0021AE
:10C630000120FCF795FF834601210846FCF790FF97
:10C6400001460020AB1918BF47F6FF7206D02BF841
:10C6500010A021F81020401C8342F8D8B8F804003C
:10C660000026864238BF4FF0000B6FD2FCF7EDFD7D
:10C6700001286BD00DF59A60F5F785F800285FD09A
:10C68000DDF8D404002857D098F8020010F0100FFD
:10C690000BD0DDF8D454F7F756FB2A4601464B463B
:10C6A00010460097F7F736FA22E00023CDF800B0E5
:10C6B000CDF804B0CDF808B0CDF80CB01A46194644
:10C6C000DDF8D404FEF736F8054698F8020010F0BD
:10C6D000200F03D0FEF728F8054608E0F7F733FBF4
:10C6E0002A4601464B4610460097F7F713FA1DB34A
:10C6F0000021002C88BF53461ED935F91100B0F532
:10C70000004FA8BF47F6FF7003DA10F5004FB8BF1F
:10C710001846D8F8082032F911C08445B8BF22F86D
:10C720001100D8F80C2032F911C08445C8BF22F896
:10C730001100491C8C42E0D8F5F750F8761C01E056
:10C74000F8F7CEF9B8F8040086428FD30120F4F749
:10C750008AFAFEF7DAF9B8F80400B0421BD8DDF81F
:10C76000EC0410F0020F16D000234FF6FF721846AB
:10C77000002C88BFD8E902C50DD93CF9101035F955
:10C780001060891B9942C8BF0B469142B8BF0A4648
:10C79000401C8442F1D8F4F7ADFC0DF2F44DBDE835
:10C7A000F08F2DE9F041324D002484B06C70374F8A
:10C7B0004FF00108661EFCF748FD012806D1F8F786
:10C7C00055F903281CBF04B0BDE8F081287810F0AB
:10C7D000010F05D0FFF7A9FB3C702C70FCF731FD71
:10C7E000287810F0020F07D0FFF78DFE287820F090
:10C7F00002002870FCF725FD287810F0040F2FD0D8
:10C80000E8788DF801808DF8074048F6B8018DF87A
:10C810000040ADF804608DF808404843ADF8026070
:10C820008DF806408DF80940F6F761FFFCF70DFD25
:10C8300001280DD00120F6F761FAF6F76FFF002806
:10C84000F4D06846FDF78BFA0020F6F764FFEDE7B9
:10C85000F6F75CFF287820F002002870FCF7F1FC66
:10C86000F8F704F90328A6D004B0BDE8F081000071
:10C8700000070020E8861100BE050020BF0500204B
:10C88000C3050020C40500200080FFFF160700201C
:10C8900003490968A1F8E80070470249C870704769
:10C8A000E806002000070020F748C0797047002202
:10C8B0000028D8BF7047002100BF491C0829FBDBB6
:10C8C000521C8242F7DB70472DE9F04F002283B003
:10C8D000EE490092019291F804904F8AB1F81080CD
:10C8E0004E79B7FBF9FEB8FBF6FBB1F90E50944652
:10C8F0001446B9F1000F18DD0021002E11DD01EB07
:10C90000421330F91330AB4207DD0CEB441A30F917
:10C910001AA05345C4BF14468C46491C09B28E4226
:10C92000EDDC511C0AB29145E6DC5CEA04004FF0F4
:10C93000010355D0611CD54A0CF1010000FB0BF03E
:10C94000948A00B201FB0EF1D58A09B204FB00FC07
:10C950009CFBF8F005FB01F292FBF7F100B209B283
:10C960008045DCBFA8F1010000B2B942A4BF791E26
:10C9700009B2C74A1268926912F0040F14BF23EA81
:10C98000020C02F0010CBCF1000F02D0691A491E22
:10C9900009B212F0020F02D0201A401E00B212F0AB
:10C9A000040F12BF0A460246084641218DF80010C6
:10C9B0008DF8013011098DF8021001098DF803106E
:10C9C00002F00F0161F31F108DF804000A208DF8AA
:10C9D00005006846FDF728F903B00120BDE8F08F97
:10C9E00043208DF8000000208DF801308DF8020002
:10C9F0008DF804008DF803008DF805006846FDF7FA
:10CA000013F903B00020BDE8F08F9F4982B26FF3A5
:10CA10000F00C1E9040270479B48407870479A4A6A
:10CA20000028516914BF41F0020021F0020050615A
:10CA3000704710B55A20F5F718FA80220021B62069
:10CA4000F5F75FF900220121B620F5F75AF9BDE8A4
:10CA50001040A520F5F709BA10B55A20F5F705FAE8
:10CA600011220021B620F5F74CF906220121B6204B
:10CA7000F5F747F9BDE81040A520F5F7F6B9854868
:10CA800010B50068C068804910F0040F087A16D00D
:10CA9000022808BF10BD022008725A20F5F7E5F9F8
:10CAA00080220021B620F5F72CF900220121B620C2
:10CAB000F5F727F9BDE81040A520F5F7D6B902280B
:10CAC00018BF10BD012008725A20F5F7CEF91122C7
:10CAD0000021B620F5F715F906220121B620F5F759
:10CAE00010F9BDE81040A520F5F7BFB96648007DF4
:10CAF000C0F340007047644AF02303EA0010516914
:10CB000021F0F0010843506170475F48007DC0F399
:10CB1000031070475C4A0028516914BF41F00100BE
:10CB200021F00100506170475748007D00F001007E
:10CB30007047554B19690A0E120721F07F4142EAEE
:10CB400000600843186170474F480069C0F30360F4
:10CB500070474F480068406DC0F303607047012183
:10CB600001FA00F04FF47F0101EA004146480269F2
:10CB7000114301617047012101FA00F04FF47F0178
:10CB800001EA00414048026922EA0101016170475F
:10CB90003D480069C0F3074070473B48008AC0F336
:10CBA00003307047384A4FF4704C0CEA003011697A
:10CBB000C1F3033321F470410843106118467047F4
:10CBC0003148808AC0F38020704770B52E4E0446ED
:10CBD000C0F380007569C5F30021884218BFF7F7DC
:10CBE000ADF814F0040F14BF45F4807025F4807084
:10CBF00014F0080F14BF40F4007020F4007014F01B
:10CC0000200F14BF40F4806020F4806014F0100FF7
:10CC100014BF40F4006020F4006014F0800F14BFD3
:10CC200040F0800020F080007061BDE87040FEF7A9
:10CC300053B815484169002011F0400F18BF01207A
:10CC400011F4807F18BF40F0040011F4007F18BF7A
:10CC500040F0080011F4806F18BF40F0200011F47C
:10CC6000006F18BF40F0100011F0800F18BF40F0A7
:10CC7000800070470448007DC0F3401070470248B0
:10CC8000808AC0F30020704710070020F80F0020B2
:10CC9000E8060020E4861100F848808AC0F30030DE
:10CCA0007047F6484069C0F3003129B1C0F3401025
:10CCB000002804BF0120704700207047EF498A69AF
:10CCC0001043886170472DE9F047EC4F0D46396AF3
:10CCD000491C39624FF000080028C8BFC7F82480FB
:10CCE00015D0002DC8BFC7F8288014D0397D11F0A9
:10CCF000010F7DD03969DFF88893C1F303642646BC
:10CD0000062C56D2DFE804F00B2A3A556464796A9F
:10CD1000491C7962E5E7B96A491CB962E6E700286F
:10CD200005DD022000F05AFE08B1022444E0002D87
:10CD300005DD012000F052FE08B101243CE0D9F8E5
:10CD40000000396A90F8290000EB8000884231D851
:10CD500002240120C7F82080F8622DE0002804DDBD
:10CD6000022000F03BFE0028DFD11DBBD9F80000F7
:10CD7000B96AB0F85E0088421CD216E0002818BFDD
:10CD8000C7F82C8016D1012000F028FE0028D4D14D
:10CD9000D9F80000796AB0F85C00884205D3F86AD7
:10CDA000012808BFC7F82C8004D1002000F016FE2F
:10CDB00000B10024B44235D03869010E090720F0D3
:10CDC0007F4041EA0461084338610120BDE8F087F3
:10CDD000002806DD022000F001FE002818BF022412
:10CDE000E8D1002D08DD012000F0F8FD002800E06A
:10CDF00018E018BF0124DDD1042E0DD17869C0F3ED
:10CE0000003149B1C0F3401030B9052000F0E6FD13
:10CE1000002818BF0524CFD1002000F0DFFD002836
:10CE2000C8D0C6E70020BDE8F0872DE9F04188466C
:10CE30000446F5F784F8F4F7D3F8924A0321126810
:10CE4000D1611F26904D4A271CB1012C12D0022C13
:10CE500026D001217F20F3F7F7FA1F210E20F3F7E8
:10CE6000F3FA4A210820F3F7EFFA85F8EE6685F821
:10CE7000E87615E001217F20F3F7E6FA15210E2070
:10CE8000F3F7E2FA75210820F3F7DEFA152085F8AA
:10CE9000EE067520794985F8E80601208870C8708B
:10CEA000B8F1010F04BF0020F7F75DF8F4F79BF924
:10CEB000BDE8F041F5F726B82DE9F04FA3B04FF0EB
:10CEC000000A4FF0FF3BCDF818B0ADF864A08DF824
:10CED00068A0CDF828B0CDF81CB0CDF814B0CDF8CE
:10CEE00010B0CDF854A044680746CDF86CA0CDF83A
:10CEF00024A00020D7F808901490189008905F4E56
:10CF00001CA85546D0460B90B9F1000F08D016AAC0
:10CF100005A94846FDF753FD1790FDF74EFD149007
:10CF20009CB15A4A1AA919A80A9B8DE80F0096F9D4
:10CF3000003007A920460B9AFDF7FCFB0990FDF78E
:10CF4000F3FB1B90FDF7F3FB80467169C1F34000D2
:10CF5000002800F0D7804E480195806811F0400FFE
:10CF6000C0F3072B38680D901B98CDE90E080B987D
:10CF70001095CDE9125014981190BDF88400ADF8C9
:10CF80003000B069B56140F400701CBF11F0040FAF
:10CF900040F0010011F4807F18BF40F0040011F44C
:10CFA000007F18BF40F0080011F4806F18BF40F0F8
:10CFB000200011F4006F18BF40F0100011F4805FE2
:10CFC00018BF40F0400011F0800F18BF40F0800003
:10CFD000318AC1F3033140EA0140002918BF40F40F
:10CFE0008060002C08BF20F001000799B1F1FF3FDD
:10CFF00008BF4FF0010AF1780127012904BF04217D
:10D00000ADF8641005D0BDF86410072908BF77712A
:10D0100002D07179012902D10721ADF86410CDF851
:10D0200000A0BDF8643001AA0CA901F046FC8246BC
:10D030000198806820F0080110F0080FF16114BF1A
:10D040007770757013490968C96811F0040F05D12C
:10D050000B49096891F8831177292ED1BBF1A10FF3
:10D0600004BF7178002928D110F0100F25D0B078B6
:10D0700090B1F07801281AD01FE0000010070020BE
:10D08000E8060020E88611009C5D00201C070020B7
:10D0900014160020E48611003079F17808430CD191
:10D0A00000210120FFF7C1FEB770F77005E00021F5
:10D0B0000846FFF7BAFEB57037710198007A10F094
:10D0C000200FB07A07D070B9B7720122642107200F
:10D0D000FFF745F907E0012805D1B5720022642168
:10D0E0000720FFF73CF9019801680029CCBF377091
:10D0F0003570BAF1000F06BF4168002975721FD064
:10D10000D0F800B007980028C4BFF581F57206DC9E
:10D11000F189B0F1FF3F0CBF891C491CF181F74F29
:10D1200039680A7F12F0010F64D0497FF2898A4280
:10D130001CD8F26A012A18BFB0F1FF3F5AD115E09E
:10D14000017A4FF0C80211F0400F02D007957272B9
:10D15000D6E7717A29B1491CC9B27172C829F5D2D2
:10D16000CEE70799012908BF7772C9E7F581F57005
:10D1700035717571F089814204D20122992107200D
:10D18000FFF7EDF8F06A012804D102229921072067
:10D19000FFF7E5F80798B0F1FF3F04D1032299218A
:10D1A0000720FFF7DCF864B115991898CDE900085D
:10D1B000CDE902B1DDE90703DDE90921F7F72BFC31
:10D1C0007572179820B1726A01460598F7F70AFC44
:10D1D000F07A401CC0B2F07204280BD90520F0721E
:10D1E000B078012806D101210020FFF71EFEF5705E
:10D1F000B5703571C24C2078242804BF1B98FCF709
:10D20000E5FA2078012804BF1B98FCF7DFFA2078A4
:10D210000E2804BF1B98FCF7D9FAB9F1000F1CBF08
:10D22000307B022811D0386890F86C0010F0010FA4
:10D230000BD0BDF95800149A0599FDF7F5FC0028AC
:10D240001EBF012023B0BDE8F08FDDE90610DDE947
:10D250000432FFF738FD23B0BDE8F08FF0B587B09A
:10D260000746F7F703FC0546F7F703FCA549064612
:10D27000052D0CBFA44CAFF2BF344869C0F30311B5
:10D2800018BF052E08D1C0F300322AB1C0F34010F8
:10D29000002808BF41F002013846F7F7B3FC002828
:10D2A00004BF07B0F0BDF6F719FD07460020F3F7FD
:10D2B00018FCF3F798FFFBF7C8FF012809D0F7F730
:10D2C000D5FBA84205D1F7F7D4FBB04208BF002F29
:10D2D00005D0F3F785FEF7F718FD07B0F0BD6846F7
:10D2E000F4F751FA40B16846FCF7D9FB6846A0470D
:10D2F0000746F4F773FADEE7F7F7E7FBDBE72DE91C
:10D30000F04F002485B08149049423460E780094A0
:10D3100001940294224604A90394FDF70BFAFDF749
:10D3200003FA0546002700940194F7F79FFB734921
:10D330000528096851D0888FB1F83EA0C0F30B09C9
:10D34000000BB9FBF0F80020711E04468446EE463F
:10D35000029100210CFB06F3002E2ED935F9132083
:10D360003EF91CB0934505DA0DF1040B2EF81C2094
:10D370002BF81C104A451BDD3A4431B105EB43073D
:10D3800037F9027C3A44474500DD0120029FB9424B
:10D3900006D205EB4307B7F902703A44474500DD72
:10D3A000012401280CBF012C5245A4BF0122049284
:10D3B0000027491C5B1CB142D0D30CF1010CBCF11D
:10D3C000020FC6D34E480078012804BF2846FCF758
:10D3D000FDF9049805B0BDE8F08FB1F80001B1F88F
:10D3E00002A1C0F30B09000BB9FBF0F8ABE72DE984
:10D3F000F04F87B0064600240227FDF735FD0028D0
:10D4000004BF07B0BDE8F08F3E4D287DC0F3031A7E
:10D41000F7F72CFB8146F7F72CFB80465146304648
:10D42000F7F7F0FB002804BF07B0BDE8F08FE879FC
:10D43000374E4FF0010B4FF0000A012838D0F8F7B3
:10D440001FFEF8F7F9FE0120F6F78DFDF6F77BFCDD
:10D4500001464FF490622F4809F0A0FD85F807B00F
:10D4600002212020F3F7C0FF0020F3F756FC3068BC
:10D47000406C316840F400604864012200210020C3
:10D4800000BF401C0828FBDB491C9142F7DB3068D9
:10D49000406C316820F400604864F4F733FDF3F722
:10D4A000A2FEC5F830B0002C08BF1B4E7ED113E0A1
:10D4B0003068D0F82C03316820F00400C1F82C0348
:10D4C0003068C0F810A30120F3F7CDFB1148F6F740
:10D4D0003EFCF4F7BEFAC3E7FBF7B7FE012807D01E
:10D4E000F7F7C4FA484503D1F7F7C3FA404515D01A
:10D4F000F4F725FDF3F774FD9BE00000E80600203B
:10D5000031060020100700201F9F1000BE050020DC
:10D51000E8861100E2070020AA050020F7480078FD
:10D520009C2810D0F4F70BFDF5480168D1F82C13B6
:10D53000006841F00401C0F82C130020F3F75EF8F6
:10D5400086F800A005E0307818B9F4F7DBFCF3F7B3
:10D550004AFEEC4800684069C0F30720022808BF73
:10D56000F6F75DFA6846F4F70EF900285ED06846D3
:10D57000FCF795FAE4480068C06810F0040F287AB8
:10D5800015D0022827D0022028725A20F4F76DFC0B
:10D5900080220021B620F4F7B4FB00220121B6203E
:10D5A000F4F7AFFBA520F4F760FC14E041E002289B
:10D5B00011D1012028725A20F4F757FC11220021C2
:10D5C000B620F4F79EFB06220121B620F4F799FB62
:10D5D000A520F4F74AFC4FF0FF340198A346C0B1F0
:10D5E000FFF78DFE0028C8BF012410DCE889002465
:10D5F000401CE881C5480068017F11F0010F08D088
:10D60000807FE989814204D90198F6F7A0FBA5F84B
:10D610000EA0FDF7FDFA00231A4659462046FFF7F3
:10D6200052FB0446F4F7DAF8F4F7A3FC002C3FF4BD
:10D6300053AFF3F731F8F7F719FA022805D0F7F7E7
:10D6400015FA07460220F7F720FAF7F75EFB022FDC
:10D650001CBF3846F7F719FAF8F787FC07B0BDE8A2
:10D66000F08F2DE9F04FADF21C5DF5F74DFEFDF7A3
:10D6700060FAA64C2068B0F93610B0F93400FDF716
:10D6800005F8A3484FF0010B80F8C0B6A14880F818
:10D69000C0B62068B0F85800C0F303200F2818BFA8
:10D6A000F6F736FB9C4D686940F001006861F7F7BA
:10D6B000DDF9022808BF4FF0000A40F078812869A0
:10D6C000C0F303649148A1000068806DC5F820A0F4
:10D6D000C84000F00F00C5F824A0C5F828A0062C0B
:10D6E00080F05C81DFE804F0FC030303FBFB804671
:10D6F000686900274FF00209C0F30316022C0BD112
:10D70000C0F3003131B1C0F34010002808BF46F02B
:10D71000020601D026F00206A879012843D031463E
:10D720004046F7F76FFA002800F03881F8F7A8FCB8
:10D73000F8F782FD0020F6F716FC85F806B0FDF735
:10D74000E4F9686940F002006861A86940F00100EE
:10D75000A8610020F3F7E1FAF4F7D4FB694E3068D2
:10D760008068316840F002008860F3F73CFD85F87E
:10D7700000A000F06FFFDFF8A4813068C06810F0EF
:10D78000100F07D030688068316840F01000886062
:10D79000F4F7FDFBFBF759FD012812D0F7F766F906
:10D7A000022807D00DE0F7F7D7F931464046F7F7E2
:10D7B000EDF9C4E72869C0F30360A04208BF002F59
:10D7C0001AD0F4F7BCFBF3F70BFCFDF79EF9F8F762
:10D7D00095FBF7F74BF9022805D0F7F747F9814693
:10D7E0000220F7F752F9F7F790FAB9F1020F1CBFD0
:10D7F0004846F7F74AF9D1E0404800789C2810D015
:10D80000F4F79DFB3E480168D1F82C13006841F005
:10D810000401C0F82C130020F2F7F0FE88F800A0F5
:10D8200006E098F8000018B9F4F76CFBF3F7DBFC9E
:10D8300030684069C0F30720022808BFF6F7EFF808
:10D840000DF5A060F3F79FFF002896D00DF5A060BE
:10D85000FCF725F93248007801280FD14FF4A06178
:10D86000684609F03CFC00216846FDF73CFD2D4868
:10D8700000780B2804BF6846FBF7A8FF2248006821
:10D88000C06810F0040F287A14D0022826D0022095
:10D8900028725A20F4F7E9FA80220021B620F4F722
:10D8A00030FA00220121B620F4F72BFAA520F4F774
:10D8B000DCFA13E0022811D185F808B05A20F4F7F9
:10D8C000D4FA11220021B620F4F71BFA0622012116
:10D8D000B620F4F716FAA520F4F7C7FA01E023E022
:10D8E00009E00DF5A060FFF7E7FA0746F3F776FFCA
:10D8F000F4F73FFB41E7FFF77AFD4FE0AE0500206C
:10D90000E886110004871100E4861100E806002073
:10D910009C5D0020E207002010070020AA050020DF
:10D92000EF050020310600208046F7F79FF80646F5
:10D93000F7F79FF80746052E0CBF364CAFF6872445
:10D940006869C0F3031118BF052F08D1C0F3003276
:10D950002AB1C0F34010002808BF41F00201404640
:10D96000F7F750F9D0B1F6F7B9F980460020F3F790
:10D97000B8F8F3F738FCFBF768FC01280AD0F7F792
:10D9800075F8B04206D1F7F774F8B84208BFB8F19D
:10D99000000F12D0F3F724FBF7F7B7F9FBF755FCAC
:10D9A000012804D0F7F762F802283FF488AE0DF2A0
:10D9B0001C5DBDE8F04FFDF7BCB86846F3F7E3FE29
:10D9C00040B16846FCF76BF86846A0478046F3F71D
:10D9D00005FFD0E7F7F779F8CDE770470E4A022840
:10D9E000117D1269C1F30311C2F3074205D001286A
:10D9F00008BF11F0020F0AD002E011F0040F06D0A8
:10DA0000012101FA00F0104018BF012070470020EA
:10DA1000704700001F9F100010070020FE4870474D
:10DA2000FE487047FE4800787047FD4840787047D0
:10DA30000346002002460029D8BF704753F822C091
:10DA4000521C60449142F9DC70472DE9F05F0E46AC
:10DA5000054600F0D7FC044600F0D0FC310291FBF3
:10DA6000F0FC290291FBF4F3DFF8B4E3EB4D5E1216
:10DA7000BEF80490BEF8068000214FEA6C2705F539
:10DA8000907A002C0BDD01FB03F206EB222245F815
:10DA900021204AF82120491C09B28C42F3DCDE4ED9
:10DAA000002106F5907B00280BDD01FB0CF207EB53
:10DAB000222246F821204BF82120491C09B2884235
:10DAC000F3DC0CFB09FC03FB08F34FEA6C315A133F
:10DAD0005F13CEF80C102B684FEA6C3C9B1A2B603E
:10DAE00005EB840353F8045C154443F8045C336885
:10DAF0005B1A336006EB800353F8045C0D4443F873
:10DB0000045C9EF80330002BDAF8003017D09B1A23
:10DB1000CAF800300AEB84030BEB800053F804CC06
:10DB2000624443F8042CDBF80020521ACBF80020A2
:10DB300050F8042C114440F8041CBDE8F09F9A1AD8
:10DB4000CAF800200AEB84020BEB800052F8043C78
:10DB50003B4442F8043CDBF80020511ACBF800109B
:10DB600050F8041C6144E6E7AE4930B40968AC4A99
:10DB70004FF00A0C4C8A098A1423A2F804C0D380FF
:10DB8000A020108140005081204630BC5DE7A448B1
:10DB9000C078012818BF002070475FEA000C30B43D
:10DBA000A0489F4B0268508A118A14D092F854C042
:10DBB000528B4FEADC0404FB00FCBCFBF2F21A704F
:10DBC0005A700A229A801422DA80A0221A81520006
:10DBD0005A8130BC39E700221A705A70F1E7914837
:10DBE000026892F85430508AB2F81AC0DB084343F6
:10DBF000B3FBFCF3118A8A4A137053700A23938093
:10DC00001423D380A02313815B005381C0EB001346
:10DC1000B3FBFCF393700023D37016E72DE9F04FAC
:10DC2000B3B00D460446CC227F49684609F0FBF9A3
:10DC30007C48B5F902200068012A90F805C090F8E8
:10DC40000480478A068A687800FB0CF109B2D8BFC5
:10DC500001222B78DFF8D4E1EB4683B1ACF1010966
:10DC60004B45194417D104EB410131F9021C01293C
:10DC7000D8BF0121C902494291FBF2F140E004EB17
:10DC80004101B1F902100129D8BF0121C90291FB5C
:10DC9000F2F109B235E004EB410939F9021C01291E
:10DCA000D8BF0121B9F90290B9F1010FD8BF4FF0E7
:10DCB00001094FF0640A01FB0AF109FB0AF901EBC3
:10DCC000620109EB620991FBF2F199FBF2F93BF970
:10DCD00011103BF91990494508BF002111D001EB03
:10DCE000090A1AF5004FB8BFF24604DBBAF5004F37
:10DCF000A8BF47F6FF7AA1EB0901C90291FBFAF12F
:10DD000009B2A0B1A8F101094845A0F1010909FB38
:10DD10000CF90FFA89F9994415D134F91940012CFD
:10DD2000D8BF0124E402644294FBF2F246E003EB24
:10DD30000C0934F91940012CD8BF0124E40294FBEA
:10DD4000F2F212B23BE034F91990B9F1010FD8BFE9
:10DD50004FF0010900F1010A0AFB0CFA0FFA8AFAE6
:10DD60009A4434F91AA0BAF1010FD8BF4FF0010A52
:10DD7000642409FB04F404EB620494FBF2F44FF016
:10DD800064090AFB09F909EB620999FBF2F23BF914
:10DD900014403BF91220944208BF00220FD004EB3C
:10DDA000020919F5004F05DBB9F5004FB4BFCE46A7
:10DDB00047F6FF7EA21AD20292FBFEF212B21B04B9
:10DDC000000403EB011100EB021201F5004002F523
:10DDD000004190FBFCF091FBF8F1704301FB07F16F
:10DDE00000144FEA21414CBF00220246B242C8BF94
:10DDF000304602DC0028B8BF00200029B4BF002252
:10DE00000A46BA42C8BF394602DC0029B8BF002121
:10DE1000A5F880000CE00000007D0020907D00202F
:10DE20004807002060070020508B11000080FFFF92
:10DE3000A5F8821033B0BDE8F08F70B5A4B00D46E0
:10DE4000044616469021684609F049F90023002C43
:10DE5000C8BF684609DD55F8231056F82320514302
:10DE600040F823105B1C9C42F5DC002368461A46F0
:10DE7000002C05DD50F82210521C0B449442F9DCB2
:10DE80004FF0000C6246002C05DD55F82200521CB4
:10DE900084449442F9DC93FBFCF024B070BD2DE97E
:10DEA000FF4FADF54F7D0D460646904690216846E2
:10DEB00009F015F9902124A809F011F9902186A8FC
:10DEC00009F00DF99021AAA809F009F900F070FAFB
:10DED00000F07FFA00F09AFA074600F08FFA044645
:10DEE00000F090FA7190FA480068418A8591008AA2
:10DEF000CE9098F8012098F80000F649729102FB44
:10DF0000040090394891285C00F03F0A98F80C0012
:10DF1000499098F80D3098F80FB098F80E105B45BE
:10DF20009CBFE8460DF1900E23D8499A03FB04F0FC
:10DF30001FFA80F98A4218D809EB020036F910C09E
:10DF4000285C00F03F0050450BD1BC4509DB58F878
:10DF50002200604448F822005EF8230060444EF836
:10DF60002300501C82B28A42E6D9581C83B25B451A
:10DF7000DBD900216A460846002C7CDD52F82030AF
:10DF8000401C1944A042F9DB002974DD0021719A7C
:10DF900024AB0846002A6EDD53F820C0401C6144C3
:10DFA0008242F9DC002966DD69462046489AFFF77F
:10DFB00044FFDFF82493054699F80300D8BB489E38
:10DFC000A04606EB8804EB4654F804ACA422C349EF
:10DFD00048A8376809F027F848A9CB2D0ADC7B2D23
:10DFE00001DC282015E0C5F1CB0000EBD07040101B
:10DFF0001ED40EE042F23470A84219DC42F2847062
:10E000008542EEDAA5F51C50343800EBD070401094
:10E010000ED451F820003246391A316054F8041CED
:10E02000084444F8040C59464046FFF706FF0546ED
:10E03000376044F804AC24A9729A7198FFF7FDFE8A
:10E0400099F80310E9BBDDF8C491729E044606EB13
:10E0500089070DF1900B57F804ACF422A04948A8A9
:10E06000D6F8008008F0DFFF48A9642C08DC282CD3
:10E0700002DC3C2010E037E0D4F164001CD40BE05B
:10E0800041F21460A04217DC41F250608442F0DAA1
:10E09000A4F5B05014380FD451F820003246A8EB44
:10E0A0000001316057F8041C084447F8040C594635
:10E0B0004846FFF7C2FE0446C6F8008047F804ACA5
:10E0C0002046002DB8BF00250028B8BF0020CE99FB
:10E0D000491E8D42C4BFCE994D1E8599491E884266
:10E0E000C4BF8598401E01E000252846D2990D80C6
:10E0F000DC9908800DF5537DBDE8F08F10B47949A7
:10E1000092B0B1E81C108DE81C10B1E81C10CDE9EC
:10E110000423CDE9064C51F8042B0892B1E81C10F9
:10E12000CDE90923CDE90B4CB1E81C10CDE90D2355
:10E13000CDE90F4C096811910479B0F8802041783D
:10E140006B460DF1240C012C05D0B0F93640B4F526
:10E15000E17F18DD07E0B0F93440B4F52F7F02DC31
:10E160000478142C07D833F811101144A0F880104B
:10E1700012B010BC70473CF811101144A0F8801088
:10E1800012B010BC70470478142CF4D8EBE72DE9DA
:10E19000F74F4F488B4684B00168144691F85600FB
:10E1A00091F8551000F07F0A01F07F08C709CE09E9
:10E1B00000F0FEF800F00DF900F016F994F85B108D
:10E1C00001EB011202EB411100EB810500F01AF99D
:10E1D000814602A8009001AB224659460498FFF7F9
:10E1E0005EFE0AEB8A00C1B208EB8800C2B2002FC3
:10E1F0001CBF4842C1B2002E1CBF5042C2B2BDF883
:10E2000004000844A4F88000BDF808001044A4F8F5
:10E21000820095F8AC00012804BF287800280AD1B4
:10E22000687800281CBFA9F10101884203DA94F83C
:10E23000AD00012807D095F8BC0001280BD1E0887B
:10E24000E988884207D3B5F88000A4F88000B5F8C3
:10E250008200A4F8820094F8BF0001210222022863
:10E2600013D003281CBF07B0BDE8F08F84F8C1109D
:10E2700095F8C100012820D0022812BF03280320EE
:10E2800084F8C10007B0BDE8F08F84F8C11094F89D
:10E29000AC0000281CBF07B0BDE8F08F94F8B600B2
:10E2A00000281FBF94F8B900002807B0BDE8F08F20
:10E2B00084F8C12007B0BDE8F08F94F8B6000028BC
:10E2C00004BF94F8AC000028F2D007B0BDE8F08F8E
:10E2D00060070020B07E0020480700201C8C110041
:10E2E000C08C1100B48D110010B5044600F060F828
:10E2F00000F07AF8014694F85B0000EB001202EBA4
:10E30000401001EB8001012084F8C00094F8C100A6
:10E31000022202280FD0032818BF10BD91F8C000B8
:10E32000022811BF0328032084F8C00010BD94F810
:10E33000AE0028B110BD94F8AE00002818BF10BD83
:10E3400084F8C02010BD10B51446FFF720FF00F080
:10E350002FF800F049F894F85B1001EB011202EB82
:10E36000411100EB8101012084F8C00094F8C10044
:10E37000022202280FD0032818BF10BD91F8C00058
:10E38000022811BF0328032084F8C00010BD94F8B0
:10E39000AE0028B110BD94F8AE00002818BF10BD23
:10E3A00084F8C02010BD0000A4487047A4487047FE
:10E3B000A44840F2311100784843A34901EB4000E2
:10E3C0007047A048F52140784843A04901EBC000C0
:10E3D00070479C4840F23111007880F001004843BA
:10E3E000994901EB400070479648F521407880F04C
:10E3F00001004843954901EBC0007047914880688F
:10E40000407970478F488068007970478D488068F0
:10E41000B0F90C00704710B48D4991B0B1E81C10F0
:10E420008DE81C10B1E81C10CDE90423CDE9064CA1
:10E43000B1E81C10CDE90823CDE90A4C91E80E1093
:10E440000CAC84E80E103DF9100011B010BC704700
:10E450007C480079C0F3C00070477A480179C1F365
:10E46000C001002912BF19208068B0F90E00704762
:10E470007448017881F0010101707047714841785A
:10E4800081F00101417070474FF4F56108F027BE3B
:10E4900040F2622108F001BE2A2108F0FEBD694960
:10E4A00010B58860FFF79BFBBDE8104001F0B1B9E3
:10E4B0006448017881F001010170417881F0010127
:10E4C000417070475F49887070475E488078704738
:10E4D0005C49C87070475B48C078704759494860CC
:10E4E000704758484068704756488168497A11F02B
:10E4F000010F12BF00204068C0F300707047514800
:10E500000079C0F3800070474E484068C0F38060D7
:10E5100070474C480079C0F3C010704749480079F3
:10E52000C0F300107047474900200A7912F0040F29
:10E5300008BF70478978092914BF0A29012070474C
:10E5400040F2311200203F49097851433E4A02EB24
:10E550004101897A022908BF012204D0002203293F
:10E5600008BF012300D000231A4305290CBF012155
:10E570000021114318BF012070472DE9F0410546E5
:10E5800030484FF410718068067944792B4808F0C0
:10E59000A6FD0027002E8CBFDFF8A080BDE8F0812B
:10E5A0000121012C1ED907FB041082B205EB4200A9
:10E5B00035F912C030F9020CB0EB0C0348BFACEBDC
:10E5C00000031BB2C82BC8BFC823DBB208F8023057
:10E5D000012904BF08EB020000F8013C481CC1B24D
:10E5E000A142E0D3781CC7B2B742D9D3BDE8F081CD
:10E5F00070B5044613480D46F52140784843134949
:10E6000001EBC0004FF4F56108F069FD2046FFF70B
:10E61000B4FF2946204602F0E2FD05F028FE204620
:10E6200004F0B8FF2946204603F09BFC0146204633
:10E6300000F067FFBDE8704004F01AB98093002035
:10E64000407F0020580700206A7F0020308400208F
:10E65000FC8D110070B5FFF7ABFE0446FFF7B9FE65
:10E660000546FFF7A3FE064602F0E0FD2046FFF751
:10E670000FFF2846FFF70CFF3046BDE87040FFF75C
:10E680000BBF2DE9F0410446FFF792FE0546FFF768
:10E69000A0FE0646FFF78AFE07462046FFF7FFFE6C
:10E6A00002F0C4FD2846FFF7F3FE3046FFF7F0FE08
:10E6B0003846BDE8F041FFF7EFBE70B5FFF778FED2
:10E6C0000446FFF786FE0546FFF770FE0646204625
:10E6D000FFF7DEFE2846FFF7DBFE3046FFF7DCFEE5
:10E6E000BDE8704002F0A2BD70B50446FFF78AFE97
:10E6F0000646FFF783FE0546FFF75AFE237AA27A05
:10E70000217B94F80EC00024934298BF614507D93D
:10E710008471691E0172C471711E4172C47406E075
:10E7200083710272C17180F809C00121C1748472C1
:10E73000C4730474447470BD10B50446FFF75EFEE4
:10E7400014234FF0000C002C1CBF002100280ED910
:10E7500034F91120002AB8BF524292B29A4202DD27
:10E760004FF0020C03E0491CC9B28142F0D360466D
:10E7700010BD2DE9F04700261746884681463546EC
:10E78000FFF716FE0446FFF724FE034609F0FF00DC
:10E79000022818BF012807D0042818BF072803D073
:10E7A000987A022815D021E00221A1720121E1729C
:10E7B000042808BFA173012808BF84F8581207284D
:10E7C00008BF84F861120126187B20733046BDE82B
:10E7D000F087587C48B9187B012806D077484068F4
:10E7E000B84203D2D87A012800D10225A572002DA3
:10E7F0000CBF0020D87AE07218BF012684F8588236
:10E80000E2E770B50546FFF7D3FD0446FFF7E1FDEB
:10E8100029886180E969097C2170E969897C6170D6
:10E8200090F85A1284F85A12017D217590F85D1201
:10E8300084F85D12407D28B1604909783C293CBFCD
:10E84000607570BD0020607570BD2DE9F041154602
:10E850000E460746FFF7ACFD0446FFF7A7FD002371
:10E86000002F04BF84F85A3280F82830207C534AA5
:10E87000002818BF93600FD0A07D012804BF13703B
:10E88000BDE8F0811078401CC0B210703C2824BF55
:10E890003C201070BDE8F0819068401C9060A84258
:10E8A000EAD99560237584F85D32012EE4D1A37214
:10E8B000E37284F858322373DEE72DE9F05F002518
:10E8C0009B4691460E4680462C464FF0140AFFF7B1
:10E8D0006FFD07464046FFF701FE3846FFF7D8FDBB
:10E8E00018F0010FA84648D0F069FFF7FDFE524628
:10E8F00058460A99FFF73DFF8346FFF759FD054645
:10E90000FFF767FD31886980F169097C2970F16939
:10E91000897C697090F85A1285F85A12017D297520
:10E9200090F85D1285F85D12407D28B12349097881
:10E930003C2938BF687501D385F81580D6E90201F6
:10E94000FFF756FE054652465946FFF77EFF787D93
:10E95000002818BF0824B87A022808BF44F0200411
:10E96000787B012808BF44F0100497F86002012862
:10E9700008BF44F04004FFF79BFD11480560B7F95C
:10E9800002105A29C6BF397C4160C0F804808460F7
:10E99000C9F800002846BDE8F09F0120704701201B
:10E9A0007047012070470120704704484078704745
:10E9B000024948707047002070470000640700203B
:10E9C000C09500204FF6FF71A0F88010A0F88210CB
:10E9D000A0F88410A0F88610A0F88810A0F88A107B
:10E9E000A0F88C10A0F88E1070472DE9F04F85B07C
:10E9F000FFF7E7FC0490FFF7DBFC00252C460090B6
:10EA0000FFF7FCFC0098007D01280CBF4FF4DE717D
:10EA1000DE210098FE4A4FF00008407C012888BFA4
:10EA200082F800801CBF05B0BDE8F08F4FF00007F2
:10EA30000098007C00289CBF05B0BDE8F08F07EB74
:10EA4000071000EB4712049800EB820090F8C0C05A
:10EA5000BCF1020F18BFBCF1030F40F08681EC4EF1
:10EA60003278039252B3EB4BF278029233F822B031
:10EA7000B0F88230BBEB030954BF4A46A3EB0B024C
:10EA80008A42B8BF0124DFF890A3E14A12790192CB
:10EA90003AF822A0B0F88020BAEB02064CBFA2EBF5
:10EAA0000A0EB6468E45B8BF0125BCF1020F1ED036
:10EAB000BCF1030F00F0FB8000F0F4B8BCF1020FD2
:10EAC00040F053810122D34B3270B0F882C0A3F8DA
:10EAD00000C05A80B0F88030CF4803804280727006
:10EAE000B27086F8038086F8048000F03EB954EADC
:10EAF000050C04D0002C6DD0002D7DD0D2E0C44E8A
:10EB00004FF0000AD44696F80190B9F1000F88BF83
:10EB1000DFF800E328D93EF82CB0BBEB030648BF72
:10EB2000A3EB0B068E4216DAB94E86F803C0019AA3
:10EB3000521CD3B23371B278521CD2B2B2700F2AC7
:10EB40002EBF86F80080B44A02EB830280F00D816C
:10EB5000A2F80280A6E00CF1010C0CF0FF0CCC45F1
:10EB6000D9D3BAF1000F4FD1DFF8A4C200239CF82B
:10EB700002B0BBF1000F88BFDFF89CE226D93EF857
:10EB80002360B6EB020C48BFA2EB060C8C4516DAEC
:10EB9000DFF87CC28CF80430029A09F10103521CA0
:10EBA000D2B2DBB28CF803208CF801300A2B3CBFC8
:10EBB000984B03EB8202CBD38CF80080D5E05B1C32
:10EBC000DBB25B45DBD3BAF1000F6BD1904880F824
:10EBD0000080CAE0DFF838E24FF0000A52469EF8A3
:10EBE0000190B9F1000F88BFDFF828B214D93BF8C3
:10EBF0002260B6EB030C00E023E048BFA3EB060C59
:10EC00008C4502DA8EF803204CE0521CD2B24A4501
:10EC1000EDD3BAF1000F45D1029A09F10103521C5C
:10EC2000D2B2DBB28EF803208EF801300A2B02D369
:10EC30008EF8008099E0774B03EB8202A2F8028005
:10EC400030E0DFF8CCE14FF0000A53469EF8029026
:10EC5000B9F1000F88BFDFF8C0B112D93BF82360CB
:10EC6000B6EB020C48BFA2EB060C8C4502DA8EF81C
:10EC7000043017E05B1CDBB24B45EFD3BAF1000F59
:10EC800010D1019A09F10103521CD2B2DBB28EF805
:10EC900004208EF802300F2BCAD25F4B03EB8202A6
:10ECA000A2F80280039A5A4E012A12D05DE0DFF8E2
:10ECB00060C1B9F1000F48BFA3EB0B098945BFF64E
:10ECC0007BAF002E48BFA2EB0A068E42BFF674AFA0
:10ECD000E8E7DFF84091F27809EB820CBCF80230EB
:10ECE000F3B342F2107A53450DD2B0F882A039F84E
:10ECF00022B00BFB03AA5B1C9BB2ACF80230BAFB40
:10ED0000F3F329F8223039F82230B0F882209B1A28
:10ED100003EBD37302EB6302A0F88220DFF8F890D4
:10ED2000327909EB820CBCF8023083B342F21076E0
:10ED3000B3420DD2B0F8806039F822A00AFB036616
:10ED40005B1C9BB2ACF80230B6FBF3F329F822301F
:10ED500039F82230B0F880209B1A03EBD37300E01F
:10ED60000DE002EB6302A0F88020781CC7B2009887
:10ED7000007CB8423FF663AE05B0BDE8F08FB0F856
:10ED8000823029F822300122ACF80220C6E7FFE7E2
:10ED9000B0F8800029F822000120ACF80200E4E776
:10EDA0002DE9F047FFF70DFB0446FFF701FB024694
:10EDB000007D01280CBF4FF4DE707820517C174D88
:10EDC0000026A5F10C07012907D098BFBDE8F08700
:10EDD0003E722E806E80BDE8F08792F810C04FF032
:10EDE0000001BCF1000F98BFBDE8F08701EB0112F4
:10EDF00002EB411204EB820292F8C030022B18BFE2
:10EE0000032B0DD0491CC9B28C45EFD8BDE8F08763
:10EE100070070020CC950020F49500207C0700208E
:10EE20003B7A012B14D0002BF0D101EB011000EB49
:10EE3000411004EB800090F8C0000228E6D10120C8
:10EE40003872B2F880002880B2F882006880DDE76E
:10EE500001EB011303EB411304EB8303B5F80090BE
:10EE6000B3F88030B5F80280A9EB03030FFA83FCF6
:10EE7000B2F88230BCF1000FA8EB03031BB2B4BFA1
:10EE8000CCF1000AE246504538DB002BB4BFC3F199
:10EE9000000A9A46824531DC92F8C000022815D05B
:10EEA00042F6AB200CFB00F00114A1EBE07142F63E
:10EEB000AB2058430314A3EBE070A9EB0101A2F8C7
:10EEC0008010A8EB0000A2F882009FE746F267607E
:10EED0000CFB00F04114A1EBE07146F2676058436F
:10EEE0004314A3EBE073A9EB0100A2F88000A8EBA8
:10EEF0000301A2F882102880698087E73E722E8085
:10EF00006E8092E72DE9F04F83B0FFF75AFA04467E
:10EF1000FFF74EFA0746FFF771FA0190FFF772FA12
:10EF20000090787CFF4E01254FF0000A01280DD09B
:10EF30009CBF03B0BDE8F08F757186F807A003B0E1
:10EF40004FF00100BDE8F04FFEF70EBE7079B8B18A
:10EF5000397C002000299CBF03B0BDE8F08F00EB96
:10EF6000001202EB401204EB820292F8C020022A47
:10EF70006FD0401CC0B28142F1D803B0BDE8F08F21
:10EF800097F810B00023BBF1000F9CBF03B0BDE8A1
:10EF9000F08F4FF0020EDFF8908308F1060903EBC3
:10EFA000031000EB431204EB820191F8BF0002282A
:10EFB00005D0032804BFB079022832D078E003EBF3
:10EFC000031000EB431014F82000012816D9019B10
:10EFD0009B1E984212DA04EB8200407801280DD97A
:10EFE000009B9B1E984209DA757186F807A00120E4
:10EFF000FEF7BAFDB57103B0BDE8F08F04EB8200F7
:10F0000086F806E0B0F88000A9F80000B1F88200A8
:10F01000A9F8020088F800A088F801A003B0BDE8B4
:10F02000F08FB9F80000B1F88070B1F882C0C21B4F
:10F03000B9F80200A0EB0C014CBF50421046F0287A
:10F0400018DD98F8000028B101280AD002280CD059
:10F050000EE035E0002AB4BF88F8005088F800E0E0
:10F0600006E0002A3FF768AF02E0002AFFF664AF2F
:10F07000A9F800700029B4BF48420846F02817DDFF
:10F0800098F8010020B1012809D002280BD00DE02A
:10F090000029B4BF88F8015088F801E006E0002993
:10F0A0003FF74AAF02E00029FFF646AFA9F802C0D9
:10F0B000581CC3B29B453FF672AF03B0BDE8F08F5A
:10F0C00086F807A003B0BDE8F08F2DE9F0410446B3
:10F0D00096480068C68A858AFFF786F9024694F842
:10F0E000C0000023022823D0032818BFBDE8F08108
:10F0F000207903281CBFB4F88C000A2898BFBDE80B
:10F10000F081A6F10B0C6045A8BFBDE8F081B4F812
:10F110008E000A2898BFBDE8F081A5F10B01884256
:10F12000A8BFBDE8F08194F8B300012842D064E0A4
:10F130007C49012248790028B4F88C0019D00A28AB
:10F140000DD9A6F10B0C604509DAB4F88E000A2837
:10F1500005D9A5F10B0C6045B8BFBDE8F0810B7275
:10F1600084F8B3204A71CB71BDE8F0410120FEF76D
:10F17000FBBC0A280DD3A6F10B0C604509DCB4F8E2
:10F180008E000A2805D3A5F10B0C6045D8BFBDE859
:10F19000F0810B7284F8B3202079032808BFBDE802
:10F1A000F08184F8B4204A71CB71BDE8F0410120B0
:10F1B000FEF7DABC94F85B0000EB001707EB401099
:10F1C00002EB80000B27B0F88C200A2A98BFA4F825
:10F1D0008C7005D96245A4BFA6F10C02A4F88C205E
:10F1E000B0F88E000A2898BFA4F88E7005D988421E
:10F1F000A4BFA5F10C00A4F88E0084F8B330BDE8DC
:10F20000F0812DE9F04FADF5197DFFF7DAF8939015
:10F21000FFF7CEF80646FFF7DCF80446FFF7E4F800
:10F22000929006F1170004F117059090FFF7E6F8A9
:10F2300000279190307C3C463B46002871D903EB77
:10F24000031000EB4311939800EB810191F85B00F0
:10F2500000EB001202EB4012929800EB820991F849
:10F26000AF00012868D191F8BF00022818BF032819
:10F2700062D1601CC4B291F859202D4800EB820C79
:10F280003CF8048CA8F57F40FF381FBF3CF8022CE7
:10F29000A2F57F40B0F1FF00404604BFB9F8060078
:10F2A000B9F80820B1F80690CDF8549209F1050A92
:10F2B000DFF88090A9FB0ABACAF3CF0ECDF860E25E
:10F2C000B1F808E0CDF850E20EF1050AA9FB0ABA40
:10F2D000CAF3CF0ACDF85CA200F1050AA9FB0ABA6D
:10F2E000CAF3CF0B02F1050AA9FB0AA9C9F3CF0A99
:10F2F000DDF854924CF6CD4E09FB0EF94FEAD94990
:10F30000CDF85892DDF850E24CF6CD490EFB09F9E4
:10F310004FEAD949CDF854924CF6CD4900FB09F992
:10F320000BE040E0700700207A0700206007002013
:10F3300030960020CDCCCCCC2DE04CF6CD4E02FB4F
:10F340000EFE4FEADE4ECDF850E2DDF860E24FEA05
:10F35000D949DE4504BFDDF85CB2D34507D0DDF8FE
:10F3600058A2CA4504BFDDE9949ACA4513D17F1C4F
:10F37000DFF8A0924FF6FF7AFFB2D04504BF3CF809
:10F38000028CD04507D12CF8040C91F8590009EBF8
:10F39000800020F8022C581CC3B2307C98423FF603
:10F3A0004EAFA7427ED1707C02287BD39A49487A1F
:10F3B000401CC0B248721E283CBF0DF5197DBDE847
:10F3C000F08F1E2048724FF410726846909907F033
:10F3D000E5FD307C4FF0000B002874D90BEB0B10CF
:10F3E00000EB4B11939800EB810191F85B0000EB6F
:10F3F000001202EB4012929800EB820291F8AF00EB
:10F40000012859D191F8BF00022818BF032853D111
:10F410000B7891F801C091980CFB00339098C05C78
:10F420000B7B00F03F0A107B984238BF0873507B7B
:10F430004B7B984238BF4873907B8B7B984288BF48
:10F440008873D07BCB7B984288BFC873087B95902C
:10F450004C7B9494137892F801C0919A91F80F80A4
:10F460000CFB0232887BAA5C444502F03F091CD8A1
:10F47000919A624397B2959A824210D8BB1815F8B8
:10F4800003C00CF03F0ECE4505D12CF03F0C4CEAEA
:10F490000A0C0DF803C0521C92B28242EED9621CD3
:10F4A00094B200E019E04445E2D9959A0A73949A1F
:10F4B0004A73887381F80F800BF1010000F0FF0B95
:10F4C000307C58458AD84FF410726946909807F0FE
:10F4D00065FD0DF5197DBDE8F08F4F4800214D4ABF
:10F4E000417208464FF6FF7122F8201002EB8003AC
:10F4F000401CC0B259800A28F6D30DF5197DBDE82D
:10F50000F08F2DE9F0470F468246FEF75AFF064678
:10F51000FEF74EFF0446002F57D1207C04F1170957
:10F52000002852D0FFF76DFE207C0025002888BF00
:10F530004FF6FF7822D905EB051000EB451006EBDE
:10F54000800292F8AF00012813D1A2F88080A2F8BF
:10F550008280A2F88480A2F88680A2F88880A2F82F
:10F560008A80A2F88C80A2F88E8049465046FEF729
:10F57000EAFE681CC5B2207CA842DCD8002510F049
:10F58000FF0F22D005EB051000EB451006EB8000C5
:10F5900090F8C010022918BF032906D090F8C110B6
:10F5A000022918BF032903D00AE000F0F4FE07E0A7
:10F5B000B0F88010A0F88410B0F88210A0F886107F
:10F5C000681CC5B2207CA842DCD8207C002500281D
:10F5D00098BFBDE8F08705EB051000EB451006EB82
:10F5E000800090F8AF1001290CD190F8BF100229CB
:10F5F00018BF032906D190F8B810002904BF394676
:10F6000001F0B4F9681CC5B2207CA842E3D8BDE87B
:10F61000F08700003096002070070020F8484078FE
:10F62000002818BF01207047F648006890F858007D
:10F6300000F001007047F34909688A6D60F3000229
:10F640008A657047EF4B10B4D3F800C0BCF8123095
:10F6500003FB00F4BCF81A005943B4FBF0FCB1FB07
:10F66000F0F10CFB0CF4DFF8A0C34943CCE90841EE
:10F6700003FB02F1B1FBF0F04043CCF8280010BCD2
:10F6800070474FF6FF7202EA0023DF4802EA0121C9
:10F69000C38501864FF4A051418649108186704789
:10F6A0002022D94906280ED2DFE800F00D030D050F
:10F6B000080A102000E04020888570478020FBE782
:10F6C0004FF48070F8E78A85704700B502220A215E
:10F6D0000C20FFF7B7FFDFF82CC30A231422DCF855
:10F6E000000090F85C00C0F3031100F00F00FFF77A
:10F6F000C8FFDCF80000B0F85C005DF804EBC0F374
:10F700000330CDE72DE9F04190460D460446FEF763
:10F710004FFEBE48BB4E47190A380544BCB1012C08
:10F720003AD0022C4DD0032C18BFBDE8F081042242
:10F730000E210F20FFF786FF30680A231422B0F84D
:10F740005C00C0F303200146FFF79BFF1CE0022290
:10F750000A210C20FFF776FF15F8010C002801BFE5
:10F7600017F8010C002898F8BF00032830684FF004
:10F770000A034FF0140290F85C00C0F3031100F08C
:10F780000F00E1D1FFF77DFF3068B0F85C00BDE805
:10F79000F041C0F3033083E702220E210F20FFF770
:10F7A00051FF30680A231422B0F85C00C0F3032133
:10F7B00000F00F00491CFFF764FFBDE8F041042092
:10F7C0006EE715F8010C012804BF17F8010C012899
:10F7D0004FF0040219BF112112200C210D20FFF758
:10F7E00031FF15F8010C02283068C06D18BFC0F356
:10F7F0000351C0F303404FF00A034FF0140208BF57
:10F800000321FFF73EFF3068C06DBDE8F041000FF7
:10F8100046E730B57B4C7A4D02222068418A408B06
:10F820008900B1FBF0F04043A8600A210C20FFF7EB
:10F8300009FF20680A23142290F85C00C0F303112A
:10F8400000F00F00FFF71DFF2068B0F85C00C0F368
:10F850000330FFF725FF05F110014FF6FF70088018
:10F86000488005F10C004FF0FF31018041800020FD
:10F87000287030BD644B03EB400003898B4288BF86
:10F88000991A38BF991808BF7047018170472DE950
:10F89000F04F83B09B460D460446FEF789FD01906C
:10F8A000FEF7A2FD0246574894F859A0DFF850E150
:10F8B0000068554B418A408BC1EB0111890091FBD7
:10F8C000F0F094F8C0104043022911D0A3F1500188
:10F8D00001EBCA0151E9026794F85810B5F80080AD
:10F8E0000229B5F8029094F8A81014D041B335E07D
:10F8F000002103EB0A0C2E886F880CF8011C03EB27
:10F900004A08B3F834C0A8F808C0BAF1010F08BF1C
:10F910008EF80110E0E709B394F85B1001EB011CCD
:10F920000CEB411102EB810191F8A810B1B903EB86
:10F930004A02198EB2F808C08C4588BF11810DE0CB
:10F94000834524BF94F8C010032907D103EB4A0173
:10F950001A8EB1F808C0944588BF0A81217902291E
:10F9600018BF032906D094F8A81019B9834538BFE9
:10F97000998E00D3598E598694F8A8C0BCF1000F17
:10F9800008D1834594F8C00002D2032813D101E0C6
:10F99000022810D061469A6A5A4588BF0221009118
:10F9A0009EF801100122002904BFBAF1010FBCF139
:10F9B000030F0BD101E00221EDE713488EF801207F
:10F9C0004189188E814284BF0F4948810E4B0C99A2
:10F9D0000098D3F820C0DC4503D8022801D00129C3
:10F9E00008D0094B4FF0020E5A6A5A4510D9022826
:10F9F0001ED10DE00448504400F8012C24E0000022
:10FA00008407002060070020A8960020EA960020C6
:10FA100071B15A4598BFE3450FD202280FD003EBCE
:10FA20000A0010F8011C032908BF00F801EC0BE0E4
:10FA300003EB0A0000F801EC06E0022804D103EB16
:10FA40000A00032100F8011CFEF7B2FCFE4B8646BB
:10FA500003EB0A02988D12F8012C198EB3F82EB020
:10FA6000B3F832C0022A04D0012A1CD0032A6DD078
:10FA700032E003EB4A0201EB410CB2F808B0E34577
:10FA800006D99EF80AB0BBF1000F08BFA2F808C063
:10FA9000B2F808C08C4588BFACEB000038BF6044AA
:10FAA0001AD0108118E003EB4A0CBCF808209142F0
:10FAB0000AD2501AA2EB6000000A4FF6FF7101EA69
:10FAC0000020ACF8080007E05A4588BF101A38BF7C
:10FAD000104401D0ACF8080003EB4A000289002A68
:10FAE00004BF002001461FD01046B2F5807F36BF0C
:10FAF0004FF4807101464FF48072D448009B022B72
:10FB00002ED094F859C000230CF80030A1F5807075
:10FB1000704300EB0820B0FBF1F0A2F5807179434F
:10FB200001EB0921B1FBF2F194F85930C84A02EB1C
:10FB3000C30343F8080C94F8593002EBC30242F8AF
:10FB4000041CA880E98003B0BDE8F08F03EB4A02F3
:10FB50001189614588BF081A38BF0844A1D1BBE7A5
:10FB600094F859C01CF80030FA2B3CBF5B1C0CF811
:10FB7000003094F85930185C3C28C7D30198090A22
:10FB8000120A407C0228B348006818D3B0F818A0C5
:10FB9000B0F81AC00AFB08F3B0F810800CFB09F9A2
:10FBA000408AB3FBF8F30AFB06FA0CFB07FCB9FB2F
:10FBB000F0F9BAFBF8F8BCFBF0FCB34617E0B0F87C
:10FBC00014A0B0F816C00AFB08F3B0F810800CFBC4
:10FBD00009F9408AB3FBF8F30AFB06FA0CFB07FCB1
:10FBE000B9FBF0F9BAFBF8F8BCFBF0FCB346A1F1A5
:10FBF000010000FB0830B0FBF1F3A2F1010000FBB3
:10FC00000C90B0FBF2F293480168B1F8109009FB38
:10FC100003F009D3B1F81890B1F812A0B0FBF9F0D5
:10FC20000AFB02F9498B08E0B1F81490B1F812A070
:10FC3000B0FBF9F0C98A0AFB02F9B9FBF1F14345BF
:10FC400018BF62457FF470AF434508BF5846624510
:10FC500008BF394668E72DE9F04F90F859C08FB0DA
:10FC60004FF4806300290CBF7B4C7C4C04EB4C149C
:10FC70007B4D029205EB4C1705F5A5756544203CBC
:10FC800015F8015C07EB051606EBC10858F8206C67
:10FC9000921B039290F8C00002287CD058F81C8C6C
:10FCA00004EB051206EB0809CDF83090D2F8049069
:10FCB000D6689568106809EB0602DFF8A891284419
:10FCC0001044D9F800A035445044D9F804A0524457
:10FCD000D9F808A0D9F80C9055444E44DDF808A096
:10FCE000DDF83090AAEB0909CDF82090DDF80C90F2
:10FCF000DFF874A1A9EB0809CDF82C90DAF8009090
:10FD000009EB000ECDF828E0DAF80490DAF808B034
:10FD1000DAF80CA09144B244AB440EFB0AFE09FB96
:10FD20001BEE9EFBF3FEBEF1000F08BF4FF0010E6D
:10FD30004FEA8A2A9AFBFEFA4FEA892999FBFEF9D3
:10FD4000CDF838A0C9F1000A4FEA8B29CDF834A0CC
:10FD5000DDF828A099FBFEF94FEA8A2A9AFBFEFB00
:10FD6000DDF838A0C9F1000900FB0AFA02FB09AA74
:10FD70009AFBF3FEDDF834A0CDF828E000FB0AFA88
:10FD800002FB0BAA9AFBF3FECDF824E0DDF838A0C5
:10FD900005FB0AFA00E073E006FB09A999FBF3F9F9
:10FDA000DDF834A0CDF8389005FB0AF906FB0B9975
:10FDB00099FBF3FADDF828E0DDF820900EFB09FB53
:10FDC000DDF824E0DDF82C900EFB09BEDDF820B054
:10FDD000DDF838909EFBF3FE09FB0BFBDDF82C9061
:10FDE0000AFB09B999FBF3F9C844DDF830B0DDF836
:10FDF0003890F344CDE900B8DDF828E0C9F10009F6
:10FE0000CEF58068DDF824E0CAF5806ACEF1000BFB
:10FE100008FB00FE0BFB05EE08FB02F809FB00F0F7
:10FE20000BFB06880AFB05009EFBF3FE98FBF3F82C
:10FE300090FBF3F0CDF810E0CDE9058009FB02F06E
:10FE40000AFB060012E00000A89600209D97002003
:10FE50005896002060070020A8970020E89800200E
:10FE6000289A0020C0070020D007002090FBF3F064
:10FE70000022E84604AE0790FE4800EB0C0315E0B4
:10FE8000FC4A00206244039012F8012C02AB07EBFD
:10FE9000021202EBC10253F8204002EB8005401C25
:10FEA00000B245F8204C0228F5DB20E013F8015C95
:10FEB00058F8220007EB051505EBC10505EB820597
:10FEC00045F8200C002006EBC20513F801AC55F8EC
:10FED000209004EB0A1A0AEBC20A4AF82090401C50
:10FEE00000B20228F1DB501C02B2022ADEDBE1483C
:10FEF000604410F8010C07EB001000EBC10050F853
:10FF0000200C0FB0BDE8F08F70B4012803BF0224AD
:10FF100001204FF0000C04241CBF03204FF0010C03
:10FF20000026D54D0029C8BF204609D00CEB8C0116
:10FF300005EB810101EB420121F8026C70BC7047B6
:10FF4000CE480CEB8C0100EB4100104405EB810125
:10FF500001EB420210F8010C32F8021C642924BFA4
:10FF600070BC7047491C22F8021C0121197070BC3A
:10FF700070472DE9F0010128DDE9055614BF012085
:10FF8000002000EB8000DFF8F4C20CEB400C8C4446
:10FF90001CF801CCBCF1000F04BFBDE8F0017047B4
:10FFA000DFF8DC82002408F13C07944531D1A7F149
:10FFB000280202EB800202EB410232F8022C9A4244
:10FFC00007D908EB4000084400F8014CBDE8F001F7
:10FFD000704708EB40020A4412F8013C642B24BF2E
:10FFE000BDE8F0017047002E1CBFBDE8F00170476E
:10FFF0005B1CDBB202F8013C0A2B3CBFBDE8F00100
:020000021000EC
:10000000704707EB4000084400F8014CBDE8F001E0
:10001000704708EB40020A4407EB400012F8013C2D
:100020000844052B36BF10F8011C00F8014C642968
:1000300004D20A2DA4BF491C00F8011C02F8014C8F
:10004000BDE8F00170472DE9F04F89B0824608887D
:10005000ADF8100048888946ADF81400FEF7A8F9FD
:1000600000909AF8C0009AF85940022804BF204630
:1000700000F0D3FC8348874A2044089010F8015CC4
:1000800081488349204402F1080C00F8015C7F4854
:1000900000EB040818F8010CD8B1681CC0B2142891
:1000A00021D304EB840001EBC00000EB450330F8E2
:1000B00028EC33F828BCAEEB0B0B02EB840E4EF8A9
:1000C00004BC1B8D008DC01A0CEB840343F8040C98
:1000D00020E002EB8403002043F8040C0CEB8403C3
:1000E00043F8040C16E004EB840301EBC30303EBB9
:1000F000400030F8283C30F82ABCA3EB0B0302EB9D
:10010000840B4BF8043C038DC08C181A0CEB840351
:1001100043F8040C04EB840001EBC000079000EBF3
:100120004500BDF8103020F8283CBDF814B0A0F808
:1001300028B0132D04BF012008F8010C9AF8C00064
:1001400003284FD1002D1CBF681EC0B25AD007999A
:1001500001EB400030F8281C008DA3EB010118F8DA
:10016000013CABEB00000193002B52D04A4B00291D
:1001700003EB840656F8047CACBF0B464B4207EBFE
:10018000030B464B46F804BC03EB8403002853F8EA
:1001900004ECB4BF47420746774402EB840243F8BD
:1001A000047C52F8042C002AB8BF5242ABEB020286
:1001B00046F8042C0CEB840252F8042C002AB8BF39
:1001C0005242BA1A43F8042C354A1268138B594329
:1001D000138A91FBF3F6518B4843518A90FBF1F758
:1001E000019878B32F4802212044069000F8011CA2
:1001F0002D4800EB040B0BF8011C9AF8A80003280B
:1002000061D15DE018F8010C01280CBF13202846CD
:100210009DE7214A002902EB840252F804CCB4BFC6
:100220004B420B46634442F8043C1C4A002802EB54
:10023000840252F804CCB4BF43420346634442F8FC
:10024000043CC1E7FFE71948002E00EB440030F8FA
:10025000022CB4BF714231468A4205DA002EACBF8F
:100260003146714220F8021C4288002FB4BF794207
:1002700039461DE0689B0020669D00203E9D0020C1
:10028000529D002086070020880700208A07002052
:10029000F496002098070020B0070020B80700203F
:1002A00060070020E0960020EA960020A8070020C2
:1002B0008A4297DA002FACBF39467942418091E7F4
:1002C000FEF71DF968B1204600F0A7FBBDF810004D
:1002D000A9F80400BDF81400A9F8060009B0BDE8AB
:1002E000F08F18F8010C012803D0D8B9691C072930
:1002F00018D3282ED8BF282F09DCFD4901EB440173
:1003000031F8022C282A9CBF4988282919D900983D
:1003100090F85A02012805D10699032001F8010C32
:100320000BF8010C0898089910F8010C401CC0B299
:1003300001F8010C1428C9D30899002001F8010C18
:10034000C4E7EC494FF0000C01EB840151F8042C98
:10035000E94901EB840151F8041C8A42C8BF4FF0FF
:10036000010C05A904AA1423CDE90003CDE902215B
:1003700007982B4600F12802A0F12801604600F002
:1003800074FB01280CBF01200020069901F8010C24
:100390000BF8010CC6E72DE9F04F8DB00446FDF7D0
:1003A00041FB0490FDF741FB0890FEF71DF88146E4
:1003B000FDF7FEFF079094F85960FDF7F9FF827A88
:1003C00094F859100127002A04BF427D002A06D163
:1003D000027D012A1CBF90F85D22012A01D180F81C
:1003E0005A7200258DF819508DF818708DF8175035
:1003F00090F85A02DFF804830028D8F800007DD076
:10040000826DC2F3C0438DF81430C2F340428DF8C0
:100410001520806D2246C0F380408DF81600022022
:10042000FFF770F9B548D0F8008098F8580010F040
:10043000010F00F0468294F85B10B4F8800001EBE5
:100440000112ADF8080002EB4111B4F8823009EB5B
:100450008101ADF80A300B9194F8591094F8C0C09E
:10046000A74A01EB4101BCF1020F02EB81017CD0F4
:1004700031F80AAC21F808AC31F80C2C21F80A2C20
:1004800021F80C0C31F8049C21F8029C31F806CCC0
:1004900021F804CC21F8063C81B261F30F0062F32D
:1004A0001F40914284BF62F30F0061F31F40010CB3
:1004B000514588BF6AF31F4081B2020C914284BF4C
:1004C00062F30F0061F31F40000C63F30F016CF344
:1004D0001F41634584BF6CF30F0163F31F410A0C96
:1004E0004A4588BF69F31F418AB20B0C9A4284BF08
:1004F00063F30F0162F31F410B0C00E010E09DF865
:100500001410ADF80C00ADF80E30012904BFADF8A1
:100510000800ADF80A3094F8C00002283AD0B0E0E4
:1005200090F85820C2F3C0038DF81430C2F3400293
:100530008DF8152090F85820C2F380028DF816200F
:100540002279022A1EBF032A224600207FF468AFC8
:10055000826DC2F3C0438DF81430C2F340428DF86F
:100560001520806DC0F3804000E006E08DF8160095
:1005700022460220FFF7C6F854E721F8080C21F8BC
:100580000A0C21F80C0C21F8023C21F8043C21F85B
:10059000063CB2E75B484FF0000C304400F8015CC9
:1005A00059480195304400F8017C584800EB46104A
:1005B0000A90574800EB46100990564800EB461049
:1005C00000900999002001EB0C1E009901EB0C1B17
:1005D0000A9901EB0C1900210EEBC0020BEBC003D2
:1005E00009EBC00702EB810A4AF8205C03EB810AA1
:1005F0004AF8205C07EB810A491C09B24AF8205CE2
:100600000229EFDB401C00B20228E4DB0CF1010000
:100610000FFA80FCBCF1020FD3DB099A0198DFF8D6
:10062000F8E002EB001ADDE90002002100EB0219FC
:100630003A4A002002EBC1070AEBC10C09EBC105E5
:100640000EEBC103814207D1B8F8622043F82020A5
:10065000B8F8602047F8202053F820200CEB800BDE
:1006600002EB820252004BF8202C05EB800B401C61
:1006700000B24BF8202C0228E4DB481C01B202290E
:10068000D6DBBDF8082000212046FFF7E4FA054636
:10069000BDF80A2001212046FFF7DDFA002DB8BF82
:1006A00000250028B8BF0020144F3968B1F9102088
:1006B000531EAB42B8BF1D46B1F912104A1E82420A
:1006C000B8BF1046AAB283B20E48ADF80C2081190B
:1006D0000A30ADF80E30304411F801CC10F8015C4E
:1006E00001F8015C00F801CC9DF81600012817E024
:1006F000A8070020B0070020B807002060070020EE
:100700007C9B0020689B0020729B0020289A002080
:10071000A8970020E8980020C0070020D0070020FC
:1007200004BFADF80820ADF80A3020460B9900F060
:100730008BFA94F858100B98022918BF002529D07D
:10074000C4F89050B4F88010B0F88020DFF86C84C2
:10075000891AC4F89410B4F88210B0F8820008F135
:100760000A09081AC4F89800022E9CBF9DF81700C9
:10077000012823D008EB0601022001F8010C09EB47
:10078000060101F8010C08EB0601002011F8011C1C
:10079000B1BB36E0B4F88010B0F88030CA1A48BF58
:1007A0005A1AB4F88230B0F882C0B3EB0C0148BFDB
:1007B000ACEB0301524301FB0125C1E72A4602A924
:1007C0002046FFF740FC079890F85A020028DAD13B
:1007D000FB48304410F8010C012808D00028D2D181
:1007E000F848304410F8010C401C1428CBD9BDF84F
:1007F0000C00ADF80800BDF80E00ADF80A00C2E725
:1008000004E009EB060111F8011C01B10120009080
:1008100007982B4602A9427C2046FFF738F89DF83E
:100820001500012840D0BDF80800A4F88400BDF8E8
:100830000A00A4F88600BDF80810049ABDF80A0062
:100840009142B8BF1146089A9042B8BF10463B6823
:10085000049AB3F910C0ACEB0202A2F1010C8C4572
:10086000B8BF6146B3F91230089A9A1A531E8342F0
:10087000B8BF184689B2A4F8841080B2A4F88600E4
:100880000B9AB2F88420891AC4F8A0100B9AB2F817
:100890008620801A4943C4F8A40000FB0010C4F865
:1008A0009C000DB0BDE8F08FBDF80C00ADF808005D
:1008B000BDF80E10ADF80A10A4F88400BDF80E00C3
:1008C000B7E7B4F88000A4F88400B4F88200A4F874
:1008D00086000DB0BDE8F08FBB4A30B4146894F8C0
:1008E000542012F0040F1ABF012323EA020502F07C
:1008F0000105B0F900C0B1F900301DB1E58AEB1A6D
:100900005B1E1BB212F0020F06D0A48AA4EB0C0CE3
:10091000ACF1010C0FFA8CFC12F0040F19BF03802C
:10092000A1F800C0A0F800C00B8030BC7047A64AF8
:1009300030B41268B2F8983013F0FF024FEA132374
:1009400008BF6422002B08BF64230488B1F800C0EC
:1009500062439E4CA4FB0252520902800CFB03F03E
:10096000A4FB00204009088030BC70472DE9F04707
:100970000446954882B00068B0F818A0B0F81A9004
:10098000858AC68A078AB0F812800020ADF8000078
:10099000ADF80400FDF70CFDB4F88410B4F886003F
:1009A00001FB0AF292FBF7F2A4F8882000FB09F29F
:1009B00092FBF8F26943704391FBF7F190FBF8F07A
:1009C000A4F88A20ADF80010ADF8040001A968462B
:1009D000FFF782FFBDF90000711E8842A8BF0846DC
:1009E00000B2BDF904106A1EADF800009142A8BF24
:1009F000114609B2ADF804100028D8BF0020ADF8A8
:100A000000000029D8BF0021ADF80410A4F88C0024
:100A1000A4F88E1002B0BDE8F0876A4A00210244B3
:100A200002F8011C6A4A024402F8011C644A0244AA
:100A300002F8011C674A02EB800242F8041C664A75
:100A400002EB800242F8041C644A02EB800242F886
:100A5000041C634A02EB800242F8041C614A02EB68
:100A6000400020F8021C418070472DE9F0439BB004
:100A70001F468C46DDE923350021DDF888800646D7
:100A8000259C12911391149115911691179118911B
:100A900038461991B8F1000F14BFA3F10A07471C9B
:100AA000052F40F2CD804FFA80F909F1010189B29A
:100AB0008B4298BF0021B8F1000F6FD03CF8118035
:100AC000CDF8488032F811101391A9EB530109B207
:100AD000002901DA194409B23CF81180CDF85080A0
:100AE00032F811101591F9B2CDE900310DF110086D
:100AF00013460146CDF808806246304600F005FAFC
:100B000016902A88039230492088069009684B8AFB
:100B1000B1F81AC0C3EB0313B3FBFCF317934B8A72
:100B2000B1F81AC0C3EB0313B3FBFCF318934B8A61
:100B3000498B03EB83035B00B3FBF1F11991DDF803
:100B40005CC0002E4FF000014ED0129B059A5A4314
:100B5000049B03EB2242139BD31A44BF139B9B1AA3
:100B6000634569D2149B059ADDF860C05A43049B23
:100B700003EB2242159BD31A44BF159B9B1A634576
:100B80005AD2169A199B821A44BF169A121A9A427E
:100B900052D2169880B206904DE0FFE7BCF8008074
:100BA000CDF84880B2F8008021F00101CDF84C80EA
:100BB0003CF80180CDF85080515A93E7E096002030
:100BC0008A07002088070020600700201F85EB515E
:100BD00086070020B0070020B807002098070020F3
:100BE000A0070020A8070020139B05985843049BEA
:100BF00003EB2040129BC31A44BF129B1B1A634590
:100C00001AD2159B0598DDF860C05843049B03EB8E
:100C10002040149BC31A44BF149B1B1A63450BD27C
:100C20001698199B101A44BF1698801A984203D23E
:100C3000169880B20390012103982880069820809E
:100C40001BB00846BDE8F0832DE9FF4F8BB09B46F3
:100C50008A460546FDF7ACFB90F85A22BAB114203B
:100C60004FF002080290287995F85940FE49022871
:100C700018BF032815D0012A1CBFFC4886681AD06B
:100C800095F8C000FA4A0027022840D11DE03C2117
:100C90000291407C02282CBF4FF003084FF00F0850
:100CA000E1E708686423428A408B5A43B2FBF0F0C4
:100CB00000FB00F6E4E70868428A408BC2EB0212B0
:100CC000B2FBF0F000FB00F6DAE7101900F8017C47
:100CD000E848204400F8017C4772E748204400F8C7
:100CE000017C4772E54800EB440020F8027C478213
:100CF000E34885F8A870204400F8017C4772E14879
:100D0000204400F8017CE048204400F8017CDF48E2
:100D100002EB040900EB041319F8010CDDF834C0F0
:100D200003EB400222F810CCA2F890B095F8C02056
:100D3000032A46D1C01D00F007008DF8207003EB98
:100D400040008DF8247030F8102C0D9BB0F8900006
:100D50009A1AABEB00030868018B5143028A91FB9E
:100D6000F2F10791418B408A594391FBF0FB08ABAC
:100D7000224601200799FFF7C7F8059009AB2246E4
:100D800059460220FFF7C0F803909DF820100798FD
:100D9000CDE9000121460120029B059AFFF7E9F801
:100DA0009DF82400DDE90232CDE900B021460220A1
:100DB000FFF7DFF8B0480599204400F8011C0399BB
:100DC000417219F8010C0122401CC0B209F8010C53
:100DD000082808D309F8017C9AF8A800002808BF61
:100DE0008AF8A82002E09AF8A80018B195F85800EF
:100DF000022809D085F8A870A148204400F8017C99
:100E000047720FB0BDE8F08FA04B0021084603EBFE
:100E1000041C0CEB4003401C33F8103C80B2194416
:100E20000828F6D34FEAD10A00210846E9460CEB20
:100E3000400333F8103CA3EB0A035B4349F820302E
:100E4000401C80B219440828F1D34FEAD109904BD5
:100E50000021084603EB041C0CEB4003401C33F854
:100E6000103C80B219440828F6D34FEAD10A002179
:100E70000846EB460CEB400333F8103CA3EB0A03A7
:100E80005B434BF82030401C80B219440828F1D352
:100E9000C80803234E4528BF864208D3754820441E
:100EA00010F8011C08299CBF407A082811D9754800
:100EB00085F8A830204400F8017C7348204400F8ED
:100EC000012C95F8A800032804BF0FB0BDE8F08FEF
:100ED00092E76C48204410F8011CC8293CBF491C0B
:100EE00000F8011C6849214411F8011C012908D1AE
:100EF00010F8010C40459EBF85F8A8300FB0BDE842
:100F0000F08F022085F8A80076E72DE9F04FAFB00A
:100F10000FFA81F9DDE9388C0124CA4669460028B8
:100F200048D032F81A002B90BCF1010011D441F8DE
:100F3000204001EB800632F81A503565AAF1010510
:100F40000FFA85FABAF1000FB8BFA8F1010A401EE6
:100F5000EDD5002425464846BCF101020FD433F8F4
:100F6000107051F82260401E7E43341900B245EBE8
:100F7000E6750028B8BFA8F10100521EEFD5002683
:100F80003746BCF101005DD401EB800233F819A0B3
:100F9000126DA9F1010902FB0AF296190FFA89F9FB
:100FA00047EBE277B9F1000FB8BFA8F10109401E85
:100FB000EAD547E033F81A002B90BCF1010011D4B8
:100FC00041F8204001EB800633F81A503565AAF14C
:100FD00001050FFA85FABAF1000FB8BFA8F1010AAE
:100FE000401EEDD5002425464846BCF101030FD430
:100FF00032F8107051F82360401E7E43341900B25D
:1010000045EBE6750028B8BFA8F101005B1EEFD5DF
:1010100000263746BCF1010014D401EB800332F8FE
:1010200019A01B6DA9F1010903FB0AF39E190FFA20
:1010300089F947EBE377B9F1000FB8BFA8F10109CF
:10104000401EEAD54FF000084046CDF8A080BCF124
:10105000000F24DD51F82020289B524312EB080892
:1010600043EBE27216E000006007002084070020D6
:10107000349D0020529D00203E9D0020669D002052
:101080008E9D0020A29D002094970020F49B0020BC
:10109000949C002000F1010028928445DADC0022B3
:1010A000964610462992BCF1000F11DD01EB80033A
:1010B00051F820201B6DDDF8A4905A434FEAE27AE4
:1010C00012EB0E0E4AEB0903401C29938445EDDC1C
:1010D0004FF00009CA464846BCF1000F0DDD01EB98
:1010E000800251F82030126D00F101005A4312EBDA
:1010F00009094AEBE27A8445F1DC00200346024606
:10110000BCF1000F0CDD694601EB8001096D49431C
:101110004FEAE17B8A184BEB0303401C8445F2DC69
:101120001046A8FB002C2899CDE92C0301FB00C038
:10113000AEFB09CB29992E9108FB030301FB09B1F2
:101140000EFB0A10B2EB0C0163EB0000CDE92901A4
:10115000084333D0DDE92C02A0FB0413AEFB06CB21
:1011600002FB04322E9B00FB052203FB06B30EFBA1
:101170000733B1EB0C0062EB0301DDE9293205F026
:10118000E9FE3A990860A8FB0602289901FB0621AE
:10119000A9FB04230AFB043308FB071109FB0533F1
:1011A000801A61EB03010904DDE9293241EA1041AB
:1011B000000405F0CFFE3A99486004E03A99002017
:1011C00008603A9948603A98D0E900122B98504349
:1011D00011EB204048BF00202FB0BDE8F08F70B564
:1011E000ADF5166D0E460546FDF7E2F80446FDF72F
:1011F000F0F84FF41661684605F071FF6A46314613
:10120000284605F05DFE0246E0736946284603F075
:1012100029FC20740DF5166D70BD0000F84A002001
:10122000411C1154C8B20528FAD37047F54910B5CE
:101230000020C1F88400C1F88800A1F88C0081F872
:101240008E00C1F89A00C1F89E00A1F8A20081F8B2
:10125000A400C1F88F00C1F89300A1F8970081F8AD
:1012600099000860486008818872C1F80B00C1F8D5
:101270000F00A1F81300487502F0CCF9E04A0020F5
:10128000411C1154C8B20528FAD310BDDC490844EA
:1012900010F8011C21F0800100F8011C70470020AB
:1012A000D74A0146535C13F0800F04D0491CC9B2E1
:1012B0000529F7D37047535C03F00F0043F0800318
:1012C0005354704770B50D460446FDF76FF8002380
:1012D0001A46A05CA95C884201D0012303E0501C9F
:1012E000C2B20A2AF5D3184670BD2DE9F0418AB082
:1012F00000200090019002900390049005900690C9
:1013000007900890FDF754F80446FDF762F805468B
:10131000FDF757F80746FDF767F80646FDF746F86C
:101320000346B4F90200B0F5FA7F7FDC94F8580266
:10133000012802D1607C002878D1A07A032818BF48
:10134000052873D094F85E02012804BF0AB0BDE8F6
:10135000F0810021207C4FF0010C002888BF0DF1A6
:10136000FF3813D901EB011000EB411007EB8002AD
:1013700092F8BF00022812BF032892F8590000F823
:1013800008C0481CC1B2207C8842EBD8297C0020D0
:10139000002988BF0DF10B0413D900EB001101EBFC
:1013A000401106EB810191F8BF20022A12BF032AE7
:1013B00091F8591001F804C0401C297CC0B2814248
:1013C000EBD8002006A933F92020002AC8BF01F875
:1013D00000C0401CC0B20A28F5D3687C002804BFB6
:1013E0000AB0BDE8F08193F8280003AC6D4608B35D
:1013F000FCF7DCFF00231846215C2A5C914204D1F3
:10140000401CC0B20A28F7D313B306AC6D46FCF7F4
:10141000CDFF00231846215C2A5C914206D1401C76
:10142000C0B20A28F7D300E000E08BB10AB0012077
:10143000BDE8F081FCF7BAFF00231846215C2A5C66
:101440009142F3D1401CC0B20A28F7D3002BEDD152
:101450000AB00020BDE8F0812DE9F0410026FCF73C
:10146000B0FF0746FCF7A4FF0446FCF79FFF0546C4
:10147000B4F90200B0F5CD7F06DD0221A172B0F50E
:10148000FA7FC4BF0120607394F85E0201281FBF79
:1014900094F85702012894F85A02012809D0FDF760
:1014A00023F830B9FDF74CF818B994F85802012820
:1014B00002D1FFF71AFF06460020411E25F8201032
:1014C00005EB8002401CC0B251800A28F6D3012EE1
:1014D00022D1207C002100281ED901EB011000EB55
:1014E000411007EB800090F8BF20022A18BF032AA2
:1014F0000DD190F85930C28805EB830323F8042CF2
:10150000028990F8590005EB800020F8022C481C55
:10151000C1B2207C8842E0D894F8580268B9002211
:101520003949002E08BF4A7007D04878401CC0B225
:101530004870052884BF4A70002685F82860304628
:10154000BDE8F0812DE9F05F30480025006890F893
:101550005260FCF753FFFCF72BFF0446FCF731FF0A
:101560008446B4F902004FEA600E207C002898BF40
:10157000BDE8F09F264B4FF0010B4FF0000A05EB42
:10158000051000EB45170CEB870191F85900401E40
:10159000C2B291F8BF00022802D0032854D040E024
:1015A00003EB420080F801A091F8AC00012836D08E
:1015B000B1F90200B0F5C87F31DC94F81480B8F1BD
:1015C000010F03D1B4F90280404528D1B4F902805B
:1015D00040451FD1B1F81880B4F80490C84519D11E
:1015E00003F812A081F8AEB0B1F90200C82818DAE9
:1015F0001CF82700002808BF81F8BCB011E00000EB
:10160000519E0020AC9D0020E007002060070020D4
:101610005B9E00207045C8BF03F812B022DC03F8BF
:10162000126013F8120040B303EB420013F812806B
:101630004778474516D380F801A003F812A081F837
:10164000ACA081F8ADB011E013F81200A8B1B4F964
:101650000200B0F5C87FE7DA03EB420047787F1C51
:101660004770E1E781F8ACB081F8ADA0681CC5B265
:10167000207CA84283D8BDE8F09F81F8ACA0F3E7B6
:1016800070B5FCF795FE0646FCF79BFE0546307CE0
:101690000024002814D904EB041000EB441005EBDF
:1016A000800090F8AF10012905D190F8590000286A
:1016B00018BF01F09DFF601CC4B2307CA042EAD884
:1016C000002070BD70B5FCF773FE0446FCF779FE90
:1016D000227C0021002A84BF4FF0020C032315D97D
:1016E00001EB011202EB411200EB820292F8AF50C3
:1016F000012D01BF92F8BF50022D82F8BF3082F851
:1017000058C0491C227CC9B28A42E9D8002070BD69
:101710002DE9F041FCF74CFE867AC57AFCF7A8FE6D
:10172000FCF7ACFE01F076FFFCF742FE0746FCF743
:1017300048FE8046387C0024002814D904EB0410AD
:1017400000EB441008EB800090F8AF10012905D1A0
:1017500090F85900002818BF01F04AFF601CC4B27D
:10176000387CA042EAD8FCF723FE0446FCF729FEA9
:101770008446207C0021002884BF0223032015D941
:1017800001EB011202EB41120CEB820292F8AF70F6
:10179000012F01BF92F8BF70022F82F8BF0082F8BC
:1017A0005830491C227CC9B28A42E9D8FCF700FEB5
:1017B0008672C572BDE8F08110B5FFF74DFE044694
:1017C000012804D0002C08BFFFF7BCFE01E0FFF7A2
:1017D0009FFF204610BD7047022180F86C10002248
:1017E000826680F864200121A0F86E1000EB4103AE
:1017F000491CC9B2A3F86E200929F7D3C388A0F801
:101800005C300189A0F85E10A0F86030A0F862108A
:1018100080F8B72080F8652070472DE9F047FCF785
:10182000F1FDFCF7C5FD0446FCF7CBFD0546FCF7D2
:10183000DBFD8046207C0023002898BFBDE8F087B0
:101840004FF00309012002264FF0040A002703EBA2
:10185000031101EB431105EB810191F85B2002EBD1
:10186000021C0CEB421208EB820C91F8AF20012A0B
:101870001BD191F8BD20012A18BF032A02D0022AE9
:1018800028D012E091F85820012A20D0022A0CD149
:101890009CF8BF20012A18BF042A18D0022A08BFCA
:1018A00081F8BF9001D081F8BF20227D012A08BFB6
:1018B00081F8B90091F85820022A04BF9CF8B92099
:1018C00081F8B92091F8BF20022A17D035E081F8BD
:1018D000BF60EAE791F85820012A04BF81F8BF00F1
:1018E00081F8B970E1D0022ADFD19CF8BF20022A2A
:1018F00014BF032A81F8BFA0D5D1D6E781F86C6068
:101900008F6681F86470A1F86E00012201EB420C31
:10191000521CD2B2ACF86E70092AF7D3B1F806C0E7
:10192000A1F85CC00A89A1F85E20A1F860C0A1F806
:10193000622081F8B77081F86570591CCBB2217CA8
:10194000994284D8BDE8F0872DE9F04714460F4648
:1019500080460025FCF72CFD0646FCF732FD81464B
:10196000FCF742FD0146002020706070307C0028AA
:1019700098BFBDE8F08705EB051000EB451009EBBB
:10198000800292F8AF00012822D192F85800022874
:1019900002D0012817D01BE092F86C00022817D063
:1019A00092F85B0000EB001202EB401001EB8000AC
:1019B00090F8BF0003280BD1207808F80050207859
:1019C000401C207004E060783D546078401C6070DA
:1019D000681CC5B2307CA842CDD8BDE8F0872DE99F
:1019E000F0471D4616460F460446FCF707FD94F8DF
:1019F00002C0E3780146634520D3227894F8019031
:101A00004FF0C0081046814512D30CFB0104A4B26C
:101A100017F804A038EA0A0A06D136F91440AC4295
:101A200002DB0120BDE8F087401CC0B28145ECD24A
:101A30000CF1010000F0FF0C6345E3D20020BDE88B
:101A4000F08770B50C460546FCF7BBFC05EB0511AD
:101A500001EB451100EB810204EB041101EB441191
:101A600000EB8100137B017B8B4288BF1173937B5A
:101A7000817B8B4238BF9173537B417B8B4288BF04
:101A80005173D37BC17B8B4238BFD173137C017CF4
:101A90008B4288BF1174937C817C8B4238BF9174D8
:101AA000537C417C8B4288BF5174D37CC17C8B4278
:101AB00038BFD174137D017D8B4288BF1175937D32
:101AC000817D8B4238BF9175537D417D8B4288BFAC
:101AD0005175D17DC07D814238BFD07570BD2DE973
:101AE000F041012516460F462C46FCF76AFC07EB31
:101AF000071101EB471100EB810106EB061202EB27
:101B0000461200EB82000B7D027D934284BF90F869
:101B100016C0634505D88B7D93423CBF827D9342BE
:101B200000D200254B7D427D934284BF90F817C0C0
:101B3000634505D8C97D91423CBFC07D814200D23A
:101B40000024002D16BF002C00200120BDE8F081EC
:101B50002DE9FF4F87B01F460E460546FCF731FCC6
:101B60000446FCF74BFC824605EB051000EB4510E4
:101B700004EB80090390B9F806000590B9F8080055
:101B8000049003984FF00008454614F82000029096
:101B900099F80110009101FB0A00B9F902200192A5
:101BA000385C00F03F0006900998002873D9705DFA
:101BB00000EB001101EB401014F8201004EB800042
:101BC0004278437B02FB0A11C07B795C984201F0AA
:101BD0003F0131D3705D00EB001202EB401004EBCB
:101BE0008000027B807B90421AD303FB0A201FFAFD
:101BF00080FC17F80C0000F03F0B8B451CBF4FF02A
:101C0000C00E3EEA000E7DD0501CC2B2705D00EBEB
